:1000000002CC33FFFFFFFFFFFFFFFF0267CDFFFFC3
:10002000FFFFFF0204C2FFFFFFFFFFFFFFFFFFFF15
:10004000FFFFFFFFFFFFFFFFFFFFFF02CB42FFFFAE
:10005000FFFFFF02CD31FFFFFFFFFF02CDEFFFFFEC
:10007000FF69FCFFFFFFFFFFFFFFFFFFFFFFFFFF29
:1000800090F009E4F090F008E4F002CC33FFFFFFB9
:10010000E4F5B875A890F54AF55EF55FF55CF55D28
:1001100090F0087406F0E4FFFE055DE55DAC5C70F0
:1001200002055C14F5828C83E493FD055FE55FAA0C
:100130005E7002055E14F5828A83EDF00FBF000148
:100140000EE4B507D4EEB420D090F0097402F0A309
:10015000E4F090F0097403F0E4F55EF55FF55CF50A
:100160005D7560BF90F00E74BFF012055A8F59E5AF
:1001700059B42E0B7E047F941203E2C2AF80FEE5D9
:100180006064C0F56090F00EF0E559B421031201EF
:100190009CC2AFD2AED2BED2AF80CF22E4F5541211
:1001A00003988F681203988F641203988F65E4F5A3
:1001B0006112039874412561F8A6070561E561C3E2
:1001C000940840EDE4F561120398744B2561F8A69C
:1001D000070561E561C3940840ED1203A1EF655482
:1001E00060067F6212052B22AF687401A8070880A1
:1001F00002C333D8FCF561554A706CC2AF90F00A67
:10020000E568F0C24312041050067F4512052B2208
:10021000D24312041050067F4512052B22E561429D
:100220004AE4F566F567C2AFD2AED2BED2AFF56191
:10023000E4F5620567E567AE667002056614F5824F
:100240008E83E0B4FFBD0567E567AE6670020566A4
:1002500014F5828E83E0B4FFAA0562E562B480D310
:100260000561E561B480C9C2AFD2AED2BEE564FE1D
:100270007C00E42565FFEC3EF5668F67E4F5619050
:10028000055574AAF09002AA7455F090055574A013
:10029000F074412561F8E6856782856683F085679D
:1002A00082856683E05480FF74412561F8E65480BE
:1002B000B507EB0567E567700205660561E561B4A2
:1002C00008BDE4F56190055574AAF09002AA745532
:1002D000F090055574A0F0744B2561F8E6856782AF
:1002E000856683F0856782856683E05480FF744B62
:1002F0002561F8E65480B507EB0567E567700205F0
:10030000660561E561B408BD74F02567F56774FFA3
:100310003566F566E4F5610567E567AE667002056A
:100320006614F5828E83E0FF74412561F8E6FEEFE6
:100330006E6016AF687401A807088002C333D8FC4A
:10034000F4524A7F6212052B220561E561C39408CD
:1003500040C5E4F5610567E567AE667002056614A1
:10036000F5828E83E0FF744B2561F8E6FEEF6E6048
:1003700016AF687401A807088002C333D8FCF45292
:100380004A7F6212052B220561E561C3940840C5CE
:10039000D2AF7F3F12052B221203A1EF2554F55453
:1003A00022E508700F3025F9C225C2AFD2AED2BE09
:1003B000D2AF80ED7400250CF582E434FDF583E0C6
:1003C000FFBF0D057800E214F2E50C04547FF50C34
:1003D000150822EF1FAC0670011E4C60040000805F
:1003E000F2227898EEF208EFF27898E2FE08E2F551
:1003F000828E83E49360181808E2FF2401F218E269
:100400003400F28F828E83E493FF12052B80DA2270
:1004100090055574AAF09002AA7455F09005557491
:1004200080F074AAF09002AA7455F030430890400E
:10043000007430F080069000007430F0D2AF90006D
:1004400000E05440FDE4F569D2AED2BE900000E079
:100450005440FF6D6012AD077FD07E071203D305B5
:1004600069E569C394C840E0E569C394C840097E62
:10047000047F9E1203E2D3227E047FB01203E2AF18
:100480006912058D7E047FBE1203E27F327E001268
:1004900003D3C3225265626F6F74210D0A0020449A
:1004A000656C6574652054696D656F75740D0A001F
:1004B0002044656C65746554696D653A2000200DB3
:1004C0000A00C0E0C083C082C0D0C000C00730981E
:1004D00029C298E508D3947F5020AF997400250A6B
:1004E000F582E434FDF583EFF0BF0D057800E204FA
:1004F000F2E50A04547FF50A0508309921C299E50E
:100500000960197480250DF582E434FDF583E0F56A
:1005100099E50D04547FF50D15098002D200D0072E
:10052000D000D0D0D082D083D0E032C3747F950980
:10053000C3940A40F6E509D3947F501D7480250BBF
:10054000F582E434FDF583EFF0E50B04547FF50B01
:100550000509300004C200D29922E5086027740022
:10056000250CF582E434FDF583E0FFFEBF0D057830
:1005700000E214F2E50C04547FF50C1508EE640A51
:1005800060D8AF06227F00227800E2FF22AE07EE9D
:10059000C4540F9005D093FF12052BEE540F900515
:1005A000D093FF12052B2212055AEF541F24E1F5B8
:1005B00082E43405F583E493C454F0FD12055AEF48
:1005C000541F24E1F582E43405F583E4932DFF22E2
:1005D0003031323334353637383941424344454679
:1005E00000000A0B0C0D0E0F0000000000000000C0
:1005F0000000010203040506070809E478A0F6904C
:10060000F00CF07557FCA374FCF008F6A3F090F022
:1006100001E054A7783AF2E47857F290F00BF0C278
:10062000AFF5A8F5B8758680D2AED2BED224C2B5D9
:100630000090F00A04F090F008E4F01281EC7E00E3
:100640007FE07D007B027AEC790012D0607E007F33
:10065000E07D007B027AED790012D060759204751E
:1006600083F0758201E4F592C28C438901758CF5A3
:10067000758A95D28C75C84575C10A75A90C75B96E
:1006800004C2C27F0B128F4412973643B11075908B
:100690002353B1EF12CAC412828775B80675A892A7
:1006A00090F001E030E00C783AE230E703127FA0EE
:1006B000127D39128122126D7912B2FF7B057A996F
:1006C00079FAE4FD1283277B057A9A79077D101267
:1006D00083277B057A9C79D87D1912832775192584
:1006E00075180112959FC224754B35754C01E4F5C0
:1006F0004D20210312519BE47801F2781BE660073C
:10070000D24412527A80F47FA87E611203D3C2AF22
:10071000D2AED2BED2AF7801E204F2E2C3940A4074
:10072000DA128273E47876F208F2780174FFF278D4
:1007300003740AF2087432F27882740CF27802744C
:1007400019F2C2AFD2AED2BED2AF90ECE07403F0D9
:100750007834E2A3F0A374FFF0E4A3F0A374FFF0F5
:10076000E490ECE9F090ECE8F0203D0612998D124F
:100770003426781BE67003302A05D24412527A12CE
:100780000588EF60642021611208F87887E66480AC
:1007900070030208ED301A511282737B057A9A7940
:1007A00012E4FD1283277B057A9A791B7D10128350
:1007B000277E9A7F241203E21296FDE55744FCF54A
:1007C0005790F00DF0E478A1F6A3F0D214D24512C0
:1007D000955BC2AFD2AED2BED2AF7FA87E6112030C
:1007E000D37F06129736120100303505127703C207
:1007F000357884E6FF70030207697885E630E411F6
:10080000EFD39401400B785CE2FEEFD39E4002EF01
:10081000F2788416787608E22401FFF218E23400B8
:10082000FEF2BE031EBF201BE4F208F2D245129571
:100830005B7882E2600D14F270099091C0F012C8EA
:10084000A9D2367877E2B4900818E2B40103129482
:10085000997801E2600A14F2700674FFF2127911BD
:10086000202164789FE6600E16E6700A780D74FF0A
:10087000F27F0D12052B7802E2600A14F270067402
:1008800019F2127B5A7804E2603414F27030740466
:10089000F27885E630E10578047428F230420712D8
:1008A000ADEDC2428018D242909150E0FEA3E0FF2D
:1008B000122BD0909173E0FEA3E0FF122BD01232E6
:1008C0001F302B0312413D7803E2600B14F27007D6
:1008D00012924B7803EFF2202503020769C22575B7
:1008E000A0FCC2AFD2AED2BED2AF0207697E9A7F61
:1008F000301203E212981022C24330330412C311A3
:100900002212055A8F59E4F552F553F554E559640E
:1009100063600BE55964766005E559B46905D24317
:100920005359DFE5596443604BE55964566045E52A
:1009300059644C603FE55964576039E559644F602C
:1009400033755A0912055A744B255AF8EFF6640D9F
:100950006007155AE55AB4FFEBE55AB4FF161205C5
:100960005A7867EFF2640D600B12055AEF640D6060
:1009700003022925E55924BFB41A00400302291BAC
:10098000900987F82828730211840216090209D5F4
:10099000020B840226F102165B020A2A02293F0298
:1009A0000D2402293F021BB102260E021D32021E37
:1009B000EB020A26021F2C022418022418021FFC34
:1009C00002293F02204F022490020A370211270217
:1009D000293F020B3F7885E620E30302293F1205F9
:1009E000A78F4B1205A78F4CE54C540FF559E4F532
:1009F0005BE55BC39559500E1205A7744D255BF856
:100A0000A607055B80EB304319534C0F78E07CEC74
:100A10007D027B047A00794B7E007F0A12CF68D278
:100A20002A2212519B2212C64A227885E620E3032D
:100A300002293F12C41B2212055AEF24BD601E2456
:100A4000FA601624E07003020B0B24FA604D242098
:100A50006003020B3F12C1992212C26E2212055A84
:100A6000EF644C600302293F12055AEF64456003AE
:100A700002293F12055AEF6441600302293F120523
:100A80005AEF6452600302293FD22212B2FFC222FF
:100A90007F2A12052B7F0D12052B22D207E4F55A6F
:100AA000E55A541F7005780BF208F275F02CE55AE0
:100AB000A4240DF582E5F0344EAF82F55E8F5F7FA2
:100AC0005712052B7F6912052BAF5A12058DE4F5DD
:100AD00059855F82855E83E0FF12058DE55F240105
:100AE000FFE4355EF55E8F5F0559E559C3942840F4
:100AF000E0E509D3943F50F97F0D12052B7F0A12D0
:100B0000052B055AE55A7098C20722D207E4780BE4
:100B1000F208F2F55A1205A78F54E554655A60F5AC
:100B20007E9A7F3B1203E2754B35754C01754D0D76
:100B300012519B12519B12519BD2AED2BE80FEE449
:100B4000F559301E0343590120140343590230095B
:100B5000034359043022097885E630E303435908FA
:100B6000435980789CE6FF30E103435920EF30E29F
:100B7000034359107F5A12052BAF5912058D7F0D73
:100B800012052B22E554646F7023E553B4771EE5FC
:100B900052B46E19E551B46C14E550B46F0FE54FC3
:100BA000B4610AE54EB46405D21A022925E55464FD
:100BB00065702BE55364627025E552B45F20E55102
:100BC000B4451BE550B46D16E54FB47011E54EB455
:100BD000660CE54DB4210778877680022925E55417
:100BE00064656003020C8BE55364626003020C8B46
:100BF0007F0D12052B7F0A12052B7F07122B5878C9
:100C000085A6077887A6507F04122B587887A607F9
:100C10007885E6FF12058D7887E6FF12058D785CF2
:100C2000E2D3940140207F2012052B7F4212052B36
:100C30007F4712052B7F5412052B785CE2FF1205CB
:100C40008D785C7401F27F0D12052B7F0A12052B43
:100C50007885E620E70302293FC2AFE4F5C8F5C175
:100C6000C290C291D2AED2BE7F0A7E001203D3D20E
:100C7000907F057E001203D3D29100000000C29045
:100C80007F087E001203D3C29180D9E55464657059
:100C900040E553645A703A7F0D12052B7F0A120506
:100CA0002B7F07122B587881EFF27F05122B587893
:100CB0004DEFF27881E2FF12058D7F2012052B782F
:100CC0004DE2FF12058D7F0D12052B7F0A12052BB9
:100CD000227885E6700302293F7F0D12052B7F0ADB
:100CE00012052B7885E6FF12058D7887E6FF120541
:100CF0008D785CE2D3940140207F2012052B7F4247
:100D000012052B7F4712052B7F5412052B785CE2CE
:100D1000FF12058D785C7401F27F0D12052B7F0A9E
:100D200012052B227885E620E30302293FE4F559DA
:100D3000F55DD207E554640D700302109F7F091220
:100D40002B588F5AE55A541F7005780BF208F2E5BC
:100D500009D3942050F975F02CE55AA42418F58293
:100D6000E5F0344EF583E0FF12058D75F02CE55A61
:100D7000A4241AF582E5F0344EF583E054C0F55909
:100D800030E6077F6E12052B8011E55930E7077FAB
:100D90006D12052B80057F7A12052B75F02CE55A14
:100DA000A4240DF582E5F0344EF583E04430FF12C3
:100DB000052B7F2012052B75F02CE55AA4241EF577
:100DC00082E5F0344EF583E0FF12058D75F02CE5D9
:100DD0005AA4241DF582E5F0344EF583E0FF120598
:100DE0008D7F2012052B204303020F4375F02CE565
:100DF0005AA42409F582E5F0344EF583E0FEA3E021
:100E0000AA06F97B02126C8875F02CE55AA4240B13
:100E1000F582E5F0344EF583E0FEA3E0AA06F97B07
:100E200002126C887E9A7F431203E275F02CE55A19
:100E3000A42419F582E5F0344EF583E0FF12058D08
:100E40007E9A7F471203E275F02CE55AA4241AF526
:100E500082E5F0344EF583E0FF12058D7E9A7F4BDC
:100E60001203E275F02CE55AA4241BF582E5F03458
:100E70004EF583E0FF12058D7E9A7F4F1203E275D7
:100E8000F02CE55AA4241CF582E5F0344EF583E0FD
:100E9000FF12058D7E9A7F531203E275F02CE55AFE
:100EA000A4241FF582E5F0344EF583E0FF12058D92
:100EB0007E9A7F4F1203E275F02CE55AA42420F5A8
:100EC00082E5F0344EF583E0FF12058D7E9A7F5760
:100ED0001203E275F02CE55AA42421F582E5F034E2
:100EE0004EF583E0FF12058D7E9A7F5B1203E2755B
:100EF000F02CE55AA42422F582E5F0344EF583E087
:100F0000FF12058D7E9A7F5F1203E275F02CE55A81
:100F1000A42423F582E5F0344EF583E0FF12058D1D
:100F20007E9A7F5F1203E275F02CE55AA42424F523
:100F300082E5F0344EF583E0FF12058D7E9A7F63E3
:100F40001203E27F07122B58055AEF655A6003021D
:100F50000D44E550640D700302109CE4F559755A78
:100F600001E559C39405400302109CE559B40403FC
:100F7000E4F55AE509D3942050F97E9A7F6612036E
:100F8000E275F007E55AA42449F582E5F03491F5BD
:100F900083E0FEA3E0AA06F97B02126C8875F007D5
:100FA000E55AA4244BF582E5F03491F583E0FEA3E5
:100FB000E0AA06F97B02126C8875F007E55AA424B2
:100FC0004EF582E5F03491F583E0FEA3E0AA06F940
:100FD0007B02126C8875F007E55AA4244DF582E572
:100FE000F03491F583E064AA601A7F2112052B7515
:100FF000F007E55AA4244DF582E5F03491F583E03D
:10100000FF12058D7E9A7F6A1203E275F007E55A9A
:10101000A4246CF582E5F03491F583E0FEA3E0AA08
:1010200006F97B02126C8875F007E55AA4246EF568
:1010300082E5F03491F583E0FEA3E0AA06F97B0295
:10104000126C8875F007E55AA42471F582E5F03436
:1010500091F583E0FEA3E0AA06F97B02126C887585
:10106000F007E55AA42470F582E5F03491F583E0A9
:1010700064AA601A7F2112052B75F007E55AA42493
:1010800070F582E5F03491F583E0FF12058D7E9ACC
:101090007F631203E20559055A020F61C20722E578
:1010A00009D3943F50F9E559540F70147F0D120580
:1010B0002B7F0A12052BAF5912058D7F3A12052B93
:1010C0007F2012052BAF5D055DA807E6FF12058D99
:1010D0000559E55970C97F0D12052B7F0A12052BA2
:1010E000E4F559F55DE509D3943F50F9E559540FFE
:1010F00070147F0D12052B7F0A12052BAF591205B4
:101100008D7F3A12052B7F2012052BA85DE2FF127E
:10111000058D055D0559E55970CB7F0D12052B7FB7
:101120000A12052BC207227885E620E30302293F35
:10113000E554B40D08E47884F208F2801EE554B456
:10114000620B78847400F2087418F2800EE554B4CF
:1011500061097884744EF2087409F27884E2FE081A
:10116000E2FF12052B7884E2FF12052B788408E257
:10117000FF2401F218E2FE3400F28F828E83E0FF3A
:1011800012052B22E552640D60030212D57F411235
:10119000052B7F09122B588F5912058D75F02CE500
:1011A00059A42409F582E5F0344EAF82F5608F61D1
:1011B000F583E5822411F582E43583F583E054C09C
:1011C00060087E9A7F6E1203E222E5612410F582A8
:1011D000E43560F583E030E712E561241AF582E436
:1011E0003560F583E0FF12058D8049E561240BF53C
:1011F00082E43560F583E0540FF559E5612413F579
:1012000082E43560F583E0FF30E003435910E56187
:101210002410F582E43560F583E0FE30E0034359A5
:1012200020EF30E203435940EE30E303435980AFEF
:101230005912058DE5612415F582E43560F583E0EA
:101240005407FF25E025E0FFE5612416F582E4352B
:1012500060F583E05430FEC4540F4FF559E5612426
:1012600013F582E43560F583E0FF30E30343592052
:10127000EF30E403435940EF30E503435980AF5961
:1012800012058DE5612415F582E43560F583E0FFF4
:10129000C454F0FE25E025E0FEEF54304EF559FF32
:1012A00012058DE4F559E561240EF582E43560F50B
:1012B00083E030E503435901E5612410F582E4350C
:1012C00060F583E030E703435902AF5912058D7F83
:1012D0000D12052B22E553644D600BE553644E60FF
:1012E00005E553B45A097F07122B588F5980077FA1
:1012F00008122B588F59E553644D6009E553644E2D
:1013000060030213A4E554645760030213A47F41F1
:1013100012052BE4F54BE553B44D2AE559C394402F
:10132000400302293F75F005E559A42409F582E53B
:10133000F03490AF82F5648F657F5712052B7F4D97
:1013400012052B804475F00BE559A42409F582E5BC
:10135000F0347AAF82F5648F657F05122B58EF3039
:10136000E70EE42565F565740B3564F564754B800F
:10137000856582856483A3A3E030E003434B017F4E
:101380005712052B7F4E12052BAF5912058DAF4B0F
:1013900012058D856582856483E0FF12058D7F0DC2
:1013A00012052B2275F02CE559A42409F582E5F0ED
:1013B000344EAF82F5608F61F583E5822411F582AA
:1013C000E43583F583E0F55154C0F5398F82E58229
:1013D0002410F582E43560F583E0F54B30E7317F8A
:1013E0004112052B7F5712052BE539600302293F77
:1013F0007F5A12052BAF5912058DE561241AF5822B
:10140000E43560F583E0FF12058D7F0D12052B2278
:10141000E539B44015E559D3947F400EAF61AE6015
:10142000AD59122B72400302293F7F4112052B7FD9
:101430004612052BE561240BF582E43560F583E067
:10144000F552E53970087F5A12052B53520FE539D2
:10145000644070337F4E12052BE551540CFFBF08DA
:1014600010E5521313543FF552D3941C40037552A8
:101470001CE551540CFFBF040EE552131313541F07
:10148000F552B40F021552E539B480187F4D12059C
:101490002BE552131313541FF55253520FE552B458
:1014A0000F021552AF5912058DAF5212058DE4F59A
:1014B00059E54B30E103435901E54B30E203435911
:1014C00002E551540CFFBF0403435904BF08034312
:1014D0005908BF0C0343590CE5612413F582E43528
:1014E00060F583E0FF30E003435910E54B30E00343
:1014F000435920E5397007EF30E203435940E5399D
:10150000B44012E5612411F582E43560F583E030E2
:10151000E103435940E54B30E303435980AF59128F
:10152000058DE5612413F582E43560F583E0FFC3A2
:1015300013F559E561241AF582E43560F583E0304E
:10154000E003435980AF5912058DE5612417F582F8
:10155000E43560F583E0FF12058DE539706FE561D4
:101560002415F582E43560F583E05407FF25E02576
:10157000E0FFE5612416F582E43560F583E0543040
:10158000FEC4540F4FF559E5612413F582E435602C
:10159000F583E0FF30E303435920EF30E403435980
:1015A00040EF30E503435980AF5912058DE56124C2
:1015B00015F582E43560F583E0FFC454F0FE25E0C4
:1015C00025E0FEEF54304EF559FF12058DE4F55934
:1015D000E561240EF582E43560F583E030E50343F0
:1015E0005901AF5912058DE539B44017E561241A48
:1015F000F582E43560F583E0FFC313F559540FFF1E
:1016000012058D7F0D12052B221229408F5975F07E
:101610002CEFA42409F582E5F0344EAF82F5608FFB
:1016200061FEAD59122999500302293FE539B440B2
:1016300015E559D3947F400EAF61AE60AD59122BC2
:1016400072400302293F7F07122B58E5612417F5EA
:1016500082E43560F583EFF0021CB7C244122940E2
:101660008F5975F02CEFA42409F582E5F0344EAFC4
:1016700082F5608F61FEAD59122999500302293F0E
:10168000E539B44015E559D3947F400EAF61AE60A3
:10169000AD59122B72400302293F7F07122B588F3E
:1016A000547F05122B588F59E55930E411E5612418
:1016B00013F582E43560F583E04401F0800FE561C5
:1016C0002413F582E43560F583E054FEF0E55930EB
:1016D000E511E5612410F582E43560F583E044010D
:1016E000F0800FE5612410F582E43560F583E05465
:1016F000FEF0E5396440704FE5612410F582E43571
:1017000060F583E0FF5408FEE5595480FD6E6014D7
:10171000D244E5612411F582E43560F583E030E1DF
:1017200003435B10ED6011E5612410F582E4356040
:10173000F583EF4408F0800FE5612410F582E4356D
:1017400060F583EF54F7F0E5612410F582E435602D
:10175000F583E0547FF04440F0E55930E011E56155
:101760002410F582E43560F583E04402F0800FE553
:10177000612410F582E43560F583E054FDF0E5590D
:1017800030E111E5612410F582E43560F583E04431
:1017900004F0800FE5612410F582E43560F583E004
:1017A00054FBF0E539644060030218447F03122BB8
:1017B000588F5AE561241AF582E43560F583E0FF1D
:1017C00030E733E5612413F582E43560F583E0FE0C
:1017D000C313F55CEF30E003435C80E55A655C6061
:1017E00015E561240FF582E43560F583E0FFAD5C1B
:1017F000129758435B02E5612413F582E43560F5E6
:1018000083E05401F0E5612413F582E43560F5834B
:10181000E0FFE55A25E0FEEF4EF07F01122B58EF76
:10182000540FFF25E0F54EE55A30E703434E01E53E
:1018300061241AF582E43560F583E054E0F0454E0A
:10184000F0435B07E5612410F582E43560F583E041
:1018500030E014E561240AF582E43560F583E02088
:10186000E0057411F0D243E5612410F582E435609F
:10187000F583E020E014E561240AF582E43560F5A3
:1018800083E030E0057412F0D243E5396440706DB6
:1018900053590CE5612411F582E43560F583E0F5D8
:1018A00051E559600A5351F34251E551F08006E584
:1018B00051540CF559E559B40409E554C454F0F5F4
:1018C00054801BE559B4080BE55433333354F8F511
:1018D00054800BE559B40C06E55425E0F554E56158
:1018E0002420F582E43560F583E0455BF0E5612472
:1018F00008F582E43560F5837402F08049E53964C7
:1019000080703C53590CE5612411F582E43560F593
:1019100083E0F551E559600A5351F34251E551F026
:101920008006E551540CF559E554C454F0F554E5DE
:10193000612408F582E43560F583740AF08007E5D8
:1019400054C454F0F554E5612412F582E43560F591
:1019500083E554F0E5612416F582E43560F583E013
:10196000540FC454F0FFE561240CF582E43560F5B2
:1019700083E0540F2FF0E561240EF582E43560F525
:1019800083E0FF20E61D4440F0754B34754C22E5A2
:1019900061240FF582E43560F583E0F54DE4F54E02
:1019A00012519BE5612404F582E43560F583E0641F
:1019B000016009AF61AE607D01124E0D754B42753D
:1019C0004C06E561240FF582E43560F583E0F54DC2
:1019D000E5612410F582E43560F583E0F54EE561BC
:1019E0002411F582E43560F583E0F54FE561240BC1
:1019F000F582E43560F583E0F550E5612413F58266
:101A0000E43560F583E0F551E561241AF582E435AB
:101A100060F583E0F55212519BE5612411F582E4F3
:101A20003560F583E020E003021BA1E5612410F599
:101A300082E43560F583E0F55A85605E85615FE498
:101A4000F559E55F2406F582E4355EF583E0FEA3F3
:101A5000E08E5EF55F4E700302293FE55F656170C1
:101A600004E55E6560700302293FE55F2411F5829D
:101A7000E4355EF583E020E00302293FE55F2410B2
:101A8000F582E4355EF583E054D1FFF0E55A542E3B
:101A90004FF0E55F2412F582E4355EF583E554F0FE
:101AA000E561240CF582E43560F583E0FFE55F2411
:101AB0000CF582E4355EF583EFF0E5612417F582DD
:101AC000E43560F583E0FFE55F2417F582E4355ED9
:101AD000F583EFF0E55F2420F582E4355EF583E0E1
:101AE0004401F030442DE55F2420F582E4355EF5B5
:101AF00083C083C082E0FFE55F2411F582E4355E98
:101B0000F583E030E1047E1080027E04EF4ED08247
:101B1000D083F0304326E55F2410F582E4355EF58E
:101B200083E06401F0E55F240AF582E4355EF58325
:101B3000E030E0057412F080037411F0E55F2404D6
:101B4000F582E4355EF583E064016018AF5FAE5E58
:101B50007D01124E0DE55F240EF582E4355EF583BE
:101B6000E04440F0E55F2411F582E4355EF583E062
:101B700054C0FFBF8010E55F2408F582E4355EF5B0
:101B800083740AF0800EE55F2408F582E4355EF583
:101B9000837402F00559E559C394085003021A42B0
:101BA00022E5612406F582E43560F583E4F0A3F0D4
:101BB000227F09122B588F5975F02CEFA42409F5B8
:101BC00082E5F0344EAF82F5608F61F583E58224C3
:101BD00011F582E43583F583E054C0600302293FA8
:101BE0007F07122B588F59E5612416F582E4356082
:101BF000F583E0540FFFE5595403C454F04FF0E56A
:101C0000612415F582E43560F583E054F0FFE55971
:101C1000541CFE1313543F4FFFE5612415F582E475
:101C20003560F583EFF0E55930E511E5612413F5F2
:101C300082E43560F583E04408F0800FE561241309
:101C4000F582E43560F583E054F7F0E55930E611AC
:101C5000E5612413F582E43560F583E04410F080FB
:101C60000FE5612413F582E43560F583E054EFF06D
:101C7000E55930E711E5612413F582E43560F58319
:101C8000E04420F0800FE5612413F582E43560F52F
:101C900083E054DFF07F05122B588F59E559C413A8
:101CA000135403FFE55954304FFFE5612415F582C5
:101CB000E43560F583EFF0E561240EF582E43560EC
:101CC000F583E0FF20E61D4440F0754B34754C224F
:101CD000E561240FF582E43560F583E0F54DE4F528
:101CE0004E12519BE5612404F582E43560F583E0F2
:101CF00064016009AF61AE607D01124E0DE56124A3
:101D000008F582E43560F5837408F0754B43F54CB3
:101D1000E561240FF582E43560F583E0F54D7F4EF3
:101D2000E5612413FDE43560FC7B0712CBF812510A
:101D30009B22E550B40D1B7F09122B588F5975F06B
:101D40002CEFA42409F582E5F0344EAF82F5608FC4
:101D500061221229408F59E5397003021ECB3006EB
:101D6000157F3F12052B7F3F12052B7F3F12052B5E
:101D70007F0D12052B227F07122B588F5AE55A54DC
:101D800007909F5793F54BE55A30E008E54BC31396
:101D9000F54C8006E54B25E0F54CE5396480705E36
:101DA000535A0F789CE620E20302293FE559D39469
:101DB00050400302293F7895A65AE559C3944050F4
:101DC0002E78427404F2786AE559F275F005A4247D
:101DD00009F582E5F03490AF82F5648F65E55A30FD
:101DE000E30D856483E0454BFFF0E54CF45FF0D2F2
:101DF000237899A65978837404F2E47892F6E53949
:101E00006440600302293F789CE620E10302293FF9
:101E1000C22378837404F2E47892F6D206E55A304D
:101E2000E004D2178002C217786AE559F275F00B08
:101E3000A42409F582E5F0347AAF82F5648F65E574
:101E400059543F44807899F6E5591313543F543060
:101E500044807895F6E55A30E71878427401F2E448
:101E60002565F565740B3564F5647895E64440F6B0
:101E70008004E47842F2E55A540F789546F664708F
:101E8000F6E55A30E335856582856483A3A3E030A7
:101E9000E00B856582856483E0454BF02285658291
:101EA000856483E0454BFF7850F2E54CF45FF278AF
:101EB00036E564F208E565F2D227228565828564FD
:101EC00083E0FFE54BF4FEEF5EF02275F02CE55960
:101ED000A42409F582E5F0344EAF82F5608F61FEEF
:101EE000AD59122999400302293F227F09122B582C
:101EF0008F597F07122B588F5AE550640D600302EB
:101F0000293FE559D3943F400302293FE5594480D6
:101F1000F54BE55A30E709754CA1545FF54D800843
:101F2000754CC0780DE559F212519B221229408F51
:101F30005975F02CEFA42409F582E5F0344EAF82F8
:101F4000F5608F617F07122B588F59E559C4540FE4
:101F50004259E5612419F582E43560F583E559F0CD
:101F6000E5595411600C90918FE560F0A3E561F0A4
:101F7000801390918FE0B5600CA3E0B56107E49009
:101F8000918FF0A3F0E5595422600C909195E56093
:101F9000F0A3E561F08013909195E0B5600CA3E0AB
:101FA000B56107E4909195F0A3F0E5595444600CB5
:101FB00090919BE560F0A3E561F0801390919BE028
:101FC000B5600CA3E0B56107E490919BF0A3F0E548
:101FD000595488600D9091A1E560F0A3E561F0028D
:101FE0001CB79091A1E065607004A3E06561600397
:101FF000021CB79091A1F0A3F0021CB7E55424BFD6
:10200000602424FC603024F2600302293F301E0368
:1020100002293F30140302293FD21E78887441F20E
:10202000C24512955B22D214C20C1296FD1296CBB9
:10203000C24512955B22C21EC214C209C20CC20361
:102040001296F21296BDC24512955B12973422C2C7
:10205000441229408F5975F02CEFA42409F582E52C
:10206000F0344EAF82F5608F61FEAD591229995060
:102070000302293FE539B44015E559D3947F400E5A
:10208000AF61AE60AD59122B72400302293F7F074A
:10209000122B588F59E55930E00FE5612410F58275
:1020A000E43560F583E06402F0E55930E10FE56165
:1020B0002410F582E43560F583E06404F0E55930DE
:1020C000E40FE5612413F582E43560F583E06401F3
:1020D000F0E55930E511E5612410F582E43560F54D
:1020E00083E06401F0D243E5396440703DE5593046
:1020F000E728E5612410F582E43560F583E06408A3
:10210000F0E5612411F582E43560F583E030E10A01
:10211000D244E55930E603435B10E5612408F582BB
:10212000E43560F5837402F0800EE5612408F582E1
:10213000E43560F583740AF0E550640D7003022104
:10214000D17F05122B588F59E559603AE561241A61
:10215000F582E43560F583E0FF30E72AE56124137A
:10216000F582E43560F583E0FEC313F55BEF30E004
:1021700003435B80E561240FF582E43560F583E07D
:10218000FFAD5B129758E5612413F582E43560F5E5
:1021900083E0FFE55925E0FEEF6EF0E55930E70FEB
:1021A000E561241AF582E43560F583E06401F07F8F
:1021B00003122B588F59E55925E0F559E561241A8A
:1021C000F582E43560F583E0FFE559541EFEEF6EBD
:1021D000F0304317E561240AF582E43560F583E0C9
:1021E00030E0057412F080037411F0E561240EF5FF
:1021F00082E43560F583E0FF20E61D4440F0754B36
:1022000034754C22E561240FF582E43560F583E0F6
:10221000F54DE4F54E12519BE5612404F582E43559
:1022200060F583E064016009AF61AE607D01124E2C
:102230000D754B42754C06E561240FF582E435605F
:10224000F583E0F54DE5612410F582E43560F58312
:10225000E0F54EE5612411F582E43560F583E0F5A3
:102260004FE561240BF582E43560F583E0F550E538
:10227000612413F582E43560F583E0F551E56124CE
:102280001AF582E43560F583E0F55212519BE56161
:102290002411F582E43560F583E020E00302240890
:1022A000E5612410F582E43560F583E0F55A856038
:1022B0005E85615FE4F559E55F2406F582E4355EED
:1022C000F583E0FEA3E08E5EF55F4E700302293FCA
:1022D000E55F65617004E55E6560700302293FE5B6
:1022E0005F2411F582E4355EF583E020E0030229E6
:1022F0003FE55F2410F582E4355EF583E054D1FFBD
:10230000F0E55A542E4FF0E561240CF582E4356077
:10231000F583E0FFE55F240CF582E4355EF583EF9D
:10232000F0E5612417F582E43560F583E0FFE55FB1
:102330002417F582E4355EF583EFF0E55F2420F5A0
:1023400082E4355EF583E04401F030442DE55F24FE
:1023500020F582E4355EF583C083C082E0FFE55F4F
:102360002411F582E4355EF583E030E1047E1080CF
:10237000027E04EF4ED082D083F0304326E55F2406
:1023800010F582E4355EF583E06401F0E55F240A30
:10239000F582E4355EF583E030E0057412F08003E9
:1023A0007411F0E55F2404F582E4355EF583E064A2
:1023B000016018AF5FAE5E7D01124E0DE55F240E29
:1023C000F582E4355EF583E04440F0E55F2411F5E5
:1023D00082E4355EF583E054C0FFBF8010E55F24E2
:1023E00008F582E4355EF583740AF0800EE55F241B
:1023F00008F582E4355EF5837402F00559E559C3AA
:10240000940850030222B722E5612406F582E435E0
:1024100060F583E4F0A3F022E554B44510C218300F
:10242000290475320922C22BC202D22622E559B4F0
:102430005205753721800375373F1229408F59E5C2
:1024400039700302293FE53964807027855935E5E5
:10245000376421600302293F7537553029057532ED
:102460000F8017D229E4F5327F05122B58786CEFD4
:10247000F28007E55914F535D22B7F07122B588FC0
:102480003A754B35754C01754D0512519BD218228A
:102490007885E620E20302293F20430A90ECE874A5
:1024A000FFF0A3F0800DE490ECE8F01205A790ECAB
:1024B000E9EFF01205A78F5AE55A704A7F691205B5
:1024C0002B90ECE9E0FF12058D7F6312052B90EC59
:1024D000E0E0FFF55A12058DE4F559E559C3955A28
:1024E00050197F2012052B74E02559F582E434EC55
:1024F000F583E0FF12058D055980E07F0D12052B55
:102500007F0A12052B22855A311205A78F34120536
:10251000A78F3B1205A78F3E1205A78F3F1205A775
:102520008F40E534653BF53DE531C394044004E557
:102530003E623DE531C394054004E53F623DE5312F
:10254000C394064004E540623D7F6912052B90EC80
:10255000E9E0FF12058D7F2012052B7F6312052B0A
:10256000AF3112058D7F2012052B7F6112052BAF35
:102570003412058D7F2012052B7F6412052BAF3B93
:1025800012058D7F2012052B90ECE0E531F0A3744D
:1025900033F0A3E534F0A3E53BF0A3E53DF0E531EE
:1025A000C3940440197F4412052BAF3E12058D7F62
:1025B0002012052B90ECE4E53EF0A3E53DF0E5317B
:1025C000C3940540197F4412052BAF3F12058D7F40
:1025D0002012052B90ECE5E53FF0A3E53DF0E53159
:1025E000C3940640197F4412052BAF4012058D7F1E
:1025F0002012052B90ECE6E540F0A3E53DF0AF3D61
:1026000012058D7F0D12052B7F0A12052B22301922
:102610001312055A8F5AEF6003B40DF57E9A7F7836
:102620001203E2221205A78F4E7897E66023E53861
:10263000654E601D12055A8F5AEF6003B40DF57E8A
:102640009A7F7D1203E2AF3812058D7F0D12052BA4
:10265000221205A78F4FE54F7019F5387897F612BB
:10266000055A8F5AEF700302293F640D7003022947
:102670003F80ECE54F5407F54BD39405401312050A
:102680005A8F5AEF6003B40DF57E9A7F811203E2F0
:1026900022E4F55AE55AC3954B50151205A774A2CA
:1026A000255AF8EFF67450255AF8A607055A80E423
:1026B00012055AEF640D60087E9A7F811203E222B0
:1026C000E54F30E706789776FF8004E47897F67850
:1026D00098A64BE54F131313541F54077890F685B3
:1026E0004E38D219754B45754C08754D1412519BD7
:1026F000227F4512052B7F09122B588F5A7F071214
:102700002B588F59E55A701CE559C3947850157FA2
:102710000312058DAF5A12058DAF5912058D7F0D2D
:1027200012052B22E55A44C0F543855944E4F55B74
:102730007554FF755C8075F02CE55CA4241DF58252
:10274000E5F0344EF583E0B5432B75F02CE55CA441
:10275000241EF582E5F0344EF583E0B5441775F09C
:102760002CE55CA42409F582E5F0344EAF82F560D7
:102770008F61022859E554604175F02CE55CA42472
:102780000DF582E5F0344EF583E0FFF552BF090800
:10279000855C5BE4F5548022E552701E75F02CE5F3
:1027A0005CA42427F582E5F0344EF583E0F553C3AD
:1027B00095545006855C5B855354055CE55C60036D
:1027C000022736E55B7003022906F55C75F02CA440
:1027D0002409F582E5F0344EAF82F5608F61F58310
:1027E000E582240AF582E43583F583E4F0E561248B
:1027F0000DF582E43560F583E4F0E5612414F5829B
:10280000E43560F583E543F0E5612415F582E435B0
:1028100060F583E544F0E561240CF582E43560F56C
:1028200083E4F0E5612412F582E43560F583E4F099
:10283000E561240BF582E43560F583E4F0E561247D
:1028400011F582E43560F5837448F0E5612410F5F4
:1028500082E43560F5837440F0E5612404F582E498
:102860003560F583E064097053788606E5612404D9
:10287000F582E43560F5837404F0756291756365E3
:10288000AE62AF63AD61AC601250A0E5632405F5A4
:1028900082E43562F583E0FEA3E0B5631FEEB56226
:1028A0001B856382856283E0FEA3E0FFE563240568
:1028B000F582E43562F583EEF0A3EFF0AF5C12052C
:1028C0008DAF5A12058DAF5912058D7F0D12052B54
:1028D000E5612404F582E43560F583E0F55A64018E
:1028E0006015E55A6402600FE55A64036009AF6140
:1028F000AE607D04124E0DE561241EF582E4356064
:10290000F58374FFF022E4FF12058DAF5A12058D96
:10291000AF5912058D7F0D12052B227885E66005D3
:10292000AF5912052B120588EF601412055A8F5902
:10293000EF640D600A7885E660EB12052B80E622D5
:10294000E554B44E05753940801BE554B44D05750A
:1029500039808011E554B45A05E4F5398007780EC2
:10296000E2F5398020855354855253855152855064
:1029700051854F50854E4F854D4E854C4D854B4C66
:102980007867E2F54BE554541F9005E193C454F089
:10299000FFE553541F932FFF228E668F678F828E21
:1029A00083E5822411F582E43583F583E054C0F594
:1029B0006AB53902C322E539B48008EDC3945140A9
:1029C00002D322E539B4400B783DE2FFEDD39F40BE
:1029D00002D322E567240AF582E43566F583E4F044
:1029E000E567240BF582E43566F583E4F0E56724BA
:1029F00012F582E43566F583E4F0E567240DF5828F
:102A0000E43566F583E4F0E567240CF582E4356689
:102A1000F583E4F07887E630E1267F5712052BAF87
:102A20006A12058DE5672411F582E43566F583E0C9
:102A300054C0FF12058D7F0D12052B7F0A12052B46
:102A4000AF67AE661250F7E56AB44023788616E5A4
:102A5000672404F582E43566F583E075F007A42465
:102A600049F582E5F03491AF82F5688F698021786D
:102A70009316E5672404F582E43566F583E075F086
:102A800007A4246CF582E5F03491AF82F5688F6974
:102A9000E5692405F582E43568F583E0FEA3E0FFEF
:102AA000B5670BEEB56607AD69AC68124FE2E56736
:102AB0002411F582E43566F583E0543FF04539F0A2
:102AC000E5672404F582E43566F5837404F0E5399E
:102AD000B4401D788606E5672411F582E43566F575
:102AE00083E054F3F04408F0756891756965801BC4
:102AF000E5672411F582E43566F583E054F3F0448C
:102B000008F0756891756988789306AE68AF69AD0D
:102B100067AC661250A0E5692405F582E43568F5D6
:102B200083E0FEA3E0B5691FEEB5681B8569828569
:102B30006883E0FEA3E0FFE5692405F582E43568DB
:102B4000F583EEF0A3EFF0E567240EF582E4356639
:102B5000F583E054BFF0C322744B2FF8E6541F9066
:102B600005E193C454F0FE744A2FF8E6541F932EE7
:102B7000FF228E668F678D687F4512052BE56724DF
:102B800004F582E43566F583E0B409117F0512058A
:102B90008DAF6812058D7F0D12052BC322E4FF1245
:102BA000058DAF6812058DE5672414F582E435665E
:102BB000F583E0543FFF12058DE5672415F582E4A7
:102BC0003566F583E0FF12058D7F0D12052BD322AC
:102BD0008E598F5A8F828E83E5822404F582E435E4
:102BE00083F583E06401600302321EE55A2405F593
:102BF00082E43559F583E064A560030231FDE55AAE
:102C00002410F582E43559F583E030E7030231FD05
:102C10007885E620E103022CB1E55A240FF582E421
:102C20003559F583E0FF12058D7F7312052BE55AA8
:102C3000240AF582E43559F583E0FF12058D7F6D96
:102C400012052BE55A2410F582E43559F583E0FF8F
:102C500012058D7F6112052BE55A240BF582E435B0
:102C600059F583E0FF12058D7F7312052BE55A2479
:102C700012F582E43559F583E0FF12058D7F63126A
:102C8000052BE55A240DF582E43559F583E0FF1252
:102C9000058D7F6912052BE55A240CF582E4355920
:102CA000F583E0FF12058D7F0D12052B7F0A1205BB
:102CB0002BE55A2410F582E43559F583E0FF30E521
:102CC00048E55A240BF582E43559F583E4F0E55ADA
:102CD0002412F582E43559F583E4F0E55A240DF524
:102CE00082E43559F583E4F0E55A240CF582E435A5
:102CF00059F583E054F0F0E55A240AF582E4355999
:102D0000F583E05407F00231FDE55A2411F582E421
:102D10003559F583E0FE755D0F54C0FDBD4012EEE0
:102D2000540CFDBD0805755D078006BD0C03755D7F
:102D300002E55A240CF582E43559F583E0F55BE5AC
:102D40005A2417F582E43559F583E0FEE55A240B41
:102D5000F582E43559F583E0F55CEF20E103530695
:102D60000FEF20E2035306F0E55A240AF582E4351A
:102D700059F583E0540FB4100040030231A2902DA6
:102D800085F8282873022DC5022EB5022F4B022D7F
:102D9000C5022F9E023052023106023155022DB576
:102DA000022EB5022F4B022DB5022F9E0230520289
:102DB0003106023155EE540F7003430601EE54F014
:102DC0007003430610E55A2412F582E43559F58361
:102DD000E0F9C313FFE55CC39F5060E55A240DF58D
:102DE00082E43559F583E0FD14F0ED60030231A271
:102DF0007408255CF55CE55A2412F582E43559F532
:102E000083E0FDC313FDE55CD39D40028D5C535B05
:102E1000F0E55C131313541F425BEEC4540FFDE541
:102E20005B909CF693FCED8CF0A4FDE55A240DF527
:102E300082E43559F583EDF00231A2E55CD39F4081
:102E400062E55A240DF582E43559F583E0FF14F06C
:102E5000EF60030231A274F8255CF55CE55A241298
:102E6000F582E43559F583E0FFC313FFE55CC39FAA
:102E70004005E55C30E7028F5C535BF0E55C1313C3
:102E800013541F425BE55B909CF693FFEE540F8F4B
:102E9000F0A4FFE55A240DF582E43559F583EFF0EF
:102EA0000231A2E55A240AF582E43559F583E0544B
:102EB00007F00231FDE55C7037E55A2412F582E433
:102EC0003559F583E0D3955D4006780AE2FF80022C
:102ED0007F00E55A240DF582E43559F583EFF0E5DE
:102EE0005A240AF582E43559F5837415F00231A2AB
:102EF000E55A240DF582E43559F583E0FF14F0EF2F
:102F000060030231A2EE540F7003430601EE54F049
:102F1000700343061074F8255CF55C30E703E4F5B4
:102F20005C535BF0E55C131313541F425BE55B904D
:102F30009CF693FFEE540F8FF0A4FFE55A240DF595
:102F400082E43559F583EFF00231A2E55C7037E594
:102F50005A2412F582E43559F583E0D3955D400695
:102F6000780AE2FF80027F00E55A240DF582E435FD
:102F700059F583EFF0E55A240AF582E43559F583D3
:102F80007414F00231A2E55A240DF582E43559F5A6
:102F900083E0FF14F0EF60030231A2022F05E55A2F
:102FA000240DF582E43559F583E0FF14F0EF60035A
:102FB0000231A2E55A241CF582E43559F583E0601C
:102FC00014E014F0E55A240DF582E43559F58374C4
:102FD0007DF00231A2E55A2412F582E43559F583D9
:102FE000E0D3955D40067809E2FF80027F00E55A54
:102FF000240DF582E43559F583EFF0E55A240AF5FE
:1030000082E43559F5837416F0E55A240EF582E40E
:103010003559F583E054FDF0E55A2410F582E43586
:1030200059F583E054EEF0754B35754C03754D043E
:10303000E55A240FF582E43559F583E0F54EE55A5B
:103040002410F582E43559F583E0F54F12519B02C7
:1030500031A2E55A240DF582E43559F583E0FF14D9
:10306000F0EF60030231A2E55A241CF582E43559E1
:10307000F583E06014E014F0E55A240DF582E435A0
:1030800059F583747DF00231A2E55A2412F582E4E9
:103090003559F583E0D3955D40067809E2FF80025B
:1030A0007F00E55A240DF582E43559F583EFF0E50C
:1030B0005A240AF582E43559F5837417F0E55A2449
:1030C0000EF582E43559F583E04402F0E55A241008
:1030D000F582E43559F583E04411F0754B35754CB4
:1030E00003754D04E55A240FF582E43559F583E064
:1030F000F54EE55A2410F582E43559F583E0F54F95
:1031000012519B0231A2E55A240DF582E43559F59E
:1031100083E07031E55A241DF582E43559F583E0EA
:103120006013E014F0E55A240DF582E43559F58377
:10313000747DF0806DE55A240AF582E43559F583F3
:103140007418F0805DE55A240DF582E43559F58355
:10315000E014F0804DE55A240DF582E43559F583ED
:10316000E07031E55A241DF582E43559F583E060BD
:1031700013E014F0E55A240DF582E43559F5837413
:103180007DF0801EE55A240AF582E43559F58374F2
:103190001BF0800EE55A240DF582E43559F583E0E5
:1031A00014F0E55A240CF582E43559F583E55BF01B
:1031B000E55A240BF582E43559F583E55CF0E55AD0
:1031C0002420F582E43559F583E04401F0E55A24E2
:1031D00011F582E43559F583E054C0FFBF8010E556
:1031E0005A2408F582E43559F583740AF0800EE517
:1031F0005A2408F582E43559F5837402F0855A8221
:10320000855983E0FEA3E08E59F55A8E832404F598
:1032100082E43583F583E064017003022BEB222204
:10322000789DE6FF75F02CA42409F582E5F0344E74
:10323000AD82F5598D5AF583E5822411F582E43586
:1032400083F583E0543070030232C58D82E5822419
:103250001AF582E43559F583E004F054037066757D
:103260004B35754C02754D098F4E12519B80567827
:103270009DE6FF75F02CA42409F582E5F0344EADEF
:1032800082F5598D5AF583E5822411F582E4358360
:10329000F583E05430602E8D82E582241AF582E4B5
:1032A0003559F583E0D39402400E754B35754C02C9
:1032B000754D0A8F4E12519BE55A241AF582E4355A
:1032C00059F583E4F0E4789AF6228E5C8F5DED7018
:1032D00003023425E55D2419F582E4355CF583E0CD
:1032E0005D6010E55D2410F582E4355CF583E03027
:1032F000E01322E55D2410F582E4355CF583E020DF
:10330000E003023425754B35754C03754D04855C1F
:103310005E855D5FE4F560E55F2410F582E4355E6F
:10332000F583E06401F0E55F240AF582E4355EF59B
:1033300083E030E0057412F080037411F0E55D2441
:103340001CF582E4355CF583E0FFE55F241CF58223
:10335000E4355EF583EFF0E55D241DF582E4355C30
:10336000F583E0FFE55F241DF582E4355EF583EF2C
:10337000F0E55F2404F582E4355EF583E0640160E6
:1033800048AF5FAE5E7D01124E0DE55F2420F582F1
:10339000E4355EF583E04401F0E55F2411F582E455
:1033A000355EF583E054C0FFBF8010E55F2408F56B
:1033B00082E4355EF583740AF0800EE55F2408F53B
:1033C00082E4355EF5837402F0E55F240FF582E454
:1033D000355EF583E0F54EE55F2410F582E4355E59
:1033E000F583E0F54F12519BE55F2406F582E43545
:1033F0005EF583E0FEA3E08E5EF55F4E6027E55F3D
:10340000655D7004E55E655C601BE55F2411F58217
:10341000E4355EF583E030E00C0560E560C39408B8
:10342000500302331722302103023F1E301B06C215
:103430001B128A19227885E630E255E4F55274E0D1
:103440002552F582E434ECF583E0FF74782552F8D8
:10345000EFF20552E552B408E590ECE9E0FF90EC9C
:10346000E8E0FE04F0EEC39F501D787C74FFF27814
:103470007AF2E4787BF278787403F2A3E0B4FF0C7C
:10348000E490ECE8F08005E490ECE8F012851C2272
:103490007887E630E203D38001C3924330064520AB
:1034A0002942202B3F789206E6C39405403630230C
:1034B000117899E6FF7895E6FD1289D57892760322
:1034C0008014302702D21F7899E6FF7895E6FD1226
:1034D0008501E47892F67883E214F26003023F1EDD
:1034E000129784227886E67003023B69300B030250
:1034F0003B697893E66002D20B20190302357C30D9
:10350000290302357C202B7430206FC2207898E686
:10351000FF047878F27834E27879F278A2E6FE78DF
:103520007AF278A3E6FD787BF2EE6D787CF2EFD349
:103530009402403978A4E6FE787CE26E787DF278D9
:103540007CEEF2EFD39403402478A5E6FE787DE28A
:103550006E787EF2787DEEF2EFD39404400F78A679
:10356000E6FF787EE26F787FF2787EEFF212851CBC
:103570007890E67003023F1E1622D2203019287878
:1035800090E67003D38001C3501DC219754B357589
:103590004C03754D1485384E754FFF7897E67004CF
:1035A000F54FF53812519BC2447897E6600616E64F
:1035B0007002F53830431F7E9A7F861203E2E53CA5
:1035C000909ED793FF12058D7E9A7F8E1203E2782C
:1035D00094E6FF12058D7843E2700302366B755C4A
:1035E00001E4F55BE55BC39404400302366B78436A
:1035F000E2FF555C606AE55CF4FEEF5EF2747225F2
:103600005BF8E275F02CA42409F582E5F0344EAFA6
:1036100082F5598F5AF583E5822413F582E43583C8
:10362000F583E0FF7D80541CFEC3134205E55A2458
:103630001AF582E43559F583E030E603430501EFDE
:1036400030E015E55A2411F582E43559F583E0544C
:103650000C64046003430510AF5AAE591284232250
:10366000055BE55C25E0F55C0235E4E53C909ED722
:10367000937003023ACC24FE700302378014700367
:103680000238AB1470030239D624036003023EBB38
:103690003043057F2112052B909155E0FEA3E08E6B
:1036A00059F55A2404F582E43EF583E06401600391
:1036B00002377A30430AAF5AAE597D61FB123F1F81
:1036C000E55A2405F582E43559F583E064A56017D1
:1036D000AF5AAE597D39125143AF5AAE597C917DE4
:1036E00050124FE202377A30041CE55A240FF5825B
:1036F000E43559F583E0FF7894E6B50703D38001FC
:10370000C35003023780E5386010E55A240FF58274
:10371000E43559F583E065386066AF5AAE59124713
:10372000A9AF5AAE597C917D50124FE2E55A240858
:10373000F582E43559F583E06006E014F0023EBB03
:10374000E55A240AF582E43559F583E030E40302B2
:103750003EBBAF5AAE597D02124E0DE55A2408F514
:1037600082E43559F5837402F0E55A2409F582E4C0
:103770003559F5837419F0023EBB2044030238AB7F
:103780003043057F2212052B90915CE0FEA3E08E72
:1037900059F55A2404F582E43EF583E0640260039F
:1037A0000238AB30430AAF5AAE597D61FB123F1F5E
:1037B000E55A2405F582E43559F583E064A56017E0
:1037C000AF5AAE597D41125143AF5AAE597C917DEB
:1037D00057124FE20238AB204413E55A2408F58211
:1037E000E43559F583E024FF40030238A030041C7F
:1037F000E55A240FF582E43559F583E0FF7894E625
:10380000B50703D38001C350030238ABE53860131A
:10381000E55A240FF582E43559F583E065387003E5
:103820000238ABAF5AAE591247A9AF5AAE597C9184
:103830007D57124FE220440EE55A2408F582E43504
:1038400059F583E014F0E55A2409F582E43559F579
:1038500083E06003023EBBAF5AAE597D03124E0DAA
:10386000E55A240FF582E43559F583E0D3947F407F
:103870000EE55A241EF582E43559F58374FFF0E510
:103880005A2411F582E43559F583E054CFF0E55A16
:10389000240EF582E43559F583E054DFF0023EBB97
:1038A000AF5AAE597C917D57124FE23043057F24C9
:1038B00012052B909163E0FEA3E08E59F55A240483
:1038C000F582E43EF583E0640360030239D63043B9
:1038D0000AAF5AAE597D61FB123F1FE55A2405F528
:1038E00082E43559F583E064A56017AF5AAE597D7F
:1038F00042125143AF5AAE597C917D5E124FE202A3
:1039000039D6204413E55A2408F582E43559F58365
:10391000E024FF40030239CB30041CE55A240FF5A4
:1039200082E43559F583E0FF7894E6B50703D38048
:1039300001C350030239D6E5386013E55A240FF568
:1039400082E43559F583E0653870030239D6AF5A01
:10395000AE591247A9AF5AAE597C917D5E124FE223
:1039600020440EE55A2408F582E43559F583E01425
:10397000F0E55A240FF582E43559F583E0D3947FBE
:103980005003023EBBE55A241EF582E43559F58307
:10399000E07003023EBB7851E230E003023EBBE53B
:1039A0005A241EF582E43559F583E014F0600302D1
:1039B0003EBBAF5AAE59FD124E0DE55A241EF5829C
:1039C000E43559F58374FFF0023EBBAF5AAE597C23
:1039D000917D5E124FE23043057F2512052B9091B9
:1039E0006AE0FEA3E08E59F55A2404F582E43EF520
:1039F00083E064046003023ACC30430AAF5AAE5904
:103A00007D61FB123F1FE55A2405F582E43559F527
:103A100083E064A56017AF5AAE597D43125143AF9E
:103A20005AAE597C917D65124FE2023ACC30041CAB
:103A3000E55A240FF582E43559F583E0FF7894E6E2
:103A4000B50703D38001C35003023ACCE5386010B8
:103A5000E55A240FF582E43559F583E06538606C4A
:103A6000AF5AAE591247A9AF5AAE597C917D651233
:103A70004FE2E55A240FF582E43559F583E0D394FB
:103A80007F5003023EBBE55A241EF582E43559F50A
:103A900083E07003023EBB7851E230E003023EBB9C
:103AA000E55A241EF582E43559F583E014F06003ED
:103AB000023EBBAF5AAE59FD124E0DE55A241EF51B
:103AC00082E43559F58374FFF0023EBB3043057F35
:103AD0002612052B90914EE0FEA3E08E59F55A2454
:103AE00004F582E43EF583E0706D30430AAF5AAED0
:103AF000597D61FB123F1FE55A2405F582E43559D3
:103B0000F583E064A5600BAF5AAE597D4412514372
:103B10008037300419E55A240FF582E43559F583CE
:103B2000E0FF7894E6B50703D38001C34029E53868
:103B30006010E55A240FF582E43559F583E06538C5
:103B40006015AF5AAE591247A9AF5AAE597C917D54
:103B500049124FE2023EBB204405D2440236907F18
:103B6000FFE4FD128501023EBBC20B7893E67003B1
:103B7000023EBBC24430431F7E9A7F921203E2E5AD
:103B80003C909ED793FF12058D7E9A7F8E1203E2A2
:103B90007894E6FF12058DE53C909ED79370030262
:103BA0003E5624FE7003023C82147003023D5514FD
:103BB0007003023DEF24036003023EB53043057FEE
:103BC0002112052B909178E0FEA3E08E59F55A243E
:103BD00004F582E43EF583E064016003023C723048
:103BE000430AAF5AAE597D61FB123F1FE55A2405C7
:103BF000F582E43559F583E064A56016AF5AAE59F5
:103C00007D45125143AF5AAE597C917D73124FE2FC
:103C10008060AF5AAE59124BC7AF5AAE597C917DF6
:103C200073124FE2E55A2408F582E43559F583E032
:103C30006006E014F0023EB5E55A240AF582E43548
:103C400059F583E030E403023EB5AF5AAE597D0228
:103C5000124E0DE55A2408F582E43559F5837402B5
:103C6000F0E55A2409F582E43559F5837419F00218
:103C70003EB520440D301D05C21D023D55D21D022A
:103C80003DEF3043057F2212052B90917FE0FEA38C
:103C9000E08E59F55A2404F582E43EF583E064028F
:103CA0006003023D5530430AAF5AAE597D61FB12A5
:103CB0003F1FE55A2405F582E43559F583E064A5F4
:103CC0006017AF5AAE597D46125143AF5AAE597C78
:103CD000917D7A124FE2023D55204410E55A2408A6
:103CE000F582E43559F583E024FF505EAF5AAE59B2
:103CF000124BC7AF5AAE597C917D7A124FE22044E5
:103D00000EE55A2408F582E43559F583E014F0E510
:103D10005A2409F582E43559F583E06003023EB583
:103D2000AF5AAE597D03124E0DE55A2411F582E4C7
:103D30003559F583E054CFF0E55A240EF582E43589
:103D400059F583E054DFF0023EB5AF5AAE597C918D
:103D50007D7A124FE23043057F2412052B90918625
:103D6000E0FEA3E08E59F55A2404F582E43EF58383
:103D7000E06403707A30430AAF5AAE597D61FB129A
:103D80003F1FE55A2405F582E43559F583E064A523
:103D90006016AF5AAE597D47125143AF5AAE597CA7
:103DA000917D81124FE28047204410E55A2408F5A6
:103DB00082E43559F583E024FF5029AF5AAE5912F9
:103DC0004BC7AF5AAE597C917D81124FE23044030C
:103DD000023EB5E55A2408F582E43559F583E0142E
:103DE000F0023EB5AF5AAE597C917D81124FE23060
:103DF00043057F2512052B90918DE0FEA3E08E599F
:103E0000F55A2404F582E43EF583E06404704730FB
:103E1000430AAF5AAE597D61FB123F1FE55A240594
:103E2000F582E43559F583E064A56016AF5AAE59C2
:103E30007D48125143AF5AAE597C917D88124FE2B2
:103E40008014AF5AAE59124BC7AF5AAE597C917D10
:103E500088124FE2805F3043057F2612052B909138
:103E600071E0FEA3E08E59F55A2404F582E43EF594
:103E700083E0703C30430AAF5AAE597D61FB123F7C
:103E80001FE55A2405F582E43559F583E064A56001
:103E90000BAF5AAE597D491251438007AF5AAE5904
:103EA000124BC7AF5AAE597C917D6C124FE2800520
:103EB000D244023BBC789CE620E163053C533C7F46
:103EC000E53C704A788306E6C39480500276807899
:103ED00083E6FF75F02CA4240DF582E5F0344EF551
:103EE00083E0702A75F02CEFA42427F582E5F034E6
:103EF0004EF583E060187851E220E01275F02CEF67
:103F0000A42427F582E5F0344EF583E014F078869A
:103F1000E66003123F877893E66003124062228EC8
:103F20005D8F5E8D5F8B607F2012052BAF5F12056A
:103F30002BE55E240FF582E4355DF583E0FF120585
:103F40008DE55E2404F582E4355DF583E0FF12051E
:103F50008DE55E2408F582E4355DF583E0FF12050A
:103F60008DE55E2409F582E4355DF583E0FF1205F9
:103F70008DE560B40110E55E2411F582E4355DF550
:103F800083E0FF12058D22E53C540F70709091572D
:103F9000E0FEA3E08E5DF55E2404F582E43EF58349
:103FA000E064027058E55E2405F582E4355DF58332
:103FB000E064A5600BAF5EAE5D7D4A125143803D6B
:103FC000E55E2408F582E4355DF5837402F0E55E74
:103FD0002409F582E4355DF583E06003E014F085A3
:103FE0005E82855D83E0FEA3E08E5DF55E8E8324B8
:103FF00004F582E43583F583E0640260A8E53C546F
:104000001F705E90915EE0FEA3E08E5DF55E24047D
:10401000F582E43EF583E064037046E55E2405F531
:1040200082E4355DF583E064A5600AAF5EAE5D7D38
:104030004B12514322E55E2408F582E4355DF58399
:104040007402F0855E82855D83E0FEA3E08E5DF5FF
:104050005E8E832404F582E43583F583E064036097
:10406000BA22E53C540F707090917AE0FEA3E08E86
:104070005DF55E2404F582E43EF583E06402705849
:10408000E55E2405F582E4355DF583E064A5600B0B
:10409000AF5EAE5D7D4C125143803DE55E2408F578
:1040A00082E4355DF5837402F0E55E2409F582E46F
:1040B000355DF583E06003E014F0855E82855D8305
:1040C000E0FEA3E08E5DF55E8E832404F582E43588
:1040D00083F583E0640260A8E53C541F705E909114
:1040E00081E0FEA3E08E5DF55E2404F582E43EF5FA
:1040F00083E064037046E55E2405F582E4355DF5F2
:1041000083E064A5600AAF5EAE5D7D4D125143222F
:10411000E55E2408F582E4355DF5837402F0855E82
:1041200082855D83E0FEA3E08E5DF55E8E832404D0
:10413000F582E43583F583E0640360BA227885E68E
:1041400030E403D38001C39243301604D212D21359
:10415000C244127C29500D7890E264026006D24479
:10416000127C29221282737B057A9A799AE4FD12D5
:1041700083273043077E9A7FAB1203E23013081285
:1041800096B27819742DF2E4FFFD1287B3129729C5
:10419000E47887F2F5567884F6F532202B0302474F
:1041A0000130250AC225C2AFD2AED2BED2AF781B33
:1041B000E66043C24412527A7885E630E627E5414C
:1041C00064466005E541B44703204319AF41120539
:1041D0008DAF4212058DAF4312058D7F0D12052B59
:1041E0007F0A12052BE541B4450CE543B40507757C
:1041F000320AE47884F6300C15786E7402F230439B
:10420000077E9A7FB61203E275320502466EE532EA
:10421000B40E00508690421CF828287302424602D1
:10422000427A0242D102463F02452102466E0243D3
:10423000A802419B02448F0246990246C90245CD1D
:1042400002419B0242EB12970830132B7884E6C39D
:10425000940A40F8E47884F630430C7887E27007DB
:104260007E9A7FC41203E27881E2FF7887E204F24B
:10427000C39F500302419B7532013043077E9A7FF2
:10428000CE1203E2E4F556786E74FFF2E53764521D
:104290007026FF7D011287B37819747CF27B057A52
:1042A0009A79DC7D101283273043077E9A7FE612CD
:1042B00003E275320302419B1296A77819747CF2CF
:1042C0003043077E9A7FF51203E2E47884F6753274
:1042D00002784DE2FFE556C39F500302419B3043F5
:1042E000077E9A7FFF1203E275320D7F06C24412E9
:1042F0007D12789BA6073043137E9B7F0A1203E250
:10430000789BE6FF12058D7F0A12052B789BE6D37A
:104310009499402A786E7402F23043077E9B7F1492
:104320001203E2789BE6C394FE5005E537B43F0ED6
:104330001296B27819742DF275320502466E789B8A
:10434000741E26F67B057A9B79267D10128327E55D
:10435000352401FFE433FEE4FD1283677B057A9B7D
:1043600079297D16128327E537B43F137829743FE6
:10437000F2753EE07F78AD357BE01287CE80117814
:10438000297421F2853A3E7F7CAD35AB3A1287CE57
:104390003043077E9B7F2E1203E2E4F5567896F6B3
:1043A0007889F6D208753206E556C3940A403AE594
:1043B00037B43F1CE53E20E317433E087F78AD3518
:1043C000AB3E1287CEE4F5567896F6D20802419BB2
:1043D0003043077E9B7F3F1203E2E4FFFD1287B369
:1043E000E4F55675320802419B7896E6C394045072
:1043F0000302419B3043197F4912052BAF5612052A
:104400008D7F2012052BAFD912058D7F2012052B31
:10441000E537643F7054E53E30E3125407FF740102
:10442000A807088002C333D8FC788946F6533EF7C4
:10443000754B35754C02754D067889E6F54E12516F
:104440009B78917617AF357E00E4FD128367E53ED9
:1044500064E76016053E7F78AD35AB3E1287CEE44B
:10446000F5567896F6D20802419BE537B4210585CA
:104470003A4F80057889E6F54F754C03754D0785F1
:10448000354E124721E47884F6753209024699E5E3
:1044900056C39407500302419BE535D3940740056A
:1044A000E535B41C06E53564047037E537643F70C4
:1044B00022F53EF5567896F6D2087F74AD35AB3EC0
:1044C0001287CE3043077E9B7F5F1203E275320B6B
:1044D00002419B786EE2B4FF037409F27532050263
:1044E000466EE535B41C057534748006E5354470B8
:1044F000F534E537B43F05E4F53B80064334788571
:104500003A3B3043077E9B7F751203E2E4F5567811
:1045100096F6D208AF34AD3B1287B3753204024130
:104520009BE556B401047888A63BE537B43F047F89
:104530000980027F0BEF65567045E537643F7030A8
:10454000053BE53B602A78917617FF7E00E4FD127B
:104550008367754B35754C02754D06853B4E125180
:104560009BE4F556D208AF34AD3B1287B302419BB2
:10457000786EE2B4FF037404F275320502466E7879
:1045800096E6C39404500302419B30431B7E9B7FFD
:10459000871203E2AF5612058D7F4912052BAFD962
:1045A00012058D7F0A12052B754C03754D07853555
:1045B0004EE537B42105853A4F80057888E6F54FFA
:1045C000124721E47884F6753209024699E556B41B
:1045D00001047888A63EE556C39406403D053EE5B5
:1045E0003E602C78917611FF7E00E4FD12836775A2
:1045F0004B35754C02754D06853E4E12519BE4F5C8
:1046000056D208AF34AD3BAB3E1287CE02419B7809
:104610006E7404F275320502419B7896E6C39404E9
:10462000500302419B754C03754D0785354E7888C4
:10463000E6F54F124721E47884F6753209805AE591
:1046400056D3940140031296A7E556C394505003E5
:1046500002419B754B35754C03754D07E4F54EF5DE
:104660004F12519BE47884F675320902419B304326
:10467000137E9B7F8D1203E2786EE2FF12058D7F21
:104680000A12052B754C02754D08786EE2F54E1234
:104690004721E47884F67532091296D6500F7819BE
:1046A000742DF27884E6C394C8500F80F67819749C
:1046B0002DF27884E6C3941E40F83043077E9B7F3A
:1046C000951203E2C22B02419B1296D6500F781925
:1046D000742DF27884E6C394C8500F80F67819746C
:1046E0002DF27884E6C3941E40F83043077E9B7F0A
:1046F0009F1203E2C22BD226C202E47890F202415A
:104700009B3016051296B280031296A71297137863
:10471000447414F23043077E9B7FAC1203E2C2BBA9
:1047200022754B353018307F5112052B7F4E120504
:104730002BE54DB40809786EE2FF12058D8005E483
:10474000FF12058DE53504FF12058DAF4F12058D63
:104750007F0A12052B800312519B7885E630E41DF9
:104760007E9B7FB51203E2E53504FF12058D7F2C99
:1047700012052BAF4F12058D7F0A12052BE54DB4A4
:1047800008197B057A9B79BE7D1012832778917674
:1047900016AF4E7E00E4FD1283672278917617AF44
:1047A0004F7E00E4FD128367228E5D8F5E8F828EC6
:1047B00083E582240FF582E43583F583E0F55F30ED
:1047C00029030249DD302B030249DDE55E2405F5AE
:1047D00082E4355DF583E064A5600AAF5EAE5D7D81
:1047E0004F12514322E55E2411F582E4355DF583D5
:1047F000E054C0FFBF800AAF5EAE5D7D50125143F2
:10480000227887E630E20C7E9B7FC91203E2AF5F1D
:1048100012058D301E0AE4FF7888E2FD1285012220
:10482000E55E2410F582E4355DF583E030E7087F2E
:10483000FFE4FD128501227894A65FE55F70030214
:1048400049DD7859E2655F7039E55E240EF582E452
:10485000355DF583E0A2E19241E55E240BF582E44B
:10486000355DF583E0547FF560C4540FF518E560BD
:10487000C454F0F51974252519F51974013518F586
:104880001822E55E2404F582E4355DF583E06401D9
:104890006003024965E55E2408F582E4355DF58331
:1048A000E0F561E55E2420F582E4355DF583E0F511
:1048B0006230E016AF5EAE5D124AA2E561D39401AC
:1048C00040030249DD5362FE8073E56230E116AFBA
:1048D0005EAE5D1249F5E561D3940140030249DD06
:1048E0005362FD8058E56230E216AF5EAE5D124A5B
:1048F00045E561D3940140030249DD5362FB803DED
:10490000E56230E316AF5EAE5D124A8BE561D3948B
:104910000140030249DD5362F78022E56230E4166C
:10492000AF5EAE5D1249DEE561D3940140030249FA
:10493000DD5362EF8007AF5EAE5D124AA2E56254BE
:104940001F60047F0380027F00E55E2408F582E497
:10495000355DF583EFF0E55E2420F582E4355DF505
:1049600083E562F022E55E241FF582E4355DF58380
:10497000E014601914602214603F1460482404702D
:104980004EAF5EAE5D124AA27560018042AF5EAE70
:104990005D1249F57560028036AF5EAE5D124A4524
:1049A000E55E2411F582E4355DF583E030E1047FB6
:1049B0000380027F008F608016AF5EAE5D124A8B6F
:1049C000756004800AAF5EAE5D1249DEE4F560E515
:1049D0005E241FF582E4355DF583E560F0227D3EBF
:1049E000E4FBEF2410F582E43EF583E030E3027B44
:1049F0008012848622EF241AF582E43EF583E0FCDF
:104A0000EF2413F582E43EF583E0FB7D80EC30E794
:104A100011EB541CFAC3134205EC30E60D430501BB
:104A20008008EB541EFCC3134205EB30E013EF2467
:104A300011F582E43EF583E0540C64046003430501
:104A40001012842322EF2413F582E43EF583E07DE7
:104A5000A054E0FCC41354074205EF241AF582E485
:104A60003EF583E030E003430508EF2411F582E4CE
:104A70003EF583E020E10DEF2410F582E43EF5835E
:104A8000E030E30343051012842322EF241AF58259
:104A9000E43EF583E07DA0541EFCC313420512845E
:104AA00023228E638F648F828E83E5822411F582A8
:104AB000E43583F583E0F5678F828E83E582240BEE
:104AC000F582E43583F583E0F5688F828E83E58295
:104AD000240EF582E43583F583E0F5698F828E83B9
:104AE000E5822413F582E43583F583E0F56AE56712
:104AF000540C640C704375653F8F828E83E582246D
:104B000010F582E43583F583E030E50575660180B4
:104B100014E568547FF566D394004009E566C394B4
:104B20007F50020566E56920E103436680AF64AE0D
:104B300063AD65AB6612848622756540E56920E148
:104B400003436520E5642410F582E43563F583E0D2
:104B500030E515436501E567540C6408605FE56A5C
:104B600013505A4365108055E567540C6408702F44
:104B7000E5681313543FF566D3941C400375661F14
:104B8000E566600BC3941D500674032566F566E563
:104B90006630E003436510E566C3134265801EE599
:104BA00068131313541FF5666007C3940F50020572
:104BB00066E5664265E56A30E003436510AF64AEC2
:104BC00063AD65128423228E5D8F5E302903024E11
:104BD0000C302B03024E0CE55E2405F582E4355DB6
:104BE000F583E064A5600AAF5EAE5D7D511251436E
:104BF00022E55E2411F582E4355DF583E054C0645E
:104C000080600AAF5EAE5D7D5212514322E55E24A4
:104C10000FF582E4355DF583E0F55FC39451400301
:104C2000024E0CE55E240EF582E4355DF583E0FF6F
:104C3000F561E55E2416F582E4355DF583E05430D8
:104C4000FEBE10035361EFE56130E422E55E240E01
:104C5000F582E4355DF583EF54EFF0AF5FE55E2458
:104C600013F582E4355DF583E0FD1289A822301E3C
:104C70001AE56130E00FE55E240EF582E4355DF55E
:104C800083E054FEF0E4F560024D19E56130E01177
:104C9000E55E240EF582E4355DF583E054FEF08098
:104CA0004BE561A2E292F7A2E130F701B3503D4338
:104CB0006101D21BE56130E105436104800353616A
:104CC000FBE55E240EF582E4355DF583E561F07564
:104CD00060807560C0AF5FAD60E55E2413F582E46F
:104CE000355DF583E01392451289F922E55E240BC8
:104CF000F582E4355DF583E0FF131313541F540F61
:104D0000F5606006640F60020560856062E56054CE
:104D10000F909E479354AAF560E55E241BF582E44C
:104D2000355DF583E0540714601624FE603224FEDE
:104D3000604E240524F94003024DC06063024DD546
:104D4000E55E2413F582E4355DF583E030E1047F10
:104D50001080027F00E5622F909E5793426080751D
:104D6000E55E2413F582E4355DF583E030E2047FEF
:104D70003080027F20E5622F909E579342608055DD
:104D8000E55E2413F582E4355DF583E030E3047FCE
:104D90005080027F40E5622F909E5793426080359D
:104DA000E55E2413F582E4355DF583E030E4047FAD
:104DB0007080027F60E5622F909E5793426080155D
:104DC000E56130E1054360448003436010E5602005
:104DD000E103436001E55E241BF582E4355DF58364
:104DE000E004F05403700FE55E240EF582E4355DB7
:104DF000F583E04410F0AF5FAD60E55E2413F5820B
:104E0000E4355DF583E01392451289F9228E718FA6
:104E1000728D738F828E83E5822405F582E435835B
:104E2000F583E064A560067D5312514322E57224A8
:104E300004F582E43571F583E0F5766409700302C8
:104E40004FE1E57365767003024FE17887E630E164
:104E500077E509D3947350F97F5512052BE5722439
:104E60000FF582E43571F583E0FF12058DE57224BC
:104E700011F582E43571F583E054C0FFBF80077FF0
:104E80006D12052B801EE5722411F582E43571F553
:104E900083E054C0FFBF40077F6E12052B80057F63
:104EA0007A12052BE5722404F582E43571F583E06E
:104EB0004430FF12052BE5732430FF12052B7F0DC4
:104EC00012052B7F0A12052BAF72AE711250F7E557
:104ED000722411F582E43571F583E054C0F57664EF
:104EE000407062E5722404F582E43571F583E07563
:104EF000F007A42449F582E5F03491AF82F5748F70
:104F000075F583E5822405F582E43583F583E0FEBB
:104F1000A3E0FFB5720BEEB57107AD75AC74124F1F
:104F2000E2E5722404F582E43571F583E573F075EA
:104F3000F007E573A42449F582E5F03491AF82F5DA
:104F4000748F758060E5722404F582E43571F58311
:104F5000E075F007A4246CF582E5F03491AF82F59A
:104F6000748F75F583E5822405F582E43583F58336
:104F7000E0FEA3E0FFB5720BEEB57107AD75AC7442
:104F8000124FE2E5722404F582E43571F583E5738E
:104F9000F075F007E573A4246CF582E5F03491AF69
:104FA00082F5748F75AE74AF75AD72AC711250A08E
:104FB000E5752405F582E43574F583E0FEA3E0B5DC
:104FC000751FEEB5741B857582857483E0FEA3E0C2
:104FD000FFE5752405F582E43574F583EEF0A3EF63
:104FE000F0228E778F788C798D7A7887E630E4405E
:104FF0007E9B7FCC1203E2E5782404F582E43577CA
:10500000F583E0FF12058D857882857783E0FEA326
:10501000E0AA06F97B02126C88857882857783E0A6
:10502000FEA3E02404F582E43EF583E0FF12058D43
:10503000E5782404F582E43577F583E0D3940550D0
:105040002A857882857783E0FEA3E0FFE57A240550
:10505000F582E43579F583EEF0A3EFF0EF2404F563
:1050600082E43EF583E0D39405401B857A828579FE
:1050700083E0FEA3E0FFE57A2405F582E43579F5C7
:1050800083EEF0A3EFF0E5782405F582E43577F5BB
:1050900083E064A56009AF78AE777D541251432256
:1050A0008E778F78AF05AE04EF2405F582E43EF5E8
:1050B00083E064A5703B857882857783E0FCA3E07C
:1050C000FD4C600B8D828C83A3A3EEF0A3EFF085E3
:1050D0007882857783EEF0A3EFF0F5828E83A3A329
:1050E000E577F0A3E578F08F828E83ECF0A3EDF006
:1050F000227D55125143228F828E83E0FCA3E08CE7
:1051000077F5788F828E83A3A3E0FCA3E0FDEF24E4
:1051100005F582E43EF583E0B4A522ED4C6023AAB8
:1051200077AB788D828C83EAF0A3EBF04A6013852D
:105130007882857783A3A3ECF0A3EDF0227D56124D
:105140005143228E7B8F7C8D7D8F828E83E58224DE
:105150000FF582E43583F583E090FE01F090FE00C8
:10516000E57DF07887E630E5317F2A12052BAF7DAB
:1051700012052BAE7BAF7C12058DE57BFF12058DF2
:10518000E57C240FF582E4357BF583E0FF12058D85
:105190007F0D12052B7F0A12052B22E4F57590F77F
:1051A00011E0543064207042900001E0FF90000054
:1051B000E02FFF900002E02FF5760575E575D3949A
:1051C000FA40DB303C03025279D23C90F700740382
:1051D000F0740AF0781A74FFF67885E620E5030289
:1051E00052797E9B7FD01203E22290F712E54BF0BA
:1051F000E54C54E0A3F0E54CC454F0440890F71695
:10520000F0E54C540FF576E4F575E575C3957650E9
:1052100018744D2575F8E6FF74172575F582E4348A
:10522000F7F583EFF0057580E190F7117465F0787C
:105230001CE6C394FF5001067885E630E53B7F53BA
:1052400012052BAF4B12058D7F2012052BAF4C1290
:10525000058D7F3A12052BE4F575E575C3957650FB
:105260000E744D2575F8E6FF12058D057580EB7FF0
:105270000D12052B7F0A12052B22C245302A0FC2C0
:105280002A7F417CEC7DE07B0A12CBF88054781DAC
:10529000E6FE2412F582E434F7F583E0F541741656
:1052A0002EF582E434F7F583E0FFC4540FFF741346
:1052B0002EF582E434F7F583E04FF5427F43EE2488
:1052C00017FDE434F7FCE542540FFB12CBF8781DD0
:1052D000741026F6B4F0027610781B1620440302F0
:1052E00064FD7885E6FF30E650E54164466005E5FB
:1052F00041B44704EF20E441AF4112058D7F2012F5
:10530000052BAF4212058D7F3A12052BE542540F53
:10531000F567E4F566E566C3956750137443256643
:10532000F8E6FF12058D7F2012052B056680E67FCB
:105330000D12052B7F0A12052B30210FE541643534
:105340006009E541644560030264FDE54154C0FF26
:10535000BFC00412A42922E54154C0648060030246
:105360005402E54254E0FFBFA00412B7FD22789F2B
:10537000E67058E54254E064407050E541543FFF08
:10538000780DE26F7045E542540FF5677F4E1205C8
:105390002B780DE2FF12058DE56724FCFF12058DC9
:1053A000756606E5672402FFE433FEC3E5669FEEFB
:1053B0006480F8748098500E74412566F8E6FF12F8
:1053C000058D056680DD789F763222789FE6D3943E
:1053D0000050030264FDE54254E06420600302646F
:1053E000FDE541543FFF780DE26F60030264FDE587
:1053F0004320E5030264FD541FFF12058D789F765C
:105400003222E54124E7B4360040030264FD9054A3
:1054100015F82828730264F60264FD0264FD026434
:10542000F60264FD0264FA0264FD0255F3025B15A4
:10543000025BCB025E2C0264FD025F910261E80216
:1054400061FC0262530262CB0255370263110263B0
:10545000150263190264710264FD0264FD0264FDB9
:105460000264FD0264FD0254B70254DD0264FD02D1
:1054700064FD0264FD0264FD0264FD0264FD0264D9
:10548000FD0264FD0264FD0264FD0255F3025B153A
:10549000025BCB025E2C0264FD025F910261E802B6
:1054A00061FC0262530262CB025537026311026350
:1054B0001502631902647175F02CE543A42409F503
:1054C00082E5F0344EAF82F5648F65F583E5822482
:1054D0000EF582E43583F583E054BFF022E54314F2
:1054E0006021146031146039240360030264FD12EA
:1054F00096F21296BD129734C21EC214C209C20C93
:10550000C203223014061296F21296BDD21EC214A5
:1055100078887441F2221296FD1296CBC20CD214F6
:10552000221296FD1296CBC20CE542B40204D203BD
:105530008002D209D2142275F02CE543A42409F587
:1055400082E5F0344EAF82F5648F65F583E5822401
:1055500010F582E43583F583E054C02480605D80DB
:1055600000754B307F4DE565240FFDE43564FC7B11
:105570000712CBF87859E2B54D06534FF3434F0C61
:10558000754C27E543D3947F4065E54F54C0644094
:10559000705DE5652404F582E43564F583E0640913
:1055A0006008E55254C064C06045754C05E4F55090
:1055B000F54FF54E85434D7551058033754B32756A
:1055C0004C2485434DE5652410F582E43564F5836C
:1055D000E0F54EE565241AF582E43564F583E0F5DF
:1055E0004FE565241BF582E43564F583E0F5501240
:1055F000519B22754B30754C0585434D85444E8536
:10560000454F854650E542540F64046003025875C7
:10561000E54354C064C0600775510212519B22E5F6
:1056200043543F700EE544C39478500775510312FC
:10563000519B22E4F5667554FF75678075F02CE583
:1056400067A42409F582E5F0344EAF82F5648F65D6
:10565000F583E5822414F582E43583F583E0B543D0
:10566000158F82E5822415F582E43564F583E065C3
:105670004470030257C4E5546037E5652404F5829D
:10568000E43564F583E0FFF552BF0908856766E4F9
:10569000F554801DE5527019E565241EF582E43548
:1056A00064F583E0F553C3955450068567668553CA
:1056B000540567E5677085E566700302586E75F0FE
:1056C0002CA42409F582E5F0344EAF82F5648F6591
:1056D000F583E582240AF582E43583F583E4F0E579
:1056E00065240BF582E43564F583E4F0E565240C6C
:1056F000F582E43564F583E4F0E565240DF582E494
:105700003564F583E4F0E565240EF582E43564F54F
:1057100083E4F0E5652410F582E43564F583744094
:10572000F07F1A128F44EF60047F0280027F00EF47
:105730004448FFE5652411F582E43564F583EFF014
:10574000E5652412F582E43564F583E4F0E565242B
:1057500013F582E43564F583E4F0E5652414F582FD
:10576000E43564F583E543F0E5652415F582E43519
:1057700064F583E544F0E5652416F582E43564F5C7
:1057800083E4F0E5652417F582E43564F583E4F0FD
:10579000E5652418F582E43564F583E4F0E56524D5
:1057A00019F582E43564F583E4F0E565241AF582A1
:1057B000E43564F583E4F0E565241BF582E43564A3
:1057C000F583E4F0E5652404F582E43564F583E0CF
:1057D000F56764097055788606E5652404F582E46A
:1057E0003564F5837404F0F567756991756A65AE83
:1057F00069AF6AAD65AC641250A0E56A2405F58214
:10580000E43569F583E0FEA3E0B56A1FEEB5691BD8
:10581000856A82856983E0FEA3E0FFE56A2405F5D9
:1058200082E43569F583EEF0A3EFF0E5676401608B
:1058300015E5676402600FE56764036009AF65AE54
:10584000647D04124E0D754B30754C27E565241EA2
:10585000F582E43564F58374FFF07F4DE565240F30
:10586000FDE43564FC7B0712CBF812519B22E4F572
:105870005112519B22E543D3947F40077551041286
:10588000519B2275F02CE543A42409F582E5F03400
:105890004EAF82F5648F65F583E5822411F582E4CD
:1058A0003583F583E054C0F567E54754C0656770FC
:1058B00003025A508F82E582240AF582E43564F5AA
:1058C00083E4F0E565240BF582E43564F583E4F0C8
:1058D000E5652412F582E43564F583E4F0E565249A
:1058E0000DF582E43564F583E4F0E565240CF5827A
:1058F000E43564F583E4F07887E630E1247F5712DD
:10590000052BE565240FF582E43564F583E0FF128D
:10591000058DAF6712058D7F0D12052B7F0A1205CD
:105920002BAF65AE641250F7E567B4802378931609
:10593000E5652404F582E43564F583E075F007A499
:10594000246CF582E5F03491AF82F5698F6A80218D
:10595000788616E5652404F582E43564F583E07500
:10596000F007A42449F582E5F03491AF82F5698F00
:105970006AE56A2405F582E43569F583E0FEA3E073
:10598000FFB5650BEEB56407AD6AAC69124FE2E591
:10599000652411F582E43564F583E0543FFFF0E5BA
:1059A0004754C0FE4FF0E5652404F582E43564F504
:1059B000837404F0EE64407040788606E565241137
:1059C000F582E43564F583E054F3F07859E2B543A9
:1059D00011E5652411F582E43564F583E0440CF0AB
:1059E000800FE5652411F582E43564F583E0440811
:1059F000F0756991756A65801BE5652411F582E48F
:105A00003564F583E054F3F04408F0756991756AE4
:105A100088789306AE69AF6AAD65AC641250A0E5B4
:105A20006A2405F582E43569F583E0FEA3E0B56AF2
:105A30001FEEB5691B856A82856983E0FEA3E0FFDE
:105A4000E56A2405F582E43569F583EEF0A3EFF00D
:105A5000E54454C0248060558000E5652410F5823B
:105A6000E43564F583E030E71AE565240BF582E45C
:105A70003564F583E4F0E5652412F582E43564F5D8
:105A800083E4F0E5652410F582E43564F583E054A1
:105A90007FF04440F0754B30754C277F4DE5652411
:105AA0000FFDE43564FC7B0712CBF88064E56524C8
:105AB00010F582E43564F583E030E61CE565241AD0
:105AC000F582E43564F583E4F0E5652411F582E4BC
:105AD0003564F583E054CFF0E5652410F582E435B4
:105AE00064F583E054BFF04480F0754B32754C246C
:105AF00085434DF54EE565241AF582E43564F5835A
:105B0000E0F54FE565241BF582E43564F583E0F5A7
:105B10005012519B2275F02CE543A42409F582E52F
:105B2000F0344EAF82F5648F65F583E582240EF57F
:105B300082E43583F583E030E605754B36800375E6
:105B40004B31754C0685434D7F4E75F02CE543A4D3
:105B5000241FF582E5F0344EAD82FC7B0512CBF8B4
:105B600012519BE5652404F582E43564F583E06415
:105B7000016018AF65AE647D01124E0DE565240E1F
:105B8000F582E43564F583E04420F0E5652411F501
:105B900082E43564F583E054C0FFBF8010E56524DE
:105BA00008F582E43564F583740AF0800EE5652417
:105BB00008F582E43564F5837402F0E5652420F588
:105BC00082E43564F583E04403F02275F02CE5436C
:105BD000A42409F582E5F0344EAF82F5648F657533
:105BE0004B33754C0185434DF583E5822404F582E2
:105BF000E43583F583E0B4090A754C04E4F55012EA
:105C0000519B22E543D3947F401AE54454C0FFBF23
:105C10004008E54554C06440600A754C0475500264
:105C200012519B22E565241AF582E43564F583E080
:105C3000F567E5652413F582E43564F583E0F566E0
:105C4000F568E54830E73AE5675401FFE548540157
:105C50006F700CE56654FEFEE54754FE6E6022E56B
:105C600066C313F566EF6003436680AF43AD66120B
:105C70009758E5652420F582E43564F583E0440215
:105C8000F0E4F566E5652412F582E43564F583E019
:105C900065466003436601E545540CFFBF040FE50C
:105CA000475401FFE56854016F6003436601E5470F
:105CB000541FFFE568541F6F6003436602E54754B5
:105CC000E0FFE56854E06F6003436604E548540173
:105CD000FFE56754016F6003436604E548541EFF07
:105CE000E567541E6F6003436608E5652410F5827E
:105CF000E43564F583E05408FFE54454086F60110F
:105D0000D246E54530E105436610800743660480CE
:105D100002C246E5652420F582E43564F583E0455A
:105D200066F0E565240FFFE43564FE7D437B0512D4
:105D3000CBE8E54854BFFFE56754404FFFE56524D5
:105D40001AF582E43564F583EFF012519B7885E60D
:105D500030E013E54730E00EE5435401FFE54654DB
:105D6000FE4FFF12052BE5652410F582E43564F53E
:105D700083E030E014E565240AF582E43564F583B8
:105D8000E020E0057411F0D245E5652410F582E4C9
:105D90003564F583E020E014E565240AF582E435F6
:105DA00064F583E030E0057412F0D245E565241611
:105DB000F582E43564F583E0540FC454F0FFE565E3
:105DC000240CF582E43564F583E0540F2FF0E5658B
:105DD0002404F582E43564F583E064016018AF655E
:105DE000AE647D01124E0DE565240EF582E4356446
:105DF000F583E04420F0E54554C0FFBF8010E56521
:105E00002408F582E43564F583740AF0800EE565B4
:105E10002408F582E43564F5837402F0AF65AE645E
:105E2000A2469247A24592481264FE2275F02CE5E4
:105E300043A42409F582E5F0344EAF82F5648F6502
:105E4000F583E5822404F582E43583F583E0B40923
:105E500010754B33754C0485434DE4F55012519B3E
:105E600022E543D3947F4037E5652414F582E43579
:105E700064F583E0F54EE5652415F582E43564F5B7
:105E800083E0F54FE545B54E06E546654F60107574
:105E90004B33754C0485434D75500112519B22E5DF
:105EA000652413FFE43564FE7D447B0712CBE8E5EF
:105EB0004A30E00C90918FE564F0A3E565F0801323
:105EC00090918FE0B5640CA3E0B56507E490918FE5
:105ED000F0A3F0E54A30E10C909195E564F0A3E57C
:105EE00065F08013909195E0B5640CA3E0B565076B
:105EF000E4909195F0A3F0E54A30E20C90919BE597
:105F000064F0A3E565F0801390919BE0B5640CA369
:105F1000E0B56507E490919BF0A3F0E54A30E30C0F
:105F20009091A1E564F0A3E565F080139091A1E064
:105F3000B5640CA3E0B56507E49091A1F0A3F075FA
:105F40004B33754C0185434D12519BE5652404F597
:105F500082E43564F583E064016018AF65AE647D6A
:105F600001124E0DE565240EF582E43564F583E0FB
:105F70004420F0E5652420F582E43564F583E044AF
:105F800003F0E5652408F582E43564F5837402F0D6
:105F900022302109E543641860030264FDE543B43F
:105FA000190040030264FD905FAEF8282873025F79
:105FB000F90260160260350264FD0264FD02604E63
:105FC0000260600264FD0264FD0264FD0264FD0281
:105FD00060960264FD0264FD0264FD0264FD0264D9
:105FE000FD0264FD0264FD0264FD0260B702612AE5
:105FF0000264FD0264FD0261471296F21296BDC270
:106000001EC214C209C20CC203754B35754C01E4A3
:10601000F54D12519B223014061296F21296BDD203
:106020001EC21478887441F2754B35754C01754D5C
:106030000112519B221296FD1296CBD214C20CC2B1
:1060400003754B35754C01754D0212519B22302959
:106050000475320922C22BD226C202E47890F222C1
:10606000854437E537B4551430290575320F801350
:10607000D229E4F532786CE547F28007D22BD202C0
:106080001296D685453585463A754B35754C017562
:106090004D0512519B22754B35754C02754D0BE425
:1060A000F54E789CE6FF30E103434E02EF30E20309
:1060B000434E0412519B22301910754B35754C021A
:1060C000754D1585384E12519B227897E66016E57E
:1060D0003865446010754B35754C02754D16853822
:1060E0004E12519B22E54530E706789776FF8004F3
:1060F000E47897F6E54554077898F670030264FD56
:10610000D3940540030264FDE545131313541F5453
:10611000077890F685443878A2A64608A64708A6D0
:106120004808A64908A64AD21922E543B41518E53D
:1061300044B53813754B35754C01754D1712519B8D
:10614000E4F5387897F622E542540F6407600302BD
:1061500064FDE54760030264FD780FE26544600377
:106160000264FDE5451460260460030264FD754B7E
:1061700035754C07754D18E4F54EF54FF550F55152
:10618000854852AF48128F448F5312519B22754B52
:1061900035754C07754D18E4F54E754F01F550F502
:1061A00051854852E54890A25F9330E030AF48AD4A
:1061B00049128FBC8F53128FFE12519BE54620E08F
:1061C0000CE54890A25F9320E1030264FD754B3516
:1061D000754C01754D0D12519BC2AF80FCAF48123A
:1061E0008F448F5312519B2275F02CE543A4241247
:1061F000F582E5F0344EF5837419F0227566027469
:10620000412566F8E6FF604175F02CA42409F5826B
:10621000E5F0344EAF82F5648F65F583E5822404A2
:10622000F582E43583F583E0F5676401601BE5677B
:1062300064026015AE647D02124E0DE5652409F519
:1062400082E43564F583740FF00566E566C3940750
:1062500040AD2275660274412566F8E6FF6033742E
:10626000422566F8E6FE602A75F02CA42409F58222
:10627000E5F0344EAD82FC75F02CEFA4240FF582CE
:10628000E5F0344EF583ECF0A3EDF00566E566B479
:1062900009C4E54370030264FD74412566F8E6FF16
:1062A00070030264FD75F02CE543A42409F582E532
:1062B000F0344EAD82FC75F02CEFA4240FF582E58E
:1062C000F0344EF583ECF0A3EDF0227566027441D4
:1062D0002566F8E6FF603275F02CA42409F582E506
:1062E000F0344EAF82F5648F65F583E5822411F5B5
:1062F00082E43583F583E054FEF0E5652406F582FB
:10630000E43564F583E4F0A3F00566E566B40ABEFF
:106310002212B47D2212B48622E542540F64027028
:1063200079754B3385434D85444EE54330E22875FE
:106330004C03E544C3944040030264FD75F005E559
:1063400044A42409F582E5F03490AF82F5698F6AA0
:10635000F583E0F54F803F754C0575F00BE544A4DF
:106360002409F582E5F0347AAF82F5698F6AE54356
:1063700030E00BE4256AF56A740B3569F569856AC6
:1063800082856983E0F54FA3E0F550856A828569CF
:1063900083A3A3E0F55112519B22E542540FFFBFA6
:1063A000031D53450F300610754B33754C02854362
:1063B0004D85444E12519B2212B8DD1266BC22E577
:1063C00042540F6404705A754B3385434D85444ED7
:1063D000E54330E2030264FD754C0575F00BE544BE
:1063E000A42409F582E5F0347AAF82F5698F6AE575
:1063F0004330E00BE4256AF56A740B3569F569856D
:106400006A82856983E0F54FAF458F50A3EFF0AF07
:10641000468F51856A82856983A3A3EFF012519B51
:10642000227885E620E3030264FD7858E254C0FF39
:10643000F2E54254E0FE1313543F4FFFF212058D74
:106440007F3A12052B7858E22408F27566027441EF
:106450002566F8E6FF12058D7F2012052B0566E5FF
:1064600066C3940A40E87F0D12052B7F0A12052BA4
:1064700022E54370030264FD754B38754C08F54DF9
:1064800075F02CA42409F582E5F0344EAF82F56452
:106490008F65F56985656A756603E56A2406F58288
:1064A000E43569F583E0FEA3E08E69F56A65657001
:1064B00003EE6564602AE56A2411F582E43569F526
:1064C00083E030E01BE56A240FF582E43569F5834B
:1064D000E0FF744B2566F8A6070566E566B40ABAC0
:1064E000E566C3940A500B744B2566F8E4F605661E
:1064F00080EE12519B2212ACBD2212AD0C228E6B8B
:106500008F6C8F828E83E5822411F582E43583F5CA
:1065100083E020E0030266AC8F828E83E582241044
:10652000F582E43583F583E0F56F856B6D856C6EE0
:10653000E4F570E56E2406F582E4356DF583E0FE42
:10654000A3E08E6DF56E4E70030266BBE56E656C62
:106550007004E56D656B70030266BBE56E2411F592
:1065600082E4356DF583E020E0030266BBE56E242E
:1065700010F582E4356DF583E054D1FFF0E56F54FA
:106580002E4FF0E56C240CF582E4356BF583E0FFCB
:10659000E56E240CF582E4356DF583EFF0E56C24AF
:1065A00017F582E4356BF583E0FFE56E2417F5827D
:1065B000E4356DF583EFF030472DE56E2420F5824C
:1065C000E4356DF583C083C082E0FFE56E2411F5EC
:1065D00082E4356DF583E030E1047E1080027E04B4
:1065E000EF4ED082D083F0304826E56E2410F5823D
:1065F000E4356DF583E06401F0E56E240AF582E48C
:10660000356DF583E030E0057412F080037411F00D
:10661000E56C2412F582E4356BF583E0FFE56E242A
:1066200012F582E4356DF583EFF0E56E2420F582F6
:10663000E4356DF583E04401F0E56E2411F582E464
:10664000356DF583E054C0FFBF8010E56E2408F57A
:1066500082E4356DF583740AF0800EE56E2408F54A
:1066600082E4356DF5837402F0E56E2404F582E46E
:10667000356DF583E064016026E56E2420F582E443
:10668000356DF583E06018AF6EAE6D7D01124E0D75
:10669000E56E240EF582E4356DF583E04420F005C7
:1066A00070E570C39408500302653322E56C24063C
:1066B000F582E4356BF583E4F0A3F022E545540759
:1066C000909F5793FCE54530E006ECC313FD800432
:1066D000EC25E0FD786AE544F27842E543F230E2E9
:1066E00049789CE620E2030267CCE544C39440402D
:1066F000030267CC75F005E544A42409F582E5F0B2
:106700003490FEAF827899A6447895A645E5453049
:10671000E30A8E83E04CFBF0EDF45BF0D223D2066B
:1067200078837404F27892760322789CE620E10361
:106730000267CCC223D20678837404F2E47892F61E
:1067400075F00BE544A42409F582E5F0347AFEAF38
:1067500082E54530E004D2178002C217E544543F79
:1067600044807899F6E5441313543F5430448078BC
:1067700095F6E54330E00BE42FFF740B3EFEE64454
:1067800040F67895E64545F66470F6E54530E33029
:106790008F828E83A3A3E030E00E8F828E83E04C45
:1067A000F0E47836F208F2228F828E83E04CFB7898
:1067B00050F2EDF45BF27836EEF208EFF2D22722D7
:1067C0008F828E83E0FBECF4FCEB5CF022C0E0C037
:1067D000F0C083C082C0D0C000C004C005C006C0E5
:1067E00007C28C758CF5758A95D28C788406202426
:1067F00078300826E556602275DC46E4F5DA20DCC0
:10680000FDE5D9C3789B96400D789606E6C39404BF
:106810004008C2088004E47896F675DC44E4F5DAB2
:1068200030DC0890F002E0422B80F5E5D9D3788C7B
:10683000964029786DE2FF7839E204F2C39F40293F
:10684000E55754FEF55790F00DF07857E254FDF2FD
:1068500090F00BF0D209E47839F2800D789EE6B41E
:1068600002077839E2600214F2A201B3920150707B
:10687000200D03026C4F152AE52A702078A0E6FF50
:10688000441890F00CF0EF4408F0EF4410F0EFF0F3
:10689000752A2275361454C0F6026C4FE52AB411DD
:1068A0001778A0E6FF441C90F00CF0EF440CF0EFDA
:1068B0004410F0EFF0026C4FA836E2FFC4540FFE14
:1068C00078A0E6FD4430FC4E90F00CF0ED4420FD45
:1068D0004EF0EF540FFF4CF0ED4FF00536026C4FC9
:1068E000302403026C4F789EE6FF4440F5DCE4F56B
:1068F000DA90F002E0422BEFB408004003026C4B48
:10690000906907F828287302691F0269790269D320
:10691000026A4C026AB2026B2A026B84026BE6E5E1
:106920002B30E0177845E2C394105004E22408F2BB
:106930007845E230E712748FF2800D7845E2600806
:1069400014F2E2B48002E4F2E52B30E4177849E275
:10695000C394105004E22408F27849E230E713743B
:106960008FF2800E7849E26009E214F2E2B480020C
:10697000E4F2789E7601026C4FE52B30E117784601
:10698000E2C394105004E22408F27846E230E712A1
:10699000748FF2800D7846E2600814F2E2B480024F
:1069A000E4F2E52B30E517784AE2C394105004E294
:1069B0002408F2784AE230E713748FF2800E784AA6
:1069C000E26009E214F2E2B48002E4F2789E760218
:1069D000026C4FE52B30E2177847E2C39410500465
:1069E000E22408F27847E230E713748FF2800E78E1
:1069F00047E26009E214F2E2B48002E4F2E52B30EF
:106A0000E617784BE2C394105004E22408F2784B66
:106A1000E230E713748FF2800E784BE26009E214E3
:106A2000F2E2B48002E4F220DCFDAFDAEF75F004AC
:106A3000A4E5F0FDAFD9EF75F004A4FFE5F0788A86
:106A4000F6ED4F08F6789E7603026C4FE52B30E3A7
:106A5000177848E2C394105004E22408F27848E220
:106A600030E713748FF2800E7848E26009E214F286
:106A7000E2B48002E4F2E52B30E717784CE2C394ED
:106A8000105004E22408F2784CE230E713748FF2DD
:106A9000800E784CE26009E214F2E2B48002E4F283
:106AA000E4F52B20DCFD7886E5D9F2789E760402A9
:106AB0006C4FE52B30E0177845E2C394105004E2A8
:106AC0002408F27845E230E712748FF2800D7845A1
:106AD000E2600814F2E2B48002E4F2E52B30E4173D
:106AE0007849E2C394105004E22408F27849E23075
:106AF000E713748FF2800E7849E26009E214F2E243
:106B0000B48002E4F220DCFDAFDAEF75F004A4E516
:106B1000F0FDAFD9EF75F004A4FFE5F0787FF6ED56
:106B20004F08F6789E7605026C4FE52B30E117781A
:106B300046E2C394105004E22408F27846E230E7BB
:106B400012748FF2800D7846E2600814F2E2B4808D
:106B500002E4F2E52B30E517784AE2C394105004C2
:106B6000E22408F2784AE230E713748FF2800E785C
:106B70004AE26009E214F2E2B48002E4F2789E761E
:106B800006026C4FE52B30E2177847E2C3941050B1
:106B900004E22408F27847E230E713748FF2800EA3
:106BA0007847E26009E214F2E2B48002E4F2E52BF5
:106BB00030E617784BE2C394105004E22408F278D0
:106BC0004BE230E713748FF2800E784BE26009E2FB
:106BD00014F2E2B48002E4F220DCFD785AE5D9F246
:106BE000789E76078069E52B30E3177848E2C394F6
:106BF000105004E22408F27848E230E713748FF270
:106C0000800E7848E26009E214F2E2B48002E4F215
:106C1000E52B30E717784CE2C394105004E22408C7
:106C2000F2784CE230E713748FF2800E784CE26019
:106C300009E214F2E2B48002E4F2E4F52B20DCFD78
:106C4000785EE5D9F2E4789EF68004E4789EF6D288
:106C50002530071F780B08E22401FFF218E2340008
:106C6000FEF2C3EF9460EE94045008C2AFD2AED2ED
:106C7000BED2AFD007D006D005D004D000D0D0D03F
:106C800082D083D0F0D0E0328B7B8A7C897DAE02CB
:106C9000AF01EF4E70087E9B7FDC1203E222E4F529
:106CA0007EE57E75F02CA42409F9744E35F0FAE5E2
:106CB0007B857C83857D8264027008E96582700330
:106CC000EA658370127E9B7FE21203E2AF7E1205BB
:106CD0008D7F2012052B22057EE57E70C4F57EE5B2
:106CE0007E75F007A42449F9749135F0FAE57B85A7
:106CF0007C83857D8264027008E965827003EA65A1
:106D00008370157E9B7FE51203E2E57E4430FF121F
:106D1000052B7F2012052B22057EE57EC3940540BE
:106D2000BEE4F57EE57E75F007A4246CF974913518
:106D3000F0FAE57B857C83857D8264027008E965D5
:106D4000827003EA658370157E9B7FE91203E2E59A
:106D50007E4430FF12052B7F2012052B22057EE595
:106D60007EC3940540BE7F3F12052BE57CFF1205D4
:106D70008DAF7DE57D12058D22E4F562F563C2439A
:106D8000C244783AE25406789CF6C2217F16128FEC
:106D900044BF01097F16E4FD128FBCD2437F1A1253
:106DA0008F448F5BC0077F1B128F44AE07D007EE66
:106DB0006F601AE55B600C7F1B7D01128FBC436224
:106DC00001800A7F1BE4FD128FBC4363019091C0D8
:106DD000E0FF548664807028EF30E5134362017F42
:106DE0001A7D01128FBC7F1B7D01128FBC80114365
:106DF00063017F1AE4FD128FBC7F1BE4FD128FBC80
:106E0000E49091C0F030430B755E04755F047560CB
:106E10000480157F50128F448F5E7F51128F448FF4
:106E20005F7F52128F448F60128FFEE4F55B75F026
:106E300007E55BA42449F582E5F03491F583AF8240
:106E4000FEF0A3EFF075F007E55BA4244BF582E5B7
:106E5000F03491F583EEF0A3EFF075F007E55BA455
:106E6000244EF582E5F03491F583EEF0A3EFF07552
:106E7000F007E55BA4244DF582E5F03491F58374C9
:106E8000AAF075F007E55BA4246CF582E5F0349177
:106E9000F583AF82FEF0A3EFF075F007E55BA42465
:106EA0006EF582E5F03491F583EEF0A3EFF075F026
:106EB00007E55BA42471F582E5F03491F583EEF0EB
:106EC000A3EFF075F007E55BA42470F582E5F034DC
:106ED00091F58374AAF0055BE55B64056003026EBF
:106EE0002E302103D21522D204D2AED2BE789CE637
:106EF00030E107780E7440F28005780E7480F278E5
:106F00003D7480F2E4F55B7886F67893F6304407BA
:106F10007E9B7FED1203E220440302710A75F02C80
:106F2000E55BA424DDF582E5F0344DAF82F5598FA1
:106F30005AE55B14FF12058D7F2012052BE55A24BC
:106F400004F582E43559F583E0FF12058D7F2012A8
:106F5000052BE55A2405F582E43559F583E0FF1247
:106F6000058D7F2012052BE55A2408F582E435595A
:106F7000F583E0FF12058D7F2012052BE55A2409C9
:106F8000F582E43559F583E0FF12058D7F20120567
:106F90002BE55A240AF582E43559F583E0FF120502
:106FA0008D7F2012052BE55A240BF582E43559F527
:106FB00083E0FF12058D7F2012052BE55A240CF586
:106FC00082E43559F583E0FF12058D7F2012052BF1
:106FD000E55A240DF582E43559F583E0FF12058D5D
:106FE0007F2012052BE55A240EF582E43559F583EE
:106FF000E0FF12058D7F2012052BE55A240FF58244
:10700000E43559F583E0FF12058D7F2012052BE54D
:107010005A2411F582E43559F583E0FF12058D7F7E
:107020002012052BE55A2411F582E43559F583E049
:10703000FF12058D7F2012052BE55A2412F582E4FC
:107040003559F583E0FF12058D7F2012052BE55A97
:107050002413F582E43559F583E0FF12058D7F2076
:1070600012052BE55A2414F582E43559F583E0FF27
:1070700012058DE55A2415F582E43559F583E0FFB4
:1070800012058D7F2012052BE55A2416F582E43572
:1070900059F583E0FF12058D7F2012052BE55A2458
:1070A00017F582E43559F583E0FF12058D7F201234
:1070B000052BE55A2418F582E43559F583E0FF12D3
:1070C000058D7F2012052BE55A2419F582E43559E8
:1070D000F583E0FF12058D7F2012052BE55A241A57
:1070E000F582E43559F583E0FF12058D7F20120506
:1070F0002BE55A241BF582E43559F583E0FF120590
:107100008D7F0A12052BD2AED2BE75F02CE55BA4A2
:107110002409F582E5F0344EAF82F5598F5AF58394
:10712000E582240FF582E43583F583E55BF0855A2B
:1071300082855983E4F0A3F0855A82855983A3A3FD
:10714000F0A3F0E55A2411F582E43559F583E054B3
:10715000CFF030220EE55A2411F582E43559F5833B
:107160007408F0E55A2405F582E43559F58374A5D1
:10717000F0E55A240EF582E43559F583E0549FF08A
:10718000E55A2411F582E43559F583E0F55D54C0E4
:10719000FF6440702F789CE654066404600302721A
:1071A0006D535D3F435D80E55A2414F582E4355903
:1071B000F583E4F0E55A2404F582E43559F583E4D7
:1071C000F002726DEF64807047789CE6FF30E20A4F
:1071D000E55BD39451500302726DEF20E10302721C
:1071E0006D535D33435D48E55A2414F582E4355907
:1071F000F583E4F0E55A2415F582E43559F583E486
:10720000F0E55A2404F582E43559F583E4F0805D15
:10721000789CE6FF5406FEBE0422535D3F435D802A
:10722000E55A2414F582E43559F583E4F0E55A244F
:1072300004F582E43559F583E4F08031EF30E12D37
:10724000535D33435D48E55A2414F582E43559F51E
:1072500083E4F0E55A2415F582E43559F583E4F02A
:10726000E55A2404F582E43559F583E4F0E55A241F
:1072700011F582E43559F583E55DF0E55D54C064B0
:10728000406003027574789CE620E103027574E5A2
:107290005A2410F582E43559F583E0547FF04440D8
:1072A000F0E56230E00FE55A2411F582E43559F536
:1072B00083E04402F0E56330E00FE55A2411F582E3
:1072C000E43559F583E054FDF0E55A2410F582E4E5
:1072D0003559F583E0FF30E0224410F0E55A240AE6
:1072E000F582E43559F5837403F0E55A240EF582EE
:1072F000E43559F583E04402F0802FEF20E02BE5E0
:107300005A2410F582E43559F583EF54EFF0E55A2D
:10731000240AF582E43559F583E4F0E55A240EF5A4
:1073200082E43559F583E054FDF0E55B7011E55AD0
:107330002404F582E43559F5837409F00276D67891
:107340003DE2FFE55BC39F4003027425788606E5B6
:107350005A2404F582E43559F583E0F5616069E566
:107360005E24FD601514601714601914602E1460FB
:107370004224057053756103804E7561048049E4B1
:10738000F5618044E55A2412F582E43559F583E02D
:1073900070047F0480027F038F61802CE55A2412E1
:1073A000F582E43559F583E07003FF80027F048F96
:1073B000618015E55A2412F582E43559F583E070B1
:1073C00003FF80027F038F61E561D39405400302D0
:1073D00076D675F007E561A42449F582E5F034918D
:1073E000AF82FEAD5AAC591250A075F007E561A40A
:1073F0002449F582E5F03491F583E0FEA3E0FF75C2
:10740000F007E561A4244EF582E5F03491F583EEB2
:10741000F0A3EFF0E55A2404F582E43559F583E54D
:1074200061F00276D6E55BD3947F50030276D6E511
:107430005A2414F582E43559F583E054C064C070D1
:1074400029E55A2404F582E43559F583E0FF6409FF
:107450006018E55FB4080EE55A2412F582E4355948
:10746000F583E06005E55FB4092BE55A2404F58255
:10747000E43559F5837409F0E55A2414F582E435AE
:1074800059F583E4F0E55A2415F582E43559F5837E
:10749000E4F00276D68F61EF6069E55F24FD601548
:1074A00014601714601914602E1460422405705380
:1074B000756103804E7561048049E4F5618044E59F
:1074C0005A2412F582E43559F583E070047F048074
:1074D000027F038F61802CE55A2412F582E435592E
:1074E000F583E07003FF80027F048F618015E55A09
:1074F0002412F582E43559F583E07003FF80027FA2
:10750000038F61E561C39405505075F007E561A4F0
:107510002449F582E5F03491AF82FEAD5AAC5912A0
:1075200050A075F007E561A42449F582E5F0349197
:10753000F583E0FEA3E0FF75F007E561A4244EF5B6
:1075400082E5F03491F583EEF0A3EFF0E55A2404E0
:10755000F582E43559F583E561F0788606E55A242D
:107560001EF582E43559F583E070030276D6E01407
:10757000F00276D6E55D54C0648060030276D6786A
:107580009CE620E2030276D6E55BC39451400302F9
:1075900076D6D20A789306E55A2410F582E4355956
:1075A000F583E0547FF030E02EE55A2410F582E4B4
:1075B0003559F583E04410F0E55A240AF582E435A4
:1075C00059F5837403F0E55A240EF582E43559F534
:1075D00083E04402F0802FE55A2410F582E4355907
:1075E000F583E0FF20E01F54EFF0E55A240AF5820E
:1075F000E43559F583E4F0E55A240EF582E4355973
:10760000F583E054FDF0E55A2404F582E43559F59C
:1076100083E0F5616069E56024FD6015146017146E
:10762000601914602E146042240570537561038044
:107630004E7561048049E4F5618044E55A2412F5F1
:1076400082E43559F583E070047F0480027F038F64
:1076500061802CE55A2412F582E43559F583E070F7
:1076600003FF80027F048F618015E55A2412F582A2
:10767000E43559F583E07003FF80027F038F61E5F5
:1076800061C39405505075F007E561A4246CF58240
:10769000E5F03491AF82FEAD5AAC591250A075F0AE
:1076A00007E561A4246CF582E5F03491F583E0FEF2
:1076B000A3E0FF75F007E561A42471F582E5F034DD
:1076C00091F583EEF0A3EFF0E55A2404F582E4355A
:1076D00059F583E561F0AF5B055BEFC394FF5003A1
:1076E000026F1730441C7E9B7FFC1203E27886E613
:1076F000FF12058D7E9C7F071203E27893E6FF124E
:10770000058D22D2077885E620E3030277B27F6CED
:1077100012052B7F6212052B7F6112052B78B4E6D0
:10772000FF12058D78B5E6FF12058D7F6412052BDB
:107730007F6512052B7F6612052B78B2E6FF1205D6
:107740008D78B2E6FE08E6FF12058D7F7012052BDC
:107750007F7012052B7F7012052B78B0E6FF1205A3
:107760008D78B0E6FE08E6FF12058D7F6C12052BC2
:107770007F6512052B7F6E12052B78B0E6FE08E6BA
:10778000FFC3901C1AE09F901C19E09EFF3395E008
:1077900012058D78B0E6FE08E6FF901C19E0FCA308
:1077A000E0FDC39FFF12058D7F0D12052B7F0A128E
:1077B000052B901C19E0FEA3E078B166700318E673
:1077C0006E70030278DBE4F559E55925E0246DF588
:1077D00082E4341CF583E0FEA3E0D378B396EE1880
:1077E000964024E55925E0246EF582E4341CF583A7
:1077F00078B4E6FE08E6FFC3E09FF00582D582027A
:1078000015831582E09EF00559E559B414BB78AB99
:10781000761C0876A1E4FFFEC3EF9484EE94034047
:10782000030278A178ABE6FC08E6F5828C83E0FDE4
:10783000A3E07894CDF208EDF2E2700218E2604F16
:107840007894E230E708E2547FF2D2398002C239FC
:1078500078B2E6FC08E6FDD37895E29D18E29C40FC
:107860002E78B4E6FC08E6FDC37895E29DF218E2B6
:107870009CF2303904E24480F27894E2FC08E2FDA4
:1078800078ABE6FA08E6F5828A83ECF0A3EDF00F18
:10789000BF00010E78AC740226F618E436F60278C2
:1078A0001878B0E6FE08E6FFC3901C1AE09FFD9032
:1078B0001C19E09EFCC004C005AA06A9077B02C0F3
:1078C00003C00278B2E6FE08E6AA06F8AC02AD03F1
:1078D000D002D003D007D00612D1FB78B4E6FE0860
:1078E000E6FFC3901C1AE09FFD901C19E09EFCF07F
:1078F000A3EDF0C3901C1CE09FF0901C1BE09EF0D9
:107900008D828C83E4F0C239C235C2077884760157
:10791000223002097844E2600414F27041E4789164
:10792000F6788AE6FE08E6FF7D107B021296777CE9
:10793000007D2112CFB57835E2FD12CFC97D02124C
:10794000836778187456F278197420F2781AF278EE
:107950001BF2781CF2781DF2781EF2781FF23002CA
:10796000087844E26003027A3A30160E7B057A9C6E
:1079700079127D10128327027A3A300C0E7B057A39
:107980009C79197D10128327027A3A30090E7B0503
:107990007A9C79207D10128327027A3A30140E7B6C
:1079A000057A9C79277D10128327027A3A301E0DC2
:1079B0007B057A9C792E7D10128327807D30150DF2
:1079C0007B057A9C79357D10128327806D789176BE
:1079D00010787FE6FE08E6FF7D8A7B0212967778B4
:1079E00054E2FD3395E0FC783EE22DFDE43CFCC31F
:1079F000EF9DFFEE9CFED3EF94FFEE947F400A7C58
:107A0000007D00AE04AF0580007891E2FD7C00129D
:107A1000CFB57840E2FD12CFC97D01128367782887
:107A20007441F278297420F2782AF2782BF2782CBB
:107A3000F2782DF2782EF2782FF2302103027B06B5
:107A40007887E6B4801678207454F278217445F271
:107A500078227453F2782304F2027B00781AE6FD50
:107A6000706B781CE6FF700A7821742EF27822F28F
:107A7000804BEFC3940350117821742EF2EF25E070
:107A800025E024307822F28034EF75F064A4E5F02C
:107A9000F564C394644003756463E56475F00A8417
:107AA000FF700778217420F28006EF24307821F2ED
:107AB000E56475F00A84E5F024307822F2782074C9
:107AC00043F278237425F2E4781CF680337820742E
:107AD00043F278217445F27822743AF2ED54072487
:107AE000307823F27885E630E5167F4312052B7F48
:107AF0004512052B781AE6FF12058D7F0A12052B19
:107B0000E4781AF6802378207453F27821744CF2CA
:107B1000780FE2FF75F00A8424307822F2EF75F0D6
:107B20000A84E5F024307823F290F001E0F564C493
:107B3000540F9005D0937830F2E564540F93783168
:107B4000F290F002E0F564C4540F9005D0937832BF
:107B5000F2E564540F937833F222E4F55B74452523
:107B60005BF8E220E403027C1C748FF2E55B75F0A5
:107B700006A4248FF582E43491AF82F5598F5AF52B
:107B800083A3A3E024FE605814605A14605C146060
:107B90005924046003027C1C855A82855983E0FEC7
:107BA000A3E0FF4E6076855A82855983A3A3A3E0A4
:107BB000FDEF241CF582E43EF583EDF0E55A240444
:107BC000F582E43559F583E0FDEF241DF582E43EAE
:107BD000F583EDF0E55B90A36D93FD1232CA803C16
:107BE000127CC08037127CCD8032E55A2405F582A4
:107BF000E43559F583E0FF601375F00A84F543EF2F
:107C000075F00A84E5F014F54412B486855A82852D
:107C10005983A3A3E064057003027B98055BE55BD1
:107C2000C394085003027B5D22C245204435E4F52D
:107C300064E56475F006A42491F582E43491F5833B
:107C4000E0B4060E7889E2FFE564909F5793FEEF5B
:107C50004EF20564E564B408D87889E26003D38005
:107C600001C322E4F56474452564F8E25490601180
:107C7000E564909F5793FF7889E25F6004D2458066
:107C8000070564E564B408DE7890E2701630450CB0
:107C90007B057A9C793CFD128327802278907401C1
:107CA000F2801B7890E2B4011520450D7B057A9C8B
:107CB000795DE4FD128327800578907402F2C32277
:107CC000D21E78887441F2C24512955B22D214C24A
:107CD0000CC2031296FD1296CBC24512955B22D2BE
:107CE00024EF4440F5DCE4F5DA20DCFD204507AF65
:107CF000D9C2247E0022AFDAEF75F004A4E5F0FDCE
:107D0000AFD9EF75F004A4FFAEF0E5F0ED4FFFC280
:107D10002422AC077910E4FBFAAF04A24492451286
:107D20007CDFEF2BFBEE3AFAD9EFEAC4F854F0C847
:107D300068FEEBC4540F48FF22E4F5597557FC90D8
:107D4000F00D74FCF078A1F6A3F012827390F001AC
:107D5000E020E003027F7EC2AFD2AED2BED2AFE05F
:107D6000FFC4540F9005D0937827F290F001E054AF
:107D70000F9005D0937828F290F002E0FFC4540FE2
:107D80009005D093782AF290F002E0540F9005D03D
:107D900093782BF2E55924FD6015146017146019CF
:107DA00014601B14601D2405701E755C15801E7503
:107DB0005C198019755C1D8014755C21800F755CE1
:107DC0002D800A755C318005755901802DAF59D21F
:107DD00044127D128E5A8F5BE55A9005D093AE5CAB
:107DE000055CA806F2AF5BEFC4540F93AD5C055C75
:107DF000A805F2EF540F93A85CF2055990F001E04A
:107E000020E103027D4DC2AFD2AED2BED2AFE020A0
:107E1000E60D30930A1296FD7FA87E611203D312FD
:107E200096CB1296F2C2AFD2AED2BED2AF7F507E08
:107E3000C31203D37F04D244127D12783EEFF2D3F3
:107E4000941440101282737B057A9C797EE4FD12B3
:107E5000832780A81296BD90F001E030E19E7F0458
:107E6000C244127D12D3EF9432EE94005003027F8D
:107E70005B7F02D244127D128E5A8F5BE47891F6BA
:107E8000FC7D2112CFB57D6612CFC97D02128367BA
:107E900078187455F2AE5AAF5B7C007D2812CFB5CE
:107EA0007DC612CFC97891EFF2789176067E007D7B
:107EB00001128367781E7443F27F04D244127D124C
:107EC0008E5A8F5BEF7803CEC313CE13D8F9FF78A9
:107ED00040F27891760C7E00E4FD1283677823747B
:107EE00048F278917610783EE2FF7E00E4FD12833E
:107EF000677827744CF278917615783EE2FFC3E5F7
:107F00005B9FFFE55A9400FED3EF94FFEE947F4011
:107F10000A7C007D00AE04AF0580007891E2FD7C14
:107F20000012CFB57840E2FD12CFC97D0112836700
:107F3000782D7441F27891761BAF5BAE5A7D0112B9
:107F4000836778337449F2E4FF7840E2FD128FBC16
:107F50007F027891E2FD128FBC800E1282737B0546
:107F60007A9C7996E4FD128327C2AFD2AED2BED2FC
:107F7000AF7FA87E611203D3128273027E57E4F5AD
:107F80005790F00DF0754B35754C01754D0D125134
:107F90009B12519B12519BD2AED2BEC2AF80FC222B
:107FA000E4F559F55AD2437EA37F751203E27B05AF
:107FB0007AA3797F7D10128327E4F55D7EA37F7F0E
:107FC0001203E2AF5D12058D7F0A12052B90F008B7
:107FD000E55DF0FF7401A807088002C333D8FCF503
:107FE0005FE4F559F55AF55BF55CD2AED2BEB290BE
:107FF000E4F55E055AE55AAE597002055914F5824A
:108000008E83E55FF0055EE55EB480E7055CE55CC8
:108010007002055BE4B55CD2E55BB401CD055DE5BE
:108020005DC3940840967B057AA3798A7D101283FC
:1080300027E4F55D7EA37F8A1203E2AF5D12058D12
:108040007F0A12052B90F008E55DF0FF7401A80788
:10805000088002C333D8FCF55FE4F559F55AF55BA7
:10806000F55CD2AED2BEB291E4F55E855A828559F6
:1080700083E0655F60467EA37F951203E2AF5D12E9
:10808000058D7F2012052BE55CAE5B7807C333CEF0
:1080900033CED8F97C00255EEC3EFF12058DE55C01
:1080A000AE5B7807C333CE33CED8F97C00255EFFB4
:1080B000EC3E12058D7F0A12052BC243055AE55A84
:1080C000AE597002055914F5828E83E4F0055EE521
:1080D0005EC394804095055CE55C7002055BC3E57A
:1080E0005B94015003028062055DE55DC394085016
:1080F0000302803490F008E4F03043137EA37FA2A3
:108100001203E27B057AA379A27D10128327227ED7
:10811000A37FAD1203E27B057AA379AD7D101283B4
:108120002722E4F55B7F17128F44BF6F097F17E4A6
:10813000FD128FBC802A783AE254A764A76021E53B
:108140005BC39418501AE55B909CDE93FF74002586
:108150005BF582E43400F583E0B50704055B80DF5E
:10816000E55BC3941840030281EBC2AFD2AED2BE2E
:108170007EF07F007D007B027A00790012D0607E65
:10818000037FFF7D007B027AFC790012D0607800CB
:108190007C007D027B057A9C79DE7E007F1812CF01
:1081A00068D2AED2BED2AFD2227F1A7D01128FBC6E
:1081B0007F1BE4FD128FBC7E9C7FA61203E212821D
:1081C000737B057A9C79B6E4FD128327E4F55BC2E4
:1081D000AFD2AED2BED2AF7FA87E611203D3055B11
:1081E000E55BC3940740E8C2AF80FC22E4F559F593
:1081F0005AFDFCFE7F80855A82855983E493FA7488
:1082000001932DFDEA3CFC7402255AF55AE43559D8
:10821000F559DFE27F80855A82855983E493FA74A9
:1082200001932DFDEA3CFC7402255AF55AE43559B8
:10823000F559DFE2D2AED2BE0EBE80B87557FC78DB
:10824000A176FCED4C602B90F00DE557F078A1E69F
:10825000A3F06357FCE4FCFDC3EC948050E5EFF51C
:10826000F0A4FF7C007D01D2AED2BE0DBD00010C9A
:1082700080E6227E007F207D207B037AFC79141229
:10828000D060E47891F6221282737F887E13120305
:10829000D390F00C7413F07403F07FE27E041203A9
:1082A000D390F00C7413F07403F07F327E0012034D
:1082B000D390F00C7413F07403F07F0C7E00120363
:1082C000D390F00C7412F07402F07F0C7E00120355
:1082D000D390F00C7412F07402F07418F07408F07B
:1082E0007F0C7E001203D390F00C7410F0E4F07455
:1082F0001CF0740CF0FF7E001203D390F00C74108D
:10830000F0E4F07411F07401F07FF4FE1203D390E6
:10831000F00C7410F0E4F07416F07406F07F0C7E2C
:10832000001203D3D20D228B658A668967EDF46053
:108330000AEDC3942050047891A605AB65AA66A9FE
:108340006712CF9AFF601F7891E6FEC39420501603
:1083500074142EF8EFF274012567F567E43566F5BD
:108360006678910680D5228D65AB07AA06E5656023
:10837000047F0180027F007891E624022FF566C316
:10838000648094A04003028422E56604F6AE02AF46
:10839000037C007D0A12CFC9ED2430FFAE6615665E
:1083A00074142EF8EFF2AE02AF037C007D0A12CFF8
:1083B000C9AA06AB07E565B4020BAF66156674146F
:1083C0002FF8742EF2AE02AF037C007D0A12CFC9E3
:1083D000ED2430FFAE66156674142EF8EFF2AE028F
:1083E000AF037C007D0A12CFC9AA06AB07E565B4CE
:1083F000010BAF66156674142FF8742EF2AE02AF3F
:10840000037C007D0A12CFC9ED2430FF7414256669
:10841000F8EFF2AE02AF037C007D0A12CFC9AA06C4
:10842000AB0722EF240FF582E43EF583E0FCC39412
:1084300080501A78787403F27834E27879F2787A96
:10844000ECF2787BEDF2EC6D787CF2803578787424
:1084500004F27834E27879F2EF2414F582E43EF500
:1084600083E0787AF2EF2415F582E43EF583E07834
:108470007BF2787CEDF2787BE2FF787AE26F6D78C0
:108480007DF212851C228E6B8F6C8F828E83E5822B
:10849000240FF582E43583F583E0FFC39480501FF9
:1084A00078787404F27834E27879F2787AEFF278B6
:1084B0007BEDF2787CEBF2EF6D6B787DF2803E78AD
:1084C000787405F27834E27879F2E56C2414F58258
:1084D000E4356BF583E0787AF2E56C2415F582E4F7
:1084E000356BF583E0787BF2787CEDF2787DEBF20A
:1084F000787BE2FF787AE26F6D6B787EF212851CF2
:108500002278787403F27834E27879F2787AEFF2AC
:10851000787BEDF26F787CF212851C227887E6304A
:10852000E003D38001C39245756F78AF6F056FA8E4
:1085300007E2F571700302860CD3940640030286AD
:108540000C203F13756DEC756E00E490EEE0F0A327
:10855000F0A3F0A3F08011756DED756E00E490EE60
:10856000E4F0A3F0A3F0A3F0E57175F012A42404E5
:10857000FF056EE56EAC6D7002056D14F5828C839F
:10858000EFF0AF6F056FA807E2FF056EE56EAC6D0B
:108590007002056D14F5828C83EFF03045057F4441
:1085A00012052B1571E4F570E570C39571503DAF60
:1085B0006F056FA807E2F572304504FF12058DE5DF
:1085C00070C394025013203F09742D2570F8A672D1
:1085D0008007742F2570F8A672AF6EAE6DAD72C2B3
:1085E0004612860D8E6D8F6E057080BC30450CA8CE
:1085F0006FE2FF12058D7F0A12052BAF6EAE6DA8DC
:108600006FE2FDD24612860DD23DB23F227C803011
:1086100041328F828E83E519F00FBF00010E8F82E9
:108620008E83E518F00FBF00010E8F828E837425B4
:10863000F00FBF00010E8F828E837401F00FBF0018
:10864000010E80308F828E837425F00FBF00010EE3
:108650008F828E837401F00FBF00010E8F828E8394
:10866000E519F00FBF00010E8F828E83E518F00F21
:10867000BF00010EEC70030287195D60308F828E9F
:1086800083E533F00FBF00010E8F828E83E4F00F7D
:10869000BF00010E8F828E83E533F00FBF00010E05
:1086A0008F828E83E4F00FBF00010E80653041326F
:1086B0008F828E83E519F00FBF00010E8F828E83AB
:1086C000E518F00FBF00010E8F828E837425F00F26
:1086D000BF00010E8F828E837401F00FBF00010E68
:1086E00080308F828E837425F00FBF00010E8F8241
:1086F0008E837401F00FBF00010E8F828E83E51907
:10870000F00FBF00010E8F828E83E518F00FBF00BF
:10871000010EECC313FC0286742046030287B28F5D
:10872000828E83E533F00FBF00010E8F828E83E4CB
:10873000F00FBF00010E8F828E83E533F00FBF0074
:10874000010E8F828E83E4F00FBF00010E304132A4
:108750008F828E83E519F00FBF00010E8F828E830A
:10876000E518F00FBF00010E8F828E837425F00F85
:10877000BF00010E8F828E837401F00FBF00010EC7
:1087800080308F828E837425F00FBF00010E8F82A0
:108790008E837401F00FBF00010E8F828E83E51966
:1087A000F00FBF00010E8F828E83E518F00FBF001F
:1087B000010E2278787403F2784FE27879F2787AB1
:1087C000EFF2787BEDF26F787CF21287EF22787807
:1087D0007404F2784FE27879F2787AEFF2787BEDF0
:1087E000F2787CEBF2EF6D6B787DF21287EF2278F6
:1087F00087E630E003D38001C39244756678AF66A4
:108800000566A807E2F56770030288A7D3940640BF
:10881000030288A7203F087564EC75650080067523
:1088200064ED756500E56775F012A42404FF056525
:10883000E565AC647002056414F5828C83EFF0AFDB
:10884000660566A807E2FF0565E565AC647002058C
:108850006414F5828C83EFF03044057F5012052BB1
:108860001567E5676021304407A866E2FF12058DB1
:10887000AF65AE64AD660566A805E2FDC245128827
:10888000A88E648F6580D930440CA866E2FF12057B
:108890008D7F0A12052BAF65AE64A866E2FDD24556
:1088A0001288A8D23DB23F227C808F828E837425AD
:1088B000F00FBF00010E8F828E837401F00FBF0096
:1088C000010E8F828E837425F00FBF00010E8F8200
:1088D0008E837401F00FBF00010EEC60695D6030A3
:1088E0008F828E83E533F00FBF00010E8F828E835F
:1088F000E4F00FBF00010E8F828E83E533F00FBFCF
:1089000000010E8F828E83E4F00FBF00010E8030D5
:108910008F828E837425F00FBF00010E8F828E83AD
:108920007401F00FBF00010E8F828E837425F00F4B
:10893000BF00010E8F828E837401F00FBF00010E05
:10894000ECC313FC809430455E8F828E83E533F058
:108950000FBF00010E8F828E83E4F00FBF00010E67
:108960008F828E83E533F00FBF00010E8F828E83DE
:10897000E4F00FBF00010E8F828E837425F00FBFCD
:1089800000010E8F828E837401F00FBF00010E8FE5
:10899000828E837425F00FBF00010E8F828E837448
:1089A00001F00FBF00010E2278787403F208741EE4
:1089B000F2EF909DF693787AF2EDC313540F2447AB
:1089C000F582E4349EF583E493787BF2787C74033B
:1089D000F2128A192278787403F208741EF2EF906A
:1089E0009DF693787AF2ED540F909E4793787BF240
:1089F000787C7402F2128A192278787403F208746F
:108A00001EF2EF909DF693787AF2787BEDF2A24514
:108A1000E433787CF2128A1922787AE2F566787B60
:108A2000E2F567787CE2FF139247EFA2E192487883
:108A300087E630E003D38001C39246756578203F16
:108A4000087563EC75640080067563ED7564000558
:108A500064E564AE637002056314F5828E83744925
:108A6000F0780EE2B480047F0080047879E2FF059C
:108A700064E564AC637002056314F5828C83EFF0E7
:108A8000AF64AE63AD66A248E4334402FB128B21AF
:108A90008E638F64A2479249A248924A128E778EC3
:108AA000638F64A2479249A248924A128E778E63DE
:108AB0008F64AD67A248E4334404FB128B218E63BC
:108AC0008F64AD66A248E433FB128B218E638F6402
:108AD000A2479249A248924A128E778E638F64A26F
:108AE000479249A248924A128E778E638F64AD678F
:108AF000A248E433440CFB128B218E638F64D23D79
:108B0000B23F30461B7F4D12052BAF6612058DAF6D
:108B10006712058D787CE2FF12058D7F0A12052B06
:108B2000228E688F698D6A7F80EB30E122856982B1
:108B300085688374ACF00569E5697002056885692C
:108B400082856883740AF00569E56970020568EB3F
:108B500030E003028CE4791130E3034301407E10DE
:108B6000EB30E303430640EF64017003028C03E53E
:108B70006A5F604585698285688374E5F00569E50B
:108B800069700205688569828568837401F00569EA
:108B9000E569700205688569828568837445F0051A
:108BA00069E56970020568856982856883E4F00576
:108BB00069E5697002056880438569828568837408
:108BC00045F00569E56970020568856982856883F5
:108BD000E4F00569E5697002056885698285688346
:108BE00074E5F00569E56970020568856982856844
:108BF000837401F00569E56970020568EFC313FF2E
:108C0000028B67E56A5F606E85698285688374E5BB
:108C1000F00569E569700205688569828568837475
:108C200001F00569E56970020568EB30E2248569A9
:108C3000828568837426F00569E569700205688598
:108C40006982856883EEF00569E56970020568024E
:108C50008E6E8569828568837445F00569E5697063
:108C6000020568856982856883E4F00569E56970B5
:108C7000020568028E6E8569828568837445F005F9
:108C800069E56970020568856982856883E4F00595
:108C900069E56970020568EB30E2248569828568C0
:108CA0008374C6F00569E569700205688569828587
:108CB0006883E9F00569E56970020568028E6E85D2
:108CC000698285688374E5F00569E5697002056865
:108CD0008569828568837401F00569E5697002051C
:108CE00068028E6E7908EB30E3034301407E08EBA7
:108CF00030E303430640EF64017003028D92E56A9E
:108D00005F604585698285688374F2F00569E5696D
:108D100070020568856982856883E4F00569E56904
:108D2000700205688569828568837422F00569E5AB
:108D300069700205688569828568837480F00569B9
:108D4000E5697002056880438569828568837422BD
:108D5000F00569E569700205688569828568837434
:108D600080F00569E5697002056885698285688318
:108D700074F2F00569E569700205688569828568A5
:108D800083E4F00569E56970020568EFC313FF022B
:108D90008CF6E56A5F606D85698285688374F2F0A0
:108DA0000569E56970020568856982856883E4F074
:108DB0000569E56970020568EB30E2248569828502
:108DC00068837411F00569E5697002056885698238
:108DD000856883EEF00569E56970020568028E6EAC
:108DE0008569828568837422F00569E569700205EA
:108DF000688569828568837480F00569E569700219
:108E00000568806A8569828568837422F00569E552
:108E100069700205688569828568837480F00569D8
:108E2000E56970020568EB30E22385698285688315
:108E300074E1F00569E569700205688569828568F5
:108E400083E9F00569E5697002056880218569821A
:108E500085688374F2F00569E569700205688569C3
:108E600082856883E4F00569E56970020568AC688D
:108E7000AD69AF05AE0422204A663049328F828E3A
:108E80008374E5F00FBF00010E8F828E837401F0B2
:108E90000FBF00010E8F828E837445F00FBF00015B
:108EA0000E8F828E83E4F00FBF00010E028F438F7E
:108EB000828E837445F00FBF00010E8F828E83E493
:108EC000F00FBF00010E8F828E8374E5F00FBF009C
:108ED000010E8F828E837401F00FBF00010E80633C
:108EE0003049318F828E8374F2F00FBF00010E8FF4
:108EF000828E83E4F00FBF00010E8F828E83742276
:108F0000F00FBF00010E8F828E837480F00FBF00C0
:108F1000010E802F8F828E837422F00FBF00010E0E
:108F20008F828E837480F00FBF00010E8F828E833C
:108F300074F2F00FBF00010E8F828E83E4F00FBF3A
:108F400000010E2290F0087407F075F003EFA4FD05
:108F5000ACF0F5828C83E0FEA3E0F98D828C83A3D4
:108F6000A3E0F56BEEB50103F0802CEEB56B088D38
:108F7000828C83A3F08020E9B56B08FE8D828C8300
:108F8000F08014EF90A05F93FE8D828C83F0A3F0AD
:108F90008D828C83A3A3F090F008E4F0EF909F5FA4
:108FA00093FDEEC39D400BEF90A15F93FDEED39D2B
:108FB0004007EF90A05F93FF22AF06228D6BAE07B4
:108FC00090F0087407F075F003EEA485F06CF56D71
:108FD000AF6BEE909F5F93FDEE90A15F93FB1296B7
:108FE000628F6B856D82856C83EFF0A3F0856D8257
:108FF000856C83A3A3F090F008E4F0AF6B22E4FF4C
:10900000128F447840EFF27F01128F4408EFF27F15
:1090100002128F447891EFF27F03128F4408EFF22F
:109020007F04128F44788CA607E6FB24F6FFE43415
:10903000FFFE7C017DF412CFB51C7D4912CFC978AB
:109040008EEEF208EFF27840E2FFEB8FF0A4FFAE75
:10905000F07891E2FD7C0012CFC9EF2B788CF67F7F
:1090600006128F44786DEFF27F08128F447835EF47
:10907000F27F09128F447838EFF27F0A128F448F03
:10908000337F0D128F44EF25E0147834F27F0E12F7
:109090008F44EF25E014784FF27F10128F447853FD
:1090A000EFF27F11128F44784EEFF27F12128F444D
:1090B0007859EFF27F13128F44780AEFF27F14127F
:1090C0008F4418EFF27F15128F449091BFEFF07F1D
:1090D00018128F447854EFF27F19128F4408EFF280
:1090E0007F1E128F44909191EFF07F1F128F44905A
:1090F0009197EFF07F20128F4490919DEFF07F21A8
:10910000128F449091A3EFF07F22128F449091A987
:10911000EFF07F23128F449091AFEFF07F24128FF6
:10912000449091B5EFF07F25128F449091BBEFF002
:109130007F28128F44909192EFF07F29128F4490F4
:109140009193EFF07F2A128F44909198EFF07F2B4C
:10915000128F44909199EFF07F2C128F4490919E42
:10916000EFF07F2D128F4490919FEFF07F2E128FA2
:10917000449091A4EFF07F2F128F449091A5EFF0CF
:109180007F30128F449091AAEFF07F31128F44907C
:1091900091ABEFF07F32128F449091B0EFF07F33BC
:1091A000128F449091B1EFF07F34128F449091B6BA
:1091B000EFF07F35128F449091B7EFF07F36128F2A
:1091C000449091BCEFF07F37128F449091BDEFF047
:1091D0007F38128F44909194EFF07F39128F449032
:1091E000919AEFF07F3A128F449091A0EFF07F3B7D
:1091F000128F449091A6EFF07F3C128F449091AC77
:10920000EFF07F3D128F449091B2EFF07F3E128FCE
:10921000449091B8EFF07F3F128F449091BEEFF0F1
:109220007F53128F447851EFF27F5A128F44EF3000
:10923000E003D38001C39213EF30E103D38001C375
:1092400092127F0B128F441297362290F001E0F5B4
:10925000665486FFBF80147882E26008E56654A6F3
:109260009091C0F0E56654A7783AF2E56654A7FFFE
:10927000783AE26F6021E4F55790F00DF0754B35C8
:10928000754C01754D0D12519B12519B12519BD281
:10929000AED2BEC2AF80FCE56620E6163093132046
:1092A000141020090D20150AD2091296FDC245128C
:1092B000955BE56620E333E55730E02ED3788BE607
:1092C000949A18E6940040227853E2D39401401A0D
:1092D0007856E2FF14F2EF7017D203D2141296FD03
:1092E0001296B2C24512955B8006784EE27856F22D
:1092F00020910E7860E2FF14F2EF700A1297298035
:10930000057860740AF278A1E644FCF690F00EF05D
:109310007857E220E10302939A788AE6FE08E68E07
:1093200064F565C3E56594A8E5649402400878A1F6
:10933000E6547FF6805DC3E565946AE56494024077
:109340000878A1E654BFF6804AC3E565942CE5642D
:109350009402400878A1E654DFF68037C3E56594AF
:10936000EEE5649401400878A1E654EFF68024C34A
:10937000E56594B0E5649401400878A1E654F7F6F9
:109380008011C3E5659472E5649401400678A1E616
:1093900054FBF678A1E690F00EF0E55744FCF55743
:1093A00090F00DF020B408547FF557F002946F78D8
:1093B00054E2FF3395E0FE783EE22FFFE43EFEC329
:1093C0007880E69FFF18E69EFEF5648F65D3EF94E4
:1093D000FFEE947F4005E4F564F565788EE2FE08C3
:1093E000E2FFC3E5659FE5649E400C78A1E6F45476
:1093F000FC44035257806DC3E5659499E56494017C
:109400004005535703804EC3E56594CCE564940052
:109410004005535783803EC3E5659444E56494005A
:1094200040055357C3802EC3E5659422E56494003C
:1094300040055357E3801EC3E565940DE564940031
:1094400040055357F3800EC3E5659406E564940028
:1094500040035357FB78A1E6FFF454FC4257E5570D
:1094600044035FF690F00DE557F078A1E6A3F020F5
:10947000210D30260AC24512955B12971EC2269016
:10948000F700E030E01012CAC47885E630E5077EC8
:109490009C7FC51203E27F0A227E01E4FDEDC394A6
:1094A00004400302955A74722DF8E2FC7003029591
:1094B0005275F02CECA42409F582E5F0344EAB8211
:1094C000F5598B5A74622DF8E2F47065E582241325
:1094D000F582E43559F583E0FCC313F98B82E5820C
:1094E000241AF582E43559F583E030E00343018026
:1094F0007C01E4FFEC603274052DF8E25CFBE95C72
:109500006B601FE26CF274622DF8EFF2E55A241AD8
:10951000F582E43559F583E06440F07843E24EF299
:10952000802EEC25E0FC0F80CB74722DF8E4F280E5
:109530001F74622DF8E2FC14F2EC6014E55A241A50
:10954000F582E43559F583E06440F07843E24EF269
:10955000E4FF0DEE25E0FE02949D22754B35754C1F
:1095600001300911754D03302131201531754C0240
:109570001297358026300C05754D0C801E30030582
:10958000754D038016301405754D02800E301E0592
:10959000754D018006204506E4F54D12519B229041
:1095A000F001E0F559209304C20F8002D20F300E73
:1095B000031296E6300F031296E7C2AFD2AED2BEC8
:1095C000D2AF7F507EC31203D37F04D244127D12E8
:1095D000783EEFF27F05D244127D12783FEFF21809
:1095E000E22403F208E22403F218E2FF1313543FCB
:1095F000788C26F6783FE2FF1313543F788F26F6D7
:10960000302109C2AFD2AED2BED2AF227FFFE4FD7D
:109610001285011296BD12971EE4F55A203DFD7F7A
:10962000FFE4FD128501C2AFD2AED2BED2AF055A61
:10963000E55AC3940A40E5E4FF7888E2FD1285010B
:109640001296CBE4F55A7FE27E041203D3C2AFD266
:10965000AED2BED2AF055AE55AC3940A40E812967C
:10966000BD22AE07EEC39D5003AF0522EED39B4053
:1096700003AF0322AF06228E658F66AA05A802E219
:10968000FE08E2FFC3E5669FFFE5659EFEAD037C35
:109690000012D01EA80208E22FFF18E23EFEAD0223
:1096A000A805F208EFF2227857E24402F290F00B9C
:1096B000F0227857E254FDF290F00BF02220160AC7
:1096C0007857E24402F290F00BF0227857E254FD12
:1096D000F290F00BF02230120A7857E254FDF2902B
:1096E000F00BF0A2122222E5574401F55790F00D3D
:1096F000F022E5574401F55790F00DF022E557545C
:10970000FEF55790F00DF02278A0E64480F690F038
:109710000CF02278A0E6547FF690F00CF0227857F7
:10972000E24408F290F00BF0227857E254F7F290FE
:10973000F00BF022222275985243D880EF25E024C6
:109740005FF582E434A3F583E493FC740193F5AAF6
:10975000EC5403F5BAC2B222E4FE74722EF8E26F42
:1097600060210EBE04F4E4FE74722EF8E27010EF75
:10977000F274052EF8EDF274622EF874FFF2220EE8
:10978000BE04E522C206754B33786AE2F54E784294
:10979000E2F54DE54DF4607730231E75F005E54E9A
:1097A000A42409F582E5F03490AF82F55D8F5E75F3
:1097B0004C03F583E0F54F80537836E2FE08E2FF74
:1097C0004E60087850E28F828E83F0754C0575F0FC
:1097D0000BE54EA42409F582E5F0347AAF82F55DFD
:1097E0008F5EE54D30E00BE4255EF55E740B355D74
:1097F000F55D855E82855D83E0F54FA3E0F55085DC
:109800005E82855D83A3A3E0F551C22712519B229E
:10981000E4F559F5607561FF75620AF5347834E254
:10982000F53B753F04754004203D6CE5346004153C
:10983000348061E559603E7F3F12052B7878E55909
:10984000F208E53BF2856034E5607004D21C8004C8
:10985000C21C1534E4F563E563C395595012745A7C
:109860002563F8E6FF747A2563F8EFF2056380E775
:10987000E4F559801F201C1C78787403F208E53B3E
:10988000F2787A74FFF2E4787BF2787C74FFF27FEE
:109890006912052B12851CE5087003029936E559FB
:1098A00060030299361203A18F55E555B4F00812F2
:1098B00003A18F3B029936E555B4F1071203A18F3E
:1098C0003F8073E555B4F21B753752D22B1296D6F2
:1098D0007F7212052B12413D7F5212052BE47884D2
:1098E000F68053E555B4F30280FEE55564F4704606
:1098F0001203A18F601203A18F59E55970087559A1
:10990000031296CB80031296BDE4F563E563C3951D
:1099100059501EE5632475FF12052B1203A1745ADA
:109920002563F8A607E5632455FF12052B05638020
:10993000DB7F2112052B7884E67003029828788457
:1099400016E540600ED5400B853F4090F002E0FFE9
:1099500012058DE561600ED5610B7561FF7F731295
:10996000052B127911E562600DD5620A7F6F120531
:109970002B12924B8F62202503029828C22575A0D6
:10998000FCC2AFD2AED2BED2AF0298282230106253
:10999000C210E4FF3017020F0FC205303F1E74E4FF
:1099A0002FF582E434EEF583E0602D74E52FF58227
:1099B000E434EEF583E06020D205801C74E02FF5DE
:1099C00082E434EEF583E0600F74E12FF582E43435
:1099D000EEF583E06002D2053005177850E2FF789B
:1099E00036E2FC08E2F5828C83EFF0E47883F21231
:1099F0009784301F04C21FD210224D5831206D6F42
:109A000064656C20454300202053573A4D5831453A
:109A10004300446F776E6C6F616400466C617368DD
:109A20002E2E2E00446F776E6C6F61642E2E2E00EA
:109A3000456D7066546573740D0A0045210D0A204A
:109A4000202000206D3D0020653D0020733D00205A
:109A50007A3D0020613D0020643D0020703D0020E3
:109A6000773D000D0A004E3A20004F3A20003F3F5C
:109A70003F3F3F3F3F3F0D003F3F620D003F3F6C88
:109A8000003F3F690D000D0A442D70633D006C617D
:109A90003D000D0A4D2D70633D0050726F673A20F6
:109AA000202020202020202020200050524720531A
:109AB000746172740A0049524546203E20302E32AD
:109AC00035410A0050524720494E49540A0050522D
:109AD00047204C4545524C4155460A004861726446
:109AE0007265736574005052472048415244524594
:109AF0005345540A0050524720502D55500A0050EB
:109B0000524720502D5550320A005052472049529A
:109B1000454620005052472049524546203E2030BD
:109B20002E3235410A004356003D2020200050527D
:109B30004720574F524B494E475F4449520A004E07
:109B40004F2041434B202D3E2050524720574F522B
:109B50004B494E475F4449525F454E44450A0050C9
:109B6000524720574F524B494E475F4449525F423C
:109B70005954450A0050524720574F524B494E47BF
:109B80005F504859530A00505247204300505247F3
:109B9000204552520050524720502D444E0A00504A
:109BA000524720414242525543480A0050524720F2
:109BB000456E640A000A5052472043563A004572E7
:109BC000726F723A20202020006873000D0A57003F
:109BD00043414E5F496E697420210A004E554C4C3A
:109BE000200020410020506E0020506D004C4F4757
:109BF0003A20496E69745072696F0A000A444343FF
:109C0000757365643A20000A4D4F54757365643A64
:109C10002000204F4646202000205545502020009F
:109C2000205545532020002041555320200020532B
:109C30005350202000204E6F20536900536574203C
:109C4000417578496E203C2D204F666620202020EB
:109C50002020202020202020202020200053657458
:109C600020417578496E203C2D204F6E2020202009
:109C700020202020202020202020202020004552AD
:109C8000523A2049204C6565726C617566207A7580
:109C900020686F636800204C61737420616E737478
:109CA00065636B656E00446174656E7665726C7594
:109CB0007374210D0A002020446174656E7665720C
:109CC0006C757374004255534F46463A43414E5F9C
:109CD000496E697420210A0020322E303300312E63
:109CE00030312E3030302052414D20696E204F727D
:109CF000646E756E670009090909090909090909EE
:109D00000909090909090A0A0A0A090909090909BF
:109D10000808080808080A0A0A0A0A0A09090908B4
:109D20000808070707070C0C0B0B0B0A09090808A2
:109D30000808070707070D0D0C0B0B0A090908088F
:109D40000707070606060E0E0E0C0A0A0909080880
:109D50000707060606060F0F0E0E0B0A090808076E
:109D600007070606060610100F0D0C0A090807065D
:109D700006060505050510100E0C0B0A0908070656
:109D80000505060707070F0F0E0C0B0A0908070643
:109D90000505050608080E0E0D0B0A09080706053D
:109DA0000607080809090D0D0C0A09080707060629
:109DB0000708080909090C0C0B0A09080707070717
:109DC000070809090A0A0B0B0A090807070707070A
:109DD0000809090A0A0A0A0A0909080807070708F8
:109DE0000809090A0B0B09090808080707080809E8
:109DF000090A0A0B0B0BAAC08030F0B020E0A00CBF
:109E0000CC8C3CFCBC2CECAC08C88838F8B828E8F2
:109E1000A803C38333F3B323E3A30FCF8F3FFFBF65
:109E20002FEFAF0BCB8B3BFBBB2BEBAB02C28232DA
:109E3000F2B222E2A20ECE8E3EFEBE2EEEAE0ACAD6
:109E40008A3AFABA2AEA0000C030F00CCC3CFC0393
:109E5000C333F30FCF3FFF50505044505050505039
:109E600050505050505050515151515151515151E9
:109E70005151115151515104040404440404040487
:109E80000404040404040405050505050505050589
:109E900005050511050505141414141414441414AF
:109EA0001414141414141415151515151515151569
:109EB000151515151511155454545454545444542F
:109EC0005454545454545455555555555555555549
:109ED0005555555555551101020103010201040163
:109EE0000201030102010401020103010201040154
:109EF0000201030102010001020103010201040148
:109F00000201030102010401020103010201040133
:109F10000201030102010401020103010201040123
:109F20000201030102010001020103010201040117
:109F30000201030102010401020103010201040103
:109F400002010301020104010201030102010401F3
:109F500002010301020100010204081020408001F7
:109F6000010101010101015A5A9201000A14000184
:109F700001000101010000000000000000000000DD
:109F800000000000000000000000000000000000D1
:109F9000000000000000000B0B0B0B0B0B0B0B0069
:109FA00000000000000000000000000000000001B0
:109FB000010100000000000000000000000000009F
:109FC0000000000000000000000000000000000091
:109FD0000000000000000000000000000000000081
:109FE0000000000000000000000000000000000071
:109FF0000000000000000000000000000000000061
:10A000000000000000000000000000000000000050
:10A010000000000000000000000000000000000040
:10A020000000000000000000000000000000000030
:10A030000000000000000000000000000000000020
:10A040000000000000000000000000000000000010
:10A050000000000000000000000000000000003FC1
:10A060000058005000FA006600A204001A1700020F
:10A070000A00FF644600000000010000000000002C
:10A0800000000000000000000000000000000000D0
:10A0900000000000000000000000000000000000C0
:10A0A00000000000000000000000000000000007A9
:10A0B0000707000000000000000000000000000092
:10A0C0000000000000000000000000000000000090
:10A0D0000000000000000000000000000000000080
:10A0E0000000000000000000000000000000000070
:10A0F0000000000000000000000000000000000060
:10A10000000000000000000000000000000000004F
:10A11000000000000000000000000000000000003F
:10A12000000000000000000000000000000000002F
:10A13000000000000000000000000000000000001F
:10A14000000000000000000000000000000000000F
:10A150000000000000000000000000000000007887
:10A160007878789650FEFE6E6EA206001E1E0005E0
:10A17000FE7FFFFFFFFFFFFFFF0101000006060655
:10A1800006060606060000FFFFFFFFFFFFFFFFFFBA
:10A19000FFFFFFFFFFFFFF636363636363636300AE
:10A1A00000000000000000000000000000000007A8
:10A1B0000907FF000000000000030000000000008D
:10A1C000000000000000000000000000000000008F
:10A1D000000000000000000000000000000000007F
:10A1E000000000000000000000000000000000006F
:10A1F000000000000000000000000000000000005F
:10A20000000000000000000000000000000000004E
:10A21000000000000000000000000000000000003E
:10A22000000000000000000000000000000000002E
:10A23000000000000000000000000000000000001E
:10A24000000000000000000000000000000000000E
:10A2500000000000000000000000000000000000FE
:10A2600000000001010101010101010101010101E1
:10A2700001010101010303010103000101010101C9
:10A2800001010101010101010101010101010101BE
:10A2900001010101010101010101010101010101AE
:10A2A000010101010101010101010101010101019E
:10A2B000010101010101010101010101010101018E
:10A2C000010101010101010101010101010101017E
:10A2D0000101010101010100000000000000000077
:10A2E000000000000000000000000000000000006E
:10A2F000000000000000000000000000000000005E
:10A30000000000000000000000000000000000004D
:10A31000000000000000000000000000000000003D
:10A32000000000000000000000000000000000002D
:10A33000000000000000000000000000000000001D
:10A34000000000000000000000000000000000000D
:10A3500000000000000000000000000000000003FA
:10A36000CC02600330039803CC03E603F3102040D3
:10A370008000000000546573742052616D0A00462D
:10A38000696C6C2042616E6B2000546573742042CE
:10A39000616E6B20004665686C65722042616E6B71
:10A3A000200052616D204F4B2120200A0052616D28
:10A3B000204665686C657268616674210A00018CCC
:10A3C00096018F96816DFA816FFA81600A810DFF87
:10A3D000815200818841813D64013400013B41018B
:10A3E0003D41019400013103013800C122A0201435
:10A3F000202020202020202020202020202020205D
:10A40000202020202020202020202020202020204C
:10A41000013614818164814D1E012A22012B00C165
:10A4200001012C00C1BDC1BE00E541543FF56DC323
:10A430009440400302A82D85436E74C4256DF582B7
:10A44000E43491F5837418F0E54254E0FF700A7526
:10A450004B18754C01856D4D22EF6420600302A8F6
:10A460002DE543C39408400302A82DE542540F1480
:10A47000F56F64026009E56F6406600302A82D753C
:10A480004B1AE543C43354E04401F54C856D4D123D
:10A49000519B75F070E56DA42418F582E5F0340049
:10A4A000F58375F00EE54312D054AF8285836B8F30
:10A4B0006C85436EE0F54AAE6B7D44AB6F12CBE822
:10A4C000202D0302A79220300302A792E5455430C5
:10A4D000700302A82DE4F551E5434480F54AE545B3
:10A4E00030E403434A08E5455403FFC454F0424AAC
:10A4F000303B45755180C23B78B2E6FE08E6FFF579
:10A50000828E83E54AF0A3E56DF020380302A72B85
:10A51000C23878ADA60608A6077885E620E40302CF
:10A52000A72B754B63754C0278ADE608E6F54DEE4A
:10A53000F54E12519B02A72B20370302A5FF78B7D7
:10A54000E6FE08E6FFF5828E83A3E0656D70548F0A
:10A55000828E83E054CFFFE54A54CF6F7045E54AC1
:10A56000F0E4F5517885E620E40302A82D754B65EB
:10A57000754C0778B7E6FC08E6FDECF54DAF05EF46
:10A58000F54EF5828C83E0F54FA3E0F5507551014F
:10A5900078ADE6FC08E6FDECF552AF05EFF5531299
:10A5A000519B2278B8740226F618E436F6FE08E6C7
:10A5B000F5828E83E0700D78AEE6240279B8F71844
:10A5C000E43619F778B7E6FE08E6F5828E83E0FFF9
:10A5D00054C0FEBE80CDA3E0B56D1EEF54CFFFE5A5
:10A5E0004A54CFB5071378B7E6FE08E6F5828E83A6
:10A5F000E54AF075510102A56475511002A6A078D4
:10A60000B2E6FE08E6FFF5828E83A3E0B56D188FF3
:10A61000828E83E054CFFFE54A54CFB507097551C8
:10A6200040E54AF002A72B78B3740226F618E43608
:10A63000F6901C1CE02402F0901C1BE03400F0306B
:10A64000384DC238E6FE08E678ADA60608F67885ED
:10A65000E630E414754B64754C0278ADE6FE08E60E
:10A66000F54DEEF54E12519BC3901C1CE094549096
:10A670001C1BE0942A4004D22C802578B2E6FE0808
:10A68000E6F5828E83E54AF0A3E56DF002A72BC3C1
:10A69000901C1CE09454901C1BE0942A4041D22C46
:10A6A000C22DD231901C95E0FFA3E0901C1BCFF08F
:10A6B000A3EFF0E4901C95F0A3F0901C19E0FEA32A
:10A6C000E0F5828E83E4F0A3F0201E5F20145CD2BC
:10A6D0001E754B35754C01754D0112519B804C78A0
:10A6E000B2E6FE08E6FFF5828E83E54AF0A3E56D4B
:10A6F000F020383778ADE6FC08E6FDF5828C83A3C0
:10A70000E0B56D03D38001C350218D828C83E0546A
:10A71000CFFDE54A54CFB50503D38001C3500C7576
:10A720005108D23778B7A60608A60778B2E6FE0821
:10A73000E6FFF5828E83A3A3E4F08F828E83A3A32A
:10A74000A3F07885E620E40302A82D754B62754CD2
:10A750000878B2E6FC08E6FDECF54DAF05EFF54EE6
:10A76000F5828C83E0F54FA3E0F550302D03435183
:10A770000130370343510278B7E6FC08E6FDECF5FB
:10A7800052AF05EFF55378ADE6FE08E6F5541251E9
:10A790009B22303A0CAF6CAE6BAD6DAB4312B9E19E
:10A7A0002220360302A82DE56C2408F582E4356BDF
:10A7B000F583E030E63AE5445498FFE54A54986F53
:10A7C000606BE54AA2E3500FE544A2E34009AF6C99
:10A7D000AE6BD24712A82EE54AA2E34013E544A28D
:10A7E000E3500DAF6CAE6BAD6DAB6ED24712AA2BC2
:10A7F000E56C240CF582E4356BF583E030E62EE55C
:10A800004AA2E4500FE544A2E44009AF6CAE6BC22B
:10A810004712A82EE54AA2E44013E544A2E4500DF5
:10A82000AF6CAE6BAD6DAB6EC24712AA2B228E70B1
:10A830008F7130470512CA7C8007AF71AE7012CAA3
:10A840009D304714E51054BFFFE5712406F582E4FE
:10A850003570F583EFF08012E51054BFFFE57124E9
:10A860000AF582E43570F583EFF075740A30470419
:10A870007F0880027F10E50E5F600302AA2AE513BD
:10A8800020E756E51020E70302AA2AAF741574EFFB
:10A89000700302AA2AE510543FF572E5115407F53A
:10A8A0007375F070E572A42418F582E5F03400F5B4
:10A8B0008375F00EE57312D054AF828583708F716B
:10A8C000E511A2E39247304707AE7012CA7C809D23
:10A8D000AF71AE7012CA9D809475740AE51220E7BC
:10A8E0000302AA2AE512543FF572E5135407F573E3
:10A8F00075F070E572A42418F582E5F03400F58354
:10A9000075F00EE57312D054AF828583708F71E5B8
:10A9100013A2E39247304707AE7012CA7C8007AF9C
:10A9200071AE7012CA9DE51320E7193047047F0805
:10A9300080027F10E50E5F600302AA2AAF741574CF
:10A94000EF709922C248C249754B1BE573C433545A
:10A95000E04403F54C85724D754E03E5734408F5EC
:10A960004F3047047F0880027F10E50E5F6002D2FF
:10A970004975740A30492C204829304714E5105491
:10A98000BFFFE5712406F582E43570F583EFF080B2
:10A9900012E51054BFFFE571240AF582E43570F525
:10A9A00083EFF012519BAF741574EF700302AA2A63
:10A9B000E51230E775E512543FF572E5135407F5DB
:10A9C0007375F070E572A42418F582E5F03400F593
:10A9D0008375F00EE57312D054AF828583708F714A
:10A9E000E513A2E39247304707AE7012CA7C800796
:10A9F000AF71AE7012CA9DE51330E702D2483048FD
:10AA0000133047047F0880027F10E50E5F601BE56E
:10AA10001030E616754B1BE573C43354E04402F561
:10AA20004C85724D754E0302A974228E708F718D04
:10AA3000728B7330470512CA7C8007AF71AE7012FB
:10AA4000CA9DE511C4540F5407F54EC249E51230B2
:10AA5000E74BE51330E324E512543F75F070A4246E
:10AA600021F582E5F03400F583E513540775F00E07
:10AA700012D054E030E726D2498022E512543F75C7
:10AA8000F070A42425F582E5F03400F583E5135435
:10AA90000775F00E12D054E030E702D24975740AFF
:10AAA000E51320E763E51020E70302ACBCE5105492
:10AAB0003FF572E5115407F57375F070E572A42443
:10AAC00018F582E5F03400F58375F00EE57312D0C9
:10AAD00054AF828583708F71E511A2E392473047AE
:10AAE00007AE7012CA7C8007AF71AE7012CA9DAFFC
:10AAF000741574EF700302ACBC3047047F08800209
:10AB00007F10E50E5F609922851254851353754BB3
:10AB10001BE573C43354E0F54C85724D85734FE5E6
:10AB200011C4540F54076006434C0202ABB2E51047
:10AB300020E705434C03807A75740AE510543FF50D
:10AB400072E5115407F57375F070E572A42418F5D9
:10AB500082E5F03400F58375F00EE57312D054AF42
:10AB6000828583708F71E511A2E39247304707AE6B
:10AB70007012CA7C8007AF71AE7012CA9D30470454
:10AB80007F0880027F10E50E5F6005434C03802242
:10AB9000E51330E70B434C03754E03434F08801217
:10ABA000E51020E705434C038008AF741574EF707F
:10ABB0008A2212519BE55420E70302ACBCE55454B1
:10ABC0003FF572E5535407F573E553A2E39247C28C
:10ABD00048C24A75740A75F070E572A42418F582AB
:10ABE000E5F03400F58375F00EE57312D054AF82B2
:10ABF0008583708F71304707AE7012CA7C8007AFB3
:10AC000071AE7012CA9D85724D85734FE51330E7A2
:10AC100021304A0EC249E573C43354E04402F54C76
:10AC2000800CE573C43354E04403F54CD24AD24857
:10AC3000800AE573C43354E04402F54C30480E30CA
:10AC400047047F0880027F10E50E5F606F30492760
:10AC5000304824431040304710E5712406F582E463
:10AC60003570F583E510F0800EE571240AF582E475
:10AC70003570F583E510F0304805E51030E63DE528
:10AC80000F5407B54E08E54C5407FFBF030D125192
:10AC90009B857182857083A3E54EF0AF741574EFC8
:10ACA000601AE51230E715E512543FF572E51354CA
:10ACB00007F573E513A2E3924702ABD622E541B450
:10ACC0001912E543B4630DD230202D3F202E3CD223
:10ACD0003AD22F22E541641C7031E5436463702B46
:10ACE000C2307E007F18C3EE941C50178F828E8373
:10ACF0007418F0740E2FFFE43EFE740E2FFFE43E36
:10AD0000FE80E3303A05C23A12BEAE22202D030285
:10AD1000ADEC303B0302ADEC5344074344C07885AF
:10AD2000E630E429754B66754C0678B2E6FC08E619
:10AD3000FDECF54DAF05EFF54EF5828C83E0F54F58
:10AD4000A3E0F55085445185435212519B78B2E6F9
:10AD5000FE08E6F5828E83E0B5441EA3E0B54319F4
:10AD600018E608E6FFF5828E83E544F0A3A3E4F03D
:10AD70008F828E83A3A3A3F02278B3740226F618E1
:10AD8000E436F6901C1CE02402F0901C1BE034001A
:10AD9000F0C3A3E09454901C1BE0942A402CD22CC6
:10ADA000C22DD231901C95E0FFA3E0901C1BCFF088
:10ADB000A3EFF0E4901C95F0A3F0901C19E0FEA323
:10ADC000E0F5828E83E4F0A3F02278B2E6FE08E696
:10ADD000FFF5828E83E544F0A3E543F08F828E83F6
:10ADE000A3A3E4F08F828E83A3A3A3F022203103D8
:10ADF00002AF03754B37754C0578AFE6F54D302D36
:10AE00000778A7E6F54E8003854D4E75F012E54EA6
:10AE1000A424A1F582E5F0341CAF8278ABF608A635
:10AE200007E4F551F550F54FF55FE54F1313543F27
:10AE3000F54F302D0B78AAE6B55F05434FC0802251
:10AE400078ABE6FE08E6FFF5828E83E0FCA3E04CDB
:10AE500060108F828E83E030E705434F808003438C
:10AE60004F4078AC740226F618E436F6055FE55FCD
:10AE7000B404B7E55FC394085046E5501313543F3C
:10AE8000F550302D0B78AAE6B55F054350C08022FF
:10AE900078ABE6FE08E6FFF5828E83E0FCA3E04C8B
:10AEA00060108F828E83E030E7054350808003433B
:10AEB000504078AC740226F618E436F6055F80B38D
:10AEC000E55FC394095030302D0B78AAE6B55F05D5
:10AED000435103802278ABE6FE08E6FFF5828E83BD
:10AEE000E0FCA3E04C60108F828E83E030E70543E6
:10AEF00051028003435101302C0343518012519B76
:10AF0000C231227896E2F56024C4F582E43491F5EA
:10AF100083E0700302B01974C42560F582E43491B3
:10AF2000F583E014F0704175F070E560A42418F525
:10AF300082E5F03400AF82F55B8F5CE4F55F855C01
:10AF400082855B837418F0740E255CF55CE4355BD8
:10AF5000F55B055FE55FB408E5754B19754C018538
:10AF6000604D12519B02B019303A0302B019302ED5
:10AF70000302B0197893E26560600302B01975F0BE
:10AF800070E560A42418F582E5F03400AF82F55B2B
:10AF90008F5CF583E030E775E582240EF582E435B9
:10AFA00083F583E030E7668F82E582241CF582E436
:10AFB000355BF583E030E7558F82E582242AF58200
:10AFC000E4355BF583E030E7448F82E5822438F591
:10AFD00082E4355BF583E030E7338F82E5822446F7
:10AFE000F582E4355BF583E030E7228F82E5822449
:10AFF00054F582E4355BF583E030E7118F82E5821A
:10B000002462F582E4355BF583E020E70C754B198B
:10B01000754C0185604D12519B7896E204F2C39401
:10B02000404026E4F2F55F7893E204F2C394404096
:10B0300002E4F27893E224C4F582E43491F583E0EB
:10B040007007055FE55FB40ADE30350302B2FE200B
:10B05000391B9091BFE0FF901C18E0FE04F0EEC396
:10B060009F500302B2FED239E4F078B6F678B6E625
:10B07000FFC39414400302B2FC74452FF582E434FC
:10B080001CF583E06401600302B2F6EF25E0246D55
:10B09000F582E4341CF583E0FEA3E08E5DF55E05E9
:10B0A0005EE55EAE5D7002055D14F5828E83E0F5AF
:10B0B0004F055EE55EAE5D7002055D14F5828E8320
:10B0C000E0F54D7885E630E413754B60754C0478F7
:10B0D000B6E6F54E7897E2F55012519BE54F7003B6
:10B0E00002B250E54F20E70302B1A7303A0302B2A3
:10B0F000F67897E2FFF46009EF78B666600302B273
:10B10000F678B6E67897F2202E04D22ED22FE54DAF
:10B11000543FF560E54F30E61C754B1B534F07E578
:10B120004FC43354E04403F54C434F08E4F54E124A
:10B13000519B02B09FE56044C0F541754223E54F45
:10B140005407F5437544C0E54F5430FFC4540FF520
:10B1500045E54F30E3084344084345108006434427
:10B160001043452075F070E560A42418F582E5F0E1
:10B170003400F58375F00EE54312D054AF82858319
:10B180005B8F5C754B1B534F07E54FC43354E04452
:10B1900003F54CE4F54E12519BAF5CAE5BAD60AB7A
:10B1A0004312B9E102B09FE54F30E549E54D30E784
:10B1B0002E30060302B2F6754B4D75414D754C03AA
:10B1C000754203E54D547FF54EF544534F0F854FBF
:10B1D00045754D0475430412519B1266BC8051E5C0
:10B1E0004D543F4480F54B754CA1E54F545FF54DF0
:10B1F00012519B803BE54F30E63630060302B2F633
:10B20000754B4D75414D754C03754203AF4D8F4ED7
:10B210008F44E54F30E408754D017543018005E426
:10B22000F54DF543534F0F854F4512519B1266BCA8
:10B23000855E82855D83E0601778B6E625E0246D43
:10B24000F582E4341CF583E55DF0A3E55EF00622AB
:10B250007897E278B666702C789774FFF212BEAEDB
:10B26000C22E78B6E6FF25E0246DF582E4341CF5A5
:10B2700083E4F0A3F074452FF582E4341CF5837465
:10B2800002F0806E78B6E6FD25E0241DF582E434F8
:10B290001CF583A3E025E0FF0582D5820215831506
:10B2A00082E033FE74A12FF582EE341CAF82F55D8F
:10B2B0008F5EF583E0547FF074452DF582E4341CF5
:10B2C000F583E4F0ED25E0246DF582E4341CF5838C
:10B2D000E4F0A3F0ED25E0241DF582E4341CF583B1
:10B2E000E0FEA3E0FF7C007D0912CFC978AFA6077E
:10B2F000D23178B6062278B60602B06DC23922D2B3
:10B3000007789774FFF220220D901C19E07002A3B9
:10B31000E0600302B39B7E077F087D007B027A1CFE
:10B3200079A112D0607E007F147D007B027A1C79A7
:10B330004512D0607E007F287D007B027A1C796DEB
:10B3400012D0607E007F287D007B027A1C791D125E
:10B35000D060E49023A9F0A3F0A3F0A3F0901C190F
:10B360007423F0A374ABF0901C1BE4F0A37402F000
:10B37000E4901C95F0A3F0909209F0A3F09092064F
:10B38000F0A3F09091C3F09091C1F0909204F090EE
:10B390009208F0909205F09091C2F0901C95E0FE1A
:10B3A000A3E0FF4E601D901C1BEEF0A3EFF0901C7D
:10B3B00019E0FEA3E0F5828E83E4F0A3F0901C95E3
:10B3C000F0A3F07E007F18E4FDE4FC8F828E83748E
:10B3D00018F0A3E4F0EF2406F582E43EF583E05490
:10B3E000BFF0EF240AF582E43EF583E054BFF0EFAE
:10B3F0002407F582E43EF583E030E72CEF2406F5E0
:10B4000082E43EF583E4F0EF2407F582E43EF58321
:10B41000E4F0EF2408F582E43EF583E4F0EF24093C
:10B42000F582E43EF583E4F0EF240BF582E43EF58B
:10B4300083E030E72CEF240AF582E43EF583E4F064
:10B44000EF240BF582E43EF583E4F0EF240CF58263
:10B45000E43EF583E4F0EF240DF582E43EF583E469
:10B46000F0740E2FFFE43EFE0CEC6408600302B3A0
:10B47000CB0DED6440600302B3C9C2072278AFA6CA
:10B4800043C22CD2312230350302B7FCC22CD23158
:10B4900078AFA643E54375F009A4FFAEF0E5445448
:10B4A0000FFD7A002FF56CEA3EF56BE56C25E0FFA9
:10B4B000E56B33FE74A12FF582EE341CAF8278ABBE
:10B4C000F608A607302D73E54378A766600302B738
:10B4D000FCED78AA66600302B7FCC22D303B030284
:10B4E000B7FC901C19E0FEA3E0FF08E6FC08E6F5B7
:10B4F000828C83EEF0A3EFF078B2E6FE08E6FFF56B
:10B50000828E83A3A3E4F08F828E83A3A3A3F09003
:10B510001C1CE02404F0901C1BE03400F0EF240419
:10B52000FFE43EFE901C19F0A3EFF0F5828E83E459
:10B53000F0A3F0901C95F0A3F02278ABE6FE08E6AD
:10B54000FFF5828E83E0FCA3E078B0A60408F6E560
:10B550004454C06480706530330302B7FC3032035A
:10B5600002B7FC78B1E61846600302B7FC303A0334
:10B5700002B7FC78A7A643E544540F78AAF6901CBE
:10B580001BE0FCA3E0FDC39448EC942A502B901CD4
:10B5900019E0FAA3E078B0A60208F608A60208F6B9
:10B5A000D22DD23BD238C237F5828A83E4F0A3F0A1
:10B5B000901C95ECF0A3EDF022D22C2278B0E6FCA2
:10B5C00008E6FD4C700302B7FCE54430E64BEC3076
:10B5D000E70302B7FC8F828E83E4F0A3F078B2A673
:10B5E0000408A60508F608760278B0E6FE08E6F537
:10B5F000828E83E0601678B5740226F618E436F67B
:10B6000078B1740226F618E436F680DD78B174025B
:10B6100026F618E436F6D2352278B0E60820E7039D
:10B6200002B79578ABE6FE08E6F5828E83E0547F9C
:10B63000F0E4F56DE56D25E0241DF582E4341CF59C
:10B6400083E0FEA3E0656C7003EE656B6007056D3B
:10B65000E56DB414DFE56D6414700302B7FC744546
:10B66000256DF582E4341CF583E4F0E56D25E024D6
:10B670006DF582E4341CF583E4F0A3F07897E2B52D
:10B680006D07C22EC22F74FFF278ABE6FE08E6F516
:10B69000828E83E0FEA3E078B0A60608F678B008B4
:10B6A00006E618860670010614F5828E83E0F54FD3
:10B6B00078B00806E618860670010614F5828E83B7
:10B6C000E0F54D7885E630E40C754B61754C0285EC
:10B6D0004F4E12519BE54F700302B7FCE54F54C02B
:10B6E000FFBF80B9E54D543FF56E75F070A4241886
:10B6F000F582E5F03400F583E54F540775F00E123E
:10B70000D054AF82AE83E54F30E342E5822406F5A4
:10B7100082E43583F583E4F08F828E83E58224070B
:10B72000F582E43583F583E4F08F828E83E582240D
:10B7300008F582E43583F583E4F08F828E83E58219
:10B740002409F582E43583F583E4F0802CEF240AA4
:10B75000F582E43EF583E4F0EF240BF582E43EF558
:10B7600083E4F0EF240CF582E43EF583E4F0EF246B
:10B770000DF582E43EF583E4F0754B1B534F07E56E
:10B780004FC43354E04403F54C856E4DE4F54E123E
:10B79000519B02B69DE4F56D7445256DF582E43448
:10B7A0001CF583E06007056DE56DB414EBE56D6491
:10B7B000146049E56D25E0241DF582E4341CF58311
:10B7C000E56BF0A3E56CF07445256DF582E4341C5F
:10B7D000F5837401F078B0E6FE08E6FFE56D25E03C
:10B7E000246DF582E4341CF583EEF0A3EFF078AB22
:10B7F000E6FE08E6F5828E83E04480F022202D03E9
:10B8000002B8DC53435F43432053413F303B25C2E2
:10B810003B78B2E6FE08E6FFF5828E83E543F0A3AF
:10B82000E541F08F828E83A3A3E4F08F828E83A301
:10B83000A3A3F02278B2E6FE08E6FFF5828E83A38A
:10B84000E0654170248F828E83E0541FFFE54354EE
:10B850001FB5071518E608E6FFE543F0A3A3E4F0DB
:10B860008F828E83A3A3A3F02278B3740226F618E6
:10B87000E436F6901C1CE02402F0901C1BE034001F
:10B88000F0C3A3E09452901C1BE0942A402CD22CCD
:10B89000C22DD231901C95E0FFA3E0901C1BCFF08D
:10B8A000A3EFF0E4901C95F0A3F0901C19E0FEA328
:10B8B000E0F5828E83E4F0A3F02278B2E6FE08E69B
:10B8C000FFF5828E83E543F0A3E541F08F828E83FE
:10B8D000A3A3E4F08F828E83A3A3A3F022202D03E1
:10B8E00002B9E0E54330E210E545540F4420F54944
:10B8F000E5444480F54A8013E545540F4440F5493A
:10B90000E54330E00343491085444A303B25C23BC0
:10B9100078B2E6FE08E6FFF5828E83E549F0A3E5FE
:10B920004AF08F828E83A3A3E4F08F828E83A3A339
:10B93000A3F022E54320E23578B2E6FE08E6FFF503
:10B94000828E83A3E0654A70248F828E83E0541731
:10B95000FFE5495417B5071518E608E6FFE549F075
:10B96000A3A3E4F08F828E83A3A3A3F02278B37401
:10B970000226F618E436F6901C1CE02402F0901C17
:10B980001BE03400F0C3A3E09452901C1BE0942A07
:10B99000402CD22CC22DD231901C95E0FFA3E09018
:10B9A0001C1BCFF0A3EFF0E4901C95F0A3F0901CCB
:10B9B00019E0FEA3E0F5828E83E4F0A3F02278B2D2
:10B9C000E6FE08E6FFF5828E83E549F0A3E54AF03E
:10B9D0008F828E83A3A3E4F08F828E83A3A3A3F030
:10B9E000228E708F718D728B73E545543070030217
:10B9F000BEADE545A2E49247304709AF71AE701283
:10BA0000CA7C8007AF71AE7012CA9D302F3D9092F4
:10BA100006E570F0A3E571F0909204E572F0909263
:10BA200008E573F0A247E433FF9091C1F0909209CA
:10BA3000E570F0A3E571F0909205E572F09091C287
:10BA4000E573F0A3EFF0C22F02BAF1909205E0B5D2
:10BA500072149091C2E0B5730DA247E433FFA3E0E6
:10BA60006F700302BE6D304708E5734488F574803B
:10BA700006E5734480F5749091C3E06029E5724453
:10BA800080FF909209E0FCA3E0FD2406F582E43CEF
:10BA9000F583EFF0ED2407F582E43CF583E054F004
:10BAA000F04574F08027E5724480FF909209E0FC35
:10BAB000A3E0FD240AF582E43CF583EFF0ED240BCE
:10BAC000F582E43CF583E054F0F04574F09092097F
:10BAD000E570F0A3E571F0909205E572F09091C2E7
:10BAE000E573F0A247E433A3F0E51130E70302BEAB
:10BAF0006D304714E5114480FFE5712407F582E4B9
:10BB00003570F583EFF08012E5114480FFE5712474
:10BB10000BF582E43570F583EFF0E51020E70302C2
:10BB2000BC8DE510543FF57285117330471DE571EA
:10BB30002406F582E43570F583E4F0E5712407F519
:10BB400082E43570F5837480F0801BE571240AF57A
:10BB500082E43570F583E4F0E571240BF582E43579
:10BB600070F5837480F0E573A2E392475373077511
:10BB7000F070E572A42418F582E5F03400F58375C1
:10BB8000F00EE57312D054AF828583708F71304709
:10BB90003CE5822407F582E43583F583E030E70352
:10BBA00002BC70E5712408F582E43570F583E4F099
:10BBB000E5712409F582E43570F583E4F0E571243C
:10BBC00006F582E43570F583E0F572803AE571247C
:10BBD0000BF582E43570F583E030E70302BC70E5D5
:10BBE00071240CF582E43570F583E4F0E571240DE1
:10BBF000F582E43570F583E4F0E571240AF582E41A
:10BC00003570F583E0F572E57230E76430472AE578
:10BC1000712407F582E43570F583E0F573E571244E
:10BC200006F582E43570F583E4F0E5712407F582CA
:10BC3000E43570F583E4F08028E571240BF582E4A7
:10BC40003570F583E0F573E571240AF582E435700B
:10BC5000F583E4F0E571240BF582E43570F583E4B7
:10BC6000F0E573A2E3924753730753723F02BB6F31
:10BC7000909209E0FEA3E08E70F571909205E0F5D8
:10BC8000729091C2E0F573A3E024FF9247E5122081
:10BC9000E70302BDFEE512543FF57285137330478A
:10BCA0001CE5712408F582E43570F583E4F0E57154
:10BCB0002409F582E43570F583E4F0801AE57124F7
:10BCC0000CF582E43570F583E4F0E571240DF5821E
:10BCD000E43570F583E4F0E573A2E392475373070C
:10BCE00075F070E572A42418F582E5F03400F58350
:10BCF00075F00EE57312D054AF828583708F71306A
:10BD0000474AE5822407F582E43583F583E030E78E
:10BD10000302BDE1E5712406F582E43570F583E4A4
:10BD2000F0E5712407F582E43570F583E4F0E57100
:10BD30002408F582E43570F583E0F572E571240995
:10BD4000F582E43570F583E0F5738048E571240BE6
:10BD5000F582E43570F583E030E70302BDE1E5717B
:10BD6000240AF582E43570F583E4F0E571240BF5DF
:10BD700082E43570F583E4F0E571240CF582E43556
:10BD800070F583E0F572E571240DF582E43570F508
:10BD900083E0F57330471CE5712408F582E43570C3
:10BDA000F583E4F0E5712409F582E43570F583E468
:10BDB000F0801AE571240CF582E43570F583E4F027
:10BDC000E571240DF582E43570F583E4F0E5723019
:10BDD000E70FE573A2E3924753730753723F02BC28
:10BDE000E0909209E0FEA3E08E70F571909205E07C
:10BDF000F5729091C2E0F573A3E024FF92473047BB
:10BE000037E5712406F582E43570F583E4F0E571D9
:10BE10002407F582E43570F5837480F0E571240819
:10BE2000F582E43570F583E4F0E5712409F582E4E8
:10BE30003570F583E4F08035E571240AF582E43548
:10BE400070F583E4F0E571240BF582E43570F58339
:10BE50007480F0E571240CF582E43570F583E4F02C
:10BE6000E571240DF582E43570F583E4F030471F69
:10BE7000E5455407FFC454F0FFE511548F44804F4B
:10BE8000FFE5712407F582E43570F583EFF022E5D4
:10BE9000455407FFC454F0FFE511548F44804FFF11
:10BEA000E571240BF582E43570F583EFF022302F35
:10BEB0000302C198909206E0FEA3E08E6DF56E90AD
:10BEC0009204E0F573909208E0F5719091C1E0243E
:10BED000FF9247856E82856D837418F0304723AFDB
:10BEE0006EAE6D12CA7CE51120E70302C198E51120
:10BEF000547FFFE56E2407F582E4356DF583EFF09E
:10BF00008021AF6EAE6D12CA9DE51120E70302C11C
:10BF100098E511547FFFE56E240BF582E4356DF54D
:10BF200083EFF0E510543FFF6573600302BFAEE599
:10BF300011540765717077E511A2E3304701B340F2
:10BF40006D304735E56E2406F582E4356DF583E402
:10BF5000F0E56E2407F582E4356DF583E4F0E56ED7
:10BF60002408F582E4356DF583E4F0E56E2409F5E7
:10BF700082E4356DF583E4F022E56E240AF582E46F
:10BF8000356DF583E4F0E56E240BF582E4356DF54F
:10BF900083E4F0E56E240CF582E4356DF583E4F07E
:10BFA000E56E240DF582E4356DF583E4F02220473B
:10BFB0000302C06EE56E2408F582E4356DF583E07A
:10BFC0004440F0E51020E725E51220E710E56E2457
:10BFD00008F582E4356DF583E054BFF022E56E2468
:10BFE00009F582E4356DF583E04480F0228F74E535
:10BFF000115407F572E511A2E3924875F070E574EB
:10C00000A42418F582E5F03400F58375F00EE5728E
:10C0100012D054AD8285836F8D70304816E582242E
:10C0200007F582E43583F583E0FEC4540F5407F529
:10C03000548014E570240BF582E4356FF583E0FE3F
:10C04000C4540F5407F554E511C4540F5407F55365
:10C05000600302C11EE554700302C11EE56E24098F
:10C06000F582E4356DF583E04480F002C11EE56E93
:10C07000240CF582E4356DF583E04440F0E51020B2
:10C08000E725E51220E710E56E240CF582E4356D16
:10C09000F583E054BFF022E56E240DF582E4356DA2
:10C0A000F583E04480F0228F74E5115407F572E5C2
:10C0B00011A2E3924875F070EFA42418F582E5F020
:10C0C0003400F58375F00EE57212D054AF8285838B
:10C0D0006F8F70304816E5822407F582E43583F5CA
:10C0E00083E0FFC4540F5407F5548014E570240B0B
:10C0F000F582E4356FF583E0FFC4540F5407F5541F
:10C10000E511C4540F5407F5537013E554600FE55F
:10C110006E240DF582E4356DF583E04480F0304700
:10C1200003437108304823E57344C0FFE5702408D9
:10C13000F582E4356FF583EFF0E5702409F582E4CC
:10C14000356FF583E04571F08021E57344C0FFE56C
:10C1500070240CF582E4356FF583EFF0E570240D63
:10C16000F582E4356FF583E04571F0909204E0B517
:10C170007413909208E0B5720CA248E433FF9091DA
:10C18000C1E06F6013856F6D85706E857473857205
:10C1900071A248924702BED322E4F566F567E567CF
:10C1A00025E0FFE56633FE74A12FF582EE341CAF67
:10C1B0008278A8F608A607F583E0FEA3E0FF4E709C
:10C1C0000302C257EE547F78B0F608A6077F5712D5
:10C1D000052B7F4912052BE566FF12058DAF67E53C
:10C1E0006712058D7F0D12052B7F0A12052B78B083
:10C1F000E6FE08E6F5828E83E06048E509D3943FC9
:10C20000400B3025F6C225D2AED2BE80EE78B00803
:10C2100006E618860670010614F5828E83E0FF128A
:10C22000058D78B00806E618860670010614F582BA
:10C230008E83E0FF12058D7F0D12052B7F0A1205FC
:10C240002B80ABE4FF12058DE4FF12058D7F0D12EC
:10C25000052B7F0A12052B0567E56770020566C38B
:10C26000E5679484E5669403500302C19E2212059B
:10C27000A7EF756700F5661205A7EF2567F567E478
:10C280003566F566C3E5679484E566940340087EE9
:10C29000C97FFD1203E222E56725E0FFE56633FE74
:10C2A00074A12FF582EE341CAF8278A8F608A60799
:10C2B000F583E0FEA3E04E60087ECA7F171203E21A
:10C2C00022302D087ECA7F321203E222C3901C1C4A
:10C2D000E09448901C1BE0942A40087ECA7F4D12CF
:10C2E00003E222901C1BE0FFA3E0901C95CFF0A37B
:10C2F000EFF0901C19E0FEA3E078ADA60608F67FEB
:10C300003F12052B7F0D12052B7F0A12052BD2330E
:10C31000221205A78F661205A78F6712055A78ADFE
:10C320000806E618860670010614F5828E83E56617
:10C33000F0E566706B901C19E0FEA3E0FF78A8E6BC
:10C34000FC08E6F5828C83EEF0A3EFF078AD0806EA
:10C35000E618860670010614F5828E83E4F078AD47
:10C36000E6FE08E6FF901C19EEF0A3EFF0F5828ED2
:10C3700083E4F0A3F0901C95F0A3F0901C1CE02443
:10C3800002F0901C1BE03400F0C2337F6F12052BCB
:10C390007F6B12052B7F0D12052B7F0A12052B22B6
:10C3A00078AD0806E618860670010614F5828E83BD
:10C3B000E567F0901C1CE02402F0901C1BE03400A8
:10C3C000F0C3A3E09452901C1BE0942A403D7ECA27
:10C3D0007F4D1203E278A8E6FE08E6F5828E83E43C
:10C3E000F0A3F0901C95E0FFA3E0901C1BCFF0A3FE
:10C3F000EFF0E4901C95F0A3F0901C19E0FEA3E090
:10C40000F5828E83E4F0A3F0C233227F3F12052B26
:10C410007F0D12052B7F0A12052B227F6E12052B32
:10C420007F6612052B901C19E0FF12058D901C19D8
:10C43000E0FEA3E0FF12058D7F2012052B7F751211
:10C44000052B7F6312052B901C1BE0FF12058D90BE
:10C450001C1CE0FF12058D7F0D12052B7F0A1205B3
:10C460002B78AB761C0876A1E4F566F567C3E56723
:10C470009484E5669403400302C54D78ABE6FE085C
:10C48000E6F5828E83E0FEA3E04E700302C5387F9E
:10C490004612052BE566FF12058DAF67E5671205AD
:10C4A0008D7F3A12052B7F2012052B78ABE6FE0814
:10C4B000E6F5828E83E0FF12058D78ABE6FE08E696
:10C4C000F5828E83E0A3E0FF12058D7F2012052BFD
:10C4D00078ABE6FE08E6F5828E83E0547FFEA3E0AB
:10C4E0008E68F569856982856883E06041E509D3D6
:10C4F000943F400B3025F6C225D2AED2BE80EE0569
:10C5000069E569AE687002056814F5828E83E0FF04
:10C5100012058D0569E569AE687002056814F5823B
:10C520008E83E0FF12058D7F2012052B80B67F0DD4
:10C5300012052B7F0A12052B0567E5677002056659
:10C5400078AC740226F618E436F602C46D7F411208
:10C55000052B7F0D12052B7F0A12052BE4F566F5DE
:10C560006774452567F582E4341CF583E0700302A7
:10C57000C6337F4112052BE566FF12058DAF67E5D7
:10C580006712058D7F2012052B7F4E12052B7F72BF
:10C5900012052B7F3D12052BE56725E0FFE566338D
:10C5A000FE741D2FF582EE341CF583E0FF12058D1D
:10C5B000E56725E0FFE56633FE741D2FF582EE3456
:10C5C0001CF583E0A3E0FF12058D7F2012052B747C
:10C5D000452567F582E4341CF583E0FF12058D7F65
:10C5E0002012052BE56725E0FFE56633FE746D2F0D
:10C5F000F582EE341CF583E0FF12058DE56725E03A
:10C60000FFE56633FE746D2FF582EE341CF583E092
:10C61000FEA3E0FF12058D7F0D12052B7F0A120588
:10C620002BE509D3943F400B3025F6C225D2AED27C
:10C63000BE80EE0567E56770020566C3E567941482
:10C64000E5669400500302C5612212055AEF24BD2D
:10C65000700302C86824FA700302C77924FA6003E1
:10C6600002C8A8E4F569E4F56875F070E569A424EA
:10C6700018F582E5F03400F58375F00EE56812D008
:10C6800054AF828583668F67E5822408F582E4359E
:10C6900083F583E020E6148F82E582240CF582E4A2
:10C6A0003566F583E020E60302C7607F4F12052B55
:10C6B0007F4912052BAF6912058DAF6812058D7F7A
:10C6C0003A12052BE5672406F582E43566F583E02A
:10C6D000FF12058DE5672407F582E43566F583E0F2
:10C6E000FF12058DE5672408F582E43566F583E0E1
:10C6F000FF12058DE5672409F582E43566F583E0D0
:10C70000FF12058DE567240AF582E43566F583E0BE
:10C71000FF12058DE567240BF582E43566F583E0AD
:10C72000FF12058DE567240CF582E43566F583E09C
:10C73000FF12058DE567240DF582E43566F583E08B
:10C74000FF12058D7F0D12052B7F0A12052BE509BF
:10C75000D3943F400B3025F6C225D2AED2BE80EE38
:10C760000568E568C39408500302C6690569E56970
:10C77000C39440500302C666221205A78F691205B2
:10C78000A78F6812055ABF3A0EE569C39440500757
:10C79000E568C3940840127ECA7F661203E2120560
:10C7A0005AEF700302C8A880F575F070E569A424FB
:10C7B00018F582E5F03400F58375F00EE56812D0C7
:10C7C00054AF828583668F671205A7E5672406F557
:10C7D00082E43566F583EFF01205A7E5672407F5D7
:10C7E00082E43566F583EFF01205A7E5672408F5C6
:10C7F00082E43566F583EFF01205A7E5672409F5B5
:10C8000082E43566F583EFF01205A7E567240AF5A3
:10C8100082E43566F583EFF01205A7E567240BF592
:10C8200082E43566F583EFF01205A7E567240CF581
:10C8300082E43566F583EFF01205A7E567240DF570
:10C8400082E43566F583EFF012055AEF640D60035C
:10C8500002C7977F6F12052B7F6B12052B7F0D127E
:10C86000052B7F0A12052B2212055AEF644C7038F3
:10C8700012055AEF6445703012055AEF6441702872
:10C8800012055AEF64527020D2077E1C7F007D0093
:10C890007B027A00791812D060C22212B2FF7F2A7E
:10C8A00012052B7F0D12052B22909209E0FEA3E0CA
:10C8B0008E59F55A909205E0F55B9091C2E0F55CD7
:10C8C000A3E024FF9243755DFF20430302C957850F
:10C8D0005A82855983E05488FFBF880FAF5AAE59FA
:10C8E000AD5BAB5CA243924712AA2BE55A2408F534
:10C8F00082E43559F583E0FF20E70302C9FCEF54D9
:10C900003FF55BE55A2409F582E43559F583E05497
:10C9100007F55C75F070E55BA42418F582E5F0344A
:10C9200000F58375F00EE55C12D054AF8285835913
:10C930008F5AE5822409F582E43583F583E0A2E38A
:10C9400092438F82E5822408F582E43559F583E02D
:10C9500030E60302C9D822855A82855983E0549073
:10C96000FFBF900FAF5AAE59AD5BAB5CA24392478D
:10C9700012AA2BE55A240CF582E43559F583E0FF21
:10C9800030E779EF543FF55BE55A240DF582E43545
:10C9900059F583E05407F55C75F070E55BA4241845
:10C9A000F582E5F03400F58375F00EE55C12D054A5
:10C9B000AF828583598F5AE582240DF582E4358351
:10C9C000F583E0A2E392438F82E582240CF582E4B2
:10C9D0003559F583E030E624909206E0FEA3E0B5F9
:10C9E0005A11E559B5060CA243E433FF9091C1E01A
:10C9F0006F6009155DE55D600302C8C922455252AA
:10CA00003A207A7520686F6865204673742D4E75DC
:10CA10006D6D65720D0A004552523A2046737420BE
:10CA2000626572656974732062656E75747A740DDF
:10CA30000A004552523A20446566696E6974696F0E
:10CA40006E20696D2047616E67210D0A00455252C4
:10CA50003A204673742D5370656963686572207659
:10CA60006F6C6C0D0A004552523A20496E76616C2B
:10CA7000696420466F726D61740D0A008E838F8227
:10CA8000790EE0F709A3E0F709A3A3A3A3A3E0F7B6
:10CA900009A3E0F709A3E0F709A3E0F7228E838F4B
:10CAA00082790EE0F709A3E0F709EF240AFF5001AD
:10CAB0000E8E838F82E0F709A3E0F709A3E0F70960
:10CAC000A3E0F72290F7007443F090F70474C3F0EA
:10CAD000A3741CF0A3E4F0A3F090F70CF0A3F09083
:10CAE000F7167408F090F7117455F090F7107495DC
:10CAF000F090F7207440F090F730F090F740F0900D
:10CB0000F750F090F760F090F770F090F780F090A9
:10CB1000F790F090F7A0F090F7B0F090F7C0F09099
:10CB2000F7D0F090F7E0F090F7F07499F0A3745517
:10CB3000F090F7F67480F090F700740AF0781D76A4
:10CB4000E022C0E0C083C082C0D0C000C00790F720
:10CB500001E0FF30E715203C12D23C90F70074034F
:10CB6000F0740AF0781A74FFF68070C23C781AE606
:10CB70007004EF5487F690F702E0FFC39402405B25
:10CB8000EFD394105055BF02047F0F80021F1FEF98
:10CB9000C454F0FFE42FF582E434F7F5837441F0D8
:10CBA000781B0674112FFFBF01027F21E42FF5824D
:10CBB000E434F7F5837455F01F74062FF582E434DE
:10CBC000F7F5837480F0E42FF582E434F7F583748D
:10CBD00099F0781CE6C394FF500106D007D000D02E
:10CBE000D0D082D083D0E0328E838F828D01E7094E
:10CBF000F0A3EB603DDBF7228C838D828F01E0F7A1
:10CC000009A3EB602DDBF7228F008D01E3F6080905
:10CC1000EB601FDBF7228F008D01E7F20809EB6064
:10CC200011DBF7228F008D01E7F60809EB6003DBCB
:10CC3000F7222275B12078FFE4F6D8FD75A0FC78C4
:10CC4000007F00E4F208DFFC7581B802CC890205A0
:10CC5000FBE493A3F8E493A34003F68001F208DF1A
:10CC6000F48029E493A3F85407240CC8C333C454B4
:10CC70000F4420C8834004F456800146F6DFE48068
:10CC80000B010204081020408090A3BEE47E0193B3
:10CC900060BCA3FF543F30E509541FFEE493A3603A
:10CCA000010ECF54C025E060A840B8E493A3FAE495
:10CCB00093A3F8E493A3C8C582C8CAC583CAF0A3E6
:10CCC000C8C582C8CAC583CADFE9DEE780BE35CBE6
:10CCD000F5CBC2C20582151475920490F00DE5578C
:10CCE00054FBF0D092D0D0D0E03235CBF5CBC2C2DD
:10CCF00005821514B29075920490F00DE557F0D0AE
:10CD000092D0D0D0E03235CBF5CBC2C2058215141B
:10CD1000D092D0D0D0E03235CBF5CB0582B2901591
:10CD20001475E00A10C213D5E0FAD092D0D0D0E04A
:10CD300032C0E0C0D0C092759201E5146024B40303
:10CD400000E0058225CAF5CAE010E7CB10E6B7354A
:10CD5000CBF5CBB290C2C205821514D092D0D0D000
:10CD6000E032E516603CE53325CAF5CAE435CBF57B
:10CD7000CBB290C2C2151680E2E55860DE15587538
:10CD80009203A310C2B1759204E0543060F575921D
:10CD900003E005E0F010C29F759204E0543070F596
:10CDA00080E1C23D20BB020556E53325CAF5CAE441
:10CDB00035CBF5CBC290C2C2303F2090EC00E005ED
:10CDC00082F514E00582F516202B0975920390EE8A
:10CDD000DF755804D092D0D0D0E03290ED00E0055D
:10CDE00082F514E00582F516D092D0D0D0E032C0A2
:10CDF000E0C0D0C092759202E515604CE005822536
:10CE0000C2F5C2E010E72710E61335C3F5C3B291AF
:10CE1000C2C305821515D092D0D0D0E03235CBF503
:10CE2000CBC2C305821515D092D0D0D0E03235C325
:10CE3000F5C3B2910582151575E00A10C3BAD5E0A5
:10CE4000FAD092D0D0D0E032E5176018E53325C291
:10CE5000F5C2E435C3F5C3B291C2C31517D092D061
:10CE6000D0D0E032C23E0556E53325C2F5C2E435E6
:10CE7000C3F5C3C291C2C330401490EE00E00582F6
:10CE8000F515E00582F517D092D0D0D0E03290EFC2
:10CE900000E00582F515E00582F517D092D0D0D0DC
:10CEA000E032E709F608DFFA8046E709F208DFFA20
:10CEB000803E88828C83E709F0A3DFFA8076E3095D
:10CEC000F608DFFA806EE309F208DFFA80668882EE
:10CED0008C83E309F0A3DFFA805A89828A83E0A376
:10CEE000F608DFFA804E89828A83E0A3F208DFFA2F
:10CEF000804280AE80B480BA80C480CA80D080DA9C
:10CF000080E480378023805389828A83ECFAE4931B
:10CF1000A3C8C582C8CCC583CCF0A3C8C582C8CC81
:10CF2000C583CCDFE9DEE7800D89828A83E493A3A1
:10CF3000F608DFF9ECFAA9F0EDFB2289828A83EC8E
:10CF4000FAE0A3C8C582C8CCC583CCF0A3C8C5820B
:10CF5000C8CCC583CCDFEADEE880DB89828A83E443
:10CF600093A3F208DFF980CC88F0ED14B4040050EC
:10CF7000C3241E83F582EB14B4050050B724158337
:10CF80002582F582EF4E60ACEF60010EE58290CE17
:10CF9000F273000402000C060012BB020689828AAA
:10CFA00083E0224003BB0402E722400789828A8390
:10CFB000E49322E322EFF88DF0A4FFEDC5F0CEA4B8
:10CFC0002EFEEC88F0A42EFE22BC000BBE0029EF42
:10CFD0008DF084FFADF022E4CCF875F008EF2FFF60
:10CFE000EE33FEEC33FCEE9DEC984005FCEE9DFE2E
:10CFF0000FD5F0E9E4CEFD22EDF8F5F0EE8420D275
:10D000001CFEADF075F008EF2FFFED33FD400798E3
:10D010005006D5F0F222C398FD0FD5F0EA22C2D512
:10D02000EC30E709B2D5E4C39DFDE49CFCEE30E7AB
:10D0300015B2D5E4C39FFFE49EFE12CFC9C3E49DA1
:10D04000FDE49CFC800312CFC930D507C3E49FFFE9
:10D05000E49EFE22A42582F582E5F03583F5832245
:10D06000EF4E6013EDBB021089828A83EF60010EE0
:10D07000EDF0A3DFFCDEFA2289F04003BB0407F7E2
:10D0800009DFFCA9F02250EFF309DFFCA9F022E749
:10D0900009F608DFFA8079E9D39850F3E92FF9E827
:10D0A0002FF819E718F6DFFA8066E709F208DFFAC9
:10D0B000805E88828C83E709F0A3DFFA8052E3095F
:10D0C000F608DFFA804AE9D398500EE92FF9E82FE5
:10D0D000F819E318F2DFFA8037E309F208DFFA8083
:10D0E0002F88828C83E309F0A3DFFA802389828A68
:10D0F00083E0A3F608DFFA801789828A83E493A38A
:10D10000F208DFF9800A89828A83E0A3F208DFFA55
:10D1100002D19580828093809980A380A980C2806B
:10D12000CC80E38077806380D0D3E998EA9C503943
:10D13000E92FF582EA3BF583E82FF8EC3BFC05820A
:10D14000D5820215831582E493C8C582C8CCC583F5
:10D15000CC0582D5820215831582F0C8C582C8CC61
:10D16000C583CCDFD9DED7802E89828A83ECFAE4AE
:10D1700093A3C8C582C8CCC583CCF0A3C8C582C858
:10D18000CCC583CCDFE9DEE7800D89828A83E49316
:10D19000A3F608DFF9ECFAA9F0EDFB22D3E998EA4F
:10D1A0009C5038E92FF582EA3BF583E82FF8EC3BF9
:10D1B000FC0582D5820215831582E0C8C582C8CCE1
:10D1C000C583CC0582D5820215831582F0C8C5823D
:10D1D000C8CCC583CCDFDADED880BC89828A83ECF8
:10D1E000FAE0A3C8C582C8CCC583CCF0A3C8C58269
:10D1F000C8CCC583CCDFEADEE8809C88F0ED14B4AF
:10D2000004005091242283F582EB14B4050050856C
:10D210002419832582F582EEFB4F700302D195EF2E
:10D2200060010EE58290D11373000402000C060029
:10D2300012FFFFFFFFFFFFFFFFFFFFFFFFFFFFFFEB
:00000001FF
